:10000000F8FF022099010000C1FB000079FB00000D
:1000100079FB000079FB000079FB000079FB000010
:1000200079FB000079FB000079FB0000C1FB0000B8
:10003000C1FB000079FB00001D1D0100211D010016
:10004000C1FB0000C1FB0000C1FB0000C1FB0000C0
:10005000C1FB0000C1FB0000C1FB0000C1FB0000B0
:10006000C1FB0000C1FB0000C1FB0000C1FB0000A0
:10007000C1FB0000C1FB0000C1FB0000C1FB000090
:10008000C1FB0000C1FB0000C1FB0000C1FB000080
:10009000C1FB0000C1FB0000C1FB0000C1FB000070
:1000A000C1FB0000C1FB0000C1FB0000C1FB000060
:1000B000C1FB0000C1FB0000C1FB0000C1FB000050
:1000C000C1FB0000AD060100C1FB0000D10D010025
:1000D000C1FB0000C1FB0000C1FB000075930000E4
:1000E000C1FB0000C1FB0000C1FB0000C1FB000020
:1000F000C1FB0000C1FB0000C1FB0000C1FB000010
:10010000C1FB0000C1FB0000C1FB0000C1FB0000FF
:10011000C1FB0000C1100100C1FB0000C1FB0000D9
:10012000C1FB0000C1FB0000C1FB0000C1FB0000DF
:10013000C1FB0000C1FB0000C1FB0000C1FB0000CF
:10014000C1FB0000C1FB0000C1FB0000C1FB0000BF
:10015000C1FB0000C1FB0000C1FB0000C1FB0000AF
:10016000C1FB0000C1FB0000C1FB0000C1FB00009F
:10017000C1FB0000C1FB0000C1FB0000C1FB00008F
:10018000C1FB0000C1FB0000C1FB0000C1FB00007F
:10019000C1FB0000C1FB0000584B4CF2205210B5CF
:1001A0001A804DF628121A8000BF00BF0FF00CFD18
:1001B000534B4FF030621A60524A9A60524ADA60EA
:1001C000524B4FF470021A60514A136813F4807353
:1001D00004D150490B604FF4A85313604E4B1A786A
:1001E000110703D51A7842F008021A704B4B4C499C
:1001F0002A221A704B4A4C4B8B4204D252F8040FFD
:1002000043F8040BF8E7494B494900228B4202D2DC
:1002100043F8042BFAE74749474A002352F82300E2
:1002200041F823000133662BF8D1444B444A802126
:1002300003F8011B9342FBD1424B3E4A1A60424BEA
:100240008A221A70A3F5805324225A70A0221A70B1
:100250009A799207FCD59A79D406FCD43B4A9379D3
:1002600003F00C03082B394BF9D103221A714622F3
:100270005A719A799006FCD5344A9179334B4906E4
:10028000FBD5334A4FF08271116009215160202261
:100290001A709A7902F00C020C2AFAD12D4B2E4AD0
:1002A0001A602E4B2E4A1A6000225A60072243F829
:1002B000042C2C4AC3F80C2D62B60FF09FFD154B91
:1002C0001B68DA0705D528480FF01CFD274B284A84
:1002D0001A60284B1B785B0609D5244C244B2268F6
:1002E0009A4204D120480FF00DFD002323600FF047
:1002F00071FC13F01BFC11F08BFEFEE70E20054095
:1003000030800440823F04000100002B88ED00E0B3
:1003100010D0034014D0034002D0074000E0074053
:100320007C19FF1F489E0100F806FF1F8019FF1F60
:10033000200600200002FF1F0000000000E400E093
:1003400056E400E008ED00E00050064000400640A2
:100350004480044004800440C010050014E000E024
:10036000BFD4010000002020B18440621CE00340A3
:10037000A5C3945A00F00740FFFFFFFFFFFFFFFFF8
:10038000FFFFFFFFFFFFFFFFFFFFFFFFFFFFFFFF7D
:10039000FFFFFFFFFFFFFFFFFFFFFFFFFFFFFFFF6D
:1003A000FFFFFFFFFFFFFFFFFFFFFFFFFFFFFFFF5D
:1003B000FFFFFFFFFFFFFFFFFFFFFFFFFFFFFFFF4D
:1003C000FFFFFFFFFFFFFFFFFFFFFFFFFFFFFFFF3D
:1003D000FFFFFFFFFFFFFFFFFFFFFFFFFFFFFFFF2D
:1003E000FFFFFFFFFFFFFFFFFFFFFFFFFFFFFFFF1D
:1003F000FFFFFFFFFFFFFFFFFFFFFFFFFFFFFFFF0D
:10040000FFFFFFFFFFFFFFFFFFFFFFFFDEF9FFFF23
:1004100010B5054C237833B9044B13B10448AFF33E
:1004200000800123237010BD8019FF1F0000000011
:100430004C9E0100084B10B51BB108490848AFF3AA
:1004400000800848036803B910BD074B002BFBD0A0
:10045000BDE81040184700BF000000008419FF1FCE
:100460004C9E01007C19FF1F00000000F8B50546F6
:100470000C4600F08DFA214605F5987000F00AFE52
:1004800005F5CC7600213346A5F88C11C5F89011FE
:10049000C5F8941105F5097423F8021B9C424FF02E
:1004A0000002F9D105F50E770024C5F82422A5F83D
:1004B000282285F82A22A5F82C22C5F83022C5F872
:1004C00034223B4605F5227143F8044B8B424FF032
:1004D0000002F9D1002301201146C5F88C22C5F88D
:1004E000902285F8883285F8943285F8890205F5DE
:1004F000267305F52B7243F8041B93424FF000045A
:10050000F9D10023A5F8AC3285F8AE32A5F8B032A7
:10051000A5F8B23285F8B4320B2011F081FD4FF00E
:10052000300E0E490E4BC5F824020722C5F8906123
:10053000C5F83072C5F89842C5F89C42C5F8A0428B
:10054000C5F8A442C5F8A842A5F88CE1C5F89411F5
:10055000A5F82C22C5F834322846F8BD1407FF1F31
:10056000F806FF1F38B5B0F8AC52052D40D0B0F8F2
:10057000B0225208A0F8B022D1B9B0F8B23290F847
:10058000AE42A0F8AC1201339BB2A0F8B2320546DD
:1005900004B37E2A49D0FE2A32D10024A0F82C418F
:1005A00080F8B44280F8AE42A0F8B242204638BD8E
:1005B00090F8AE42B0F8B2320133013542F0800219
:1005C0009BB2A0F8AC52A0F8B022A0F8B232054617
:1005D000002CDED190F8B41201291BD00229E5D1FC
:1005E000082BE3D1114600F0E5F9A5F8B242DDE7AA
:1005F00049B1B0F8B0220124E24080F8AE42D9E718
:100600000024204638BD0C4680F8AE12A0F8AC128B
:10061000204638BD082BC9D10223114680F8B432D8
:1006200000F0C8F9A5F8B242C0E7B0F82C31102BA1
:100630000DD80020A5F82C0100230122044685F8DE
:10064000B42285F8AE32A5F8B232204638BD00F0AB
:10065000BFF90028EDD0EFE700F5987000F034BD49
:10066000D0EDA47A9FED0C7AF4EEC77AF1EE10FA91
:100670000DD9B0EE087AF4EEC77AF1EE10FAA9BF00
:10068000002390F8940280F89432184670470123B2
:1006900080F89432184670479999193F90EDA67AE0
:1006A000DFED206AD0F89C32D0F8A0221E49F0EE8F
:1006B000407AE6EEC77A10B4C0F8A03200230433C3
:1006C000D0F8A442C0F8A842102BC0F8A42280EDB4
:1006D000A77A00F52872C0EDA67A0AD0F1EC016A7B
:1006E000B2EC017AE6EEC77A0433102BC0EDA67A9D
:1006F000F4D100F527739FED0D7A9FED0D0A0D4A99
:1007000000F52B709842A7EE270A08D0F3EC017A87
:1007100092ED017A04329842A7EE270AF6D15DF8ED
:10072000044B7047819231C03C4601003D2C8D3A0C
:10073000000000004846010010B590F888322DED09
:10074000028B8B4282B0044650D090EDA37A80F8A1
:100750008812F2EE047AB4EEE77AF1EE10FA90F82D
:1007600089323CDCDFED337A112BB1EE048A38BFDD
:10077000B0EE678A07EE903AF8EE677A0123C7EE8B
:10078000276A01AA694604F50B70CDED006A12F0E4
:1007900099FD9DED000AB5EEC00AF1EE10FA204673
:1007A0004CBF38EE400A38EE000AFFF777FFDDED68
:1007B000016AD4EDA37A84EDA40AB6EE007AE6EEDF
:1007C000C77A012384F889320020B7EE007A77EEE9
:1007D000877AC4EDA37A02B0BDEC028B10BDF3EEB4
:1007E000047A37EE677A84EDA37ABBE790F8893212
:1007F000102B0BD990EDA37AF2EE047AB4EEE77ADF
:10080000F1EE10FAEBDCB1EE048AB3E7D0EDA37A97
:10081000B2EE047AF4EEC77AF1EE10FA08DD013395
:10082000B3EE047A80F8893277EEC77A0120CCE7FC
:100830000020CAE7000000002DE9F04F85B001AEAE
:10084000154604461F4600F598703246022300F014
:1008500039FC002D67D0D4F824C2B4F828324FF008
:10086000000E02A936F81E001CF80320C043C0F396
:10087000C03042400CEB03085200013A01339BB2F6
:1008800088F8000021F81E200EF1010E0B2B5FFAF4
:100890008EF228BF00239542E4D80DF10C0AA4F88B
:1008A00028325246022304F5C67012F0B1FA4FF016
:1008B0000008C146C3463AF81860F643C6F3C0368E
:1008C00031462046FFF738FF68B194F82A1284F8C1
:1008D0002A62891BB1FA81F120464909B9F1000F5A
:1008E0000BD0FFF73FFE08F101085FFA88F39D4245
:1008F000E1D8484605B0BDE8F08FFFF733FE8146EA
:100900000028F0D04FF49672214638460FF060F878
:10091000B4F82C21B4F82E31A7F82E31A7F82C21E9
:10092000A4F82CB1DFE704F5C670022303AA02A9DC
:1009300012F06EFAA946484605B0BDE8F08F00BF38
:1009400070B4034600F59676002503F8015BB342C8
:100950004FF00004F9D1A0F82C41A0F82E41A2B12B
:10096000551EADB2013505444A1E034600F5957685
:1009700001E0B34209D00134A4B2A0F82C4112F82E
:10098000011F03F8011BAB42F3D170BC704700BFDD
:1009900010B4034600F59674002103F8011BA3422E
:1009A0004FF00002F9D1A0F82C21A0F82E215DF81B
:1009B000044B7047B0F82C31B3F5967F024605D052
:1009C000581CA2F82C010120D15470470020704718
:1009D00070B4B0F82C51AC1E25D0144E4FF0FF313E
:1009E0000023C25C4A40D2B2013336F81220C1F370
:1009F00007219BB24A40A3421146F2D3D14389B2A8
:100A0000025DCBB29A4202D0002070BC7047054410
:100A1000C1F3072315F8012C9342F5D1A0F82E114C
:100A200070BC012070472146EAE700BF5C46010028
:100A300070B4B0F82C511DB36C1E134E4FF0FF3242
:100A400010FA84F4411E11F8013F5340DBB2C2F3A7
:100A5000072236F813308C4283EA02031A46F2D199
:100A6000DA43A91C6B1C92B289B29BB2C2F3072471
:100A7000A0F82E214255A0F82C11C45470BC704728
:100A80002A4601230221F1E75C4601002DE9F041ED
:100A90000646002300F10C07384633807360B360CC
:100AA00006F5A67220F8023B90424FF00004F9D1FF
:100AB0000321FFF7DBFC062106F20440FFF7D6FC1A
:100AC000092106F2BC60FFF7D1FC1E234FF080081D
:100AD0004FF0010C4021B322C6F87C390F234FF0B0
:100AE000820E0E4886F8848986F887C986F88819A8
:100AF00086F8892986F88A39B060A6F87449C6F85C
:100B00007849C6F8804986F8854986F8864977602D
:100B1000A6F800E03046BDE8F08100BF7407FF1F73
:100B20002DE9F0410446CEB01546022301AA12F089
:100B30006FF9D4F878390133C4F8783902A804F58C
:100B4000A678FFF725FF404602AB2A4601A9FFF72A
:100B500073FEB0B1BDF83631B4F874299A425CD056
:100B6000BDF83421A4F87439023A002392B2C4F8D3
:100B7000783902A95D480DF089FD5D495B480DF0AB
:100B800081FF04F20447384602AB2A4601A9FFF769
:100B900053FEB0B1BDF83631B4F874299A4241D051
:100BA000BDF83421A4F87439023A002392B2C4F893
:100BB000783902A94D480DF069FD4E494B480DF0BA
:100BC00061FF04F2BC662A4601A9304602ABFFF77A
:100BD00033FEB0B1BDF83631B4F874299A4226D04C
:100BE000BDF83421A4F87439023A002392B202A964
:100BF000C4F878393D480DF049FD3F493B480DF0B8
:100C000041FFD4F88039D4F87C2902339342C4F8E8
:100C1000803911D24EB0BDE8F081D4F87829022A8B
:100C2000ABD99DE7D4F87829022AC6D9B8E7D4F819
:100C30007829022AE1D9D3E70023C4F88039404655
:100C4000FFF70EFD05463846FFF70AFD074630461A
:100C5000FFF706FD06469DB194F8853953B9012189
:100C6000264807F0BBFD0121244807F0C3FD0123FE
:100C700084F88539002384F886394EB0BDE8F081C8
:100C8000002FE9D10028E7D194F8853913BB94F8F7
:100C9000870994F88A3994F8882994F8891994F87E
:100CA00084590130C0B25A4042401144C9B203EBEA
:100CB00051035340DBB29D4234BF0025012584F827
:100CC000870984F8882984F88A3984F8891984F88E
:100CD00086599FE70146094807F080FD31460748DD
:100CE00007F088FD84F88569D1E700BFF04CFF1F4D
:100CF0005C480100704801008448010058A5FF1FAE
:100D000090F88609704700BF2DE9F041CEB20F463A
:100D1000F11E054649B200F5A67014469846FFF745
:100D20009BFC394605F20440FFF796FCF11C49B2E2
:100D300005F2BC60C4EB0414FFF78EFC240185F8B7
:100D40008489C5F87C49BDE8F08100BF10B4034632
:100D500000F51674002103F8011BA3424FF00002B6
:100D6000F9D14FF4B473A0F85822A0F85A22A0F891
:100D70005E2280F86022A0F85C325DF8044B704778
:100D80002DE9F04FCDB004466846FFF7D9FD68461F
:100D9000FFF74EFEB4F85C720022A4F85822A4F8C3
:100DA0005A2284F86022A4F85E22002F00F0E58029
:100DB000754E134620254FF0400E802111E014F8A7
:100DC0000C000143C9B201321FFA82F808F1020097
:100DD000474500F0070004F80C1010D97146AE46E4
:100DE000355C83F0010313F0FF034FEAE20CE6D118
:100DF0004FEAE20C14F80C0020EA0101E3E7A4F842
:100E0000587284F86032DFF880C17A1C07F1090A51
:100E10006646E14692B21FFA8AFA8020511E89B2D4
:100E200010F07E0F4FEAE10804D183F00103DBB23A
:100E300084F8603293B114F808104EEA0101C9B287
:100E4000013292B2924502F0070B04F808100CD060
:100E5000AE4619F8010F16F80B50DFE74FEAE1082C
:100E600014F8080020EA0E01EAE70837BDF82C2143
:100E7000BFB2A4F858724FEAC208002A00F082807C
:100E80000021DFF808918E46012018E015437A1CF6
:100E900004F80A5092B250B30EF1010E5FFA8EFEC2
:100EA000BEF1050F49D0013189B2884524D901F03E
:100EB000070002F0070519F80000755D1746CA1013
:100EC0001DF80220104004D183F00103DBB284F846
:100ED00060324FEAE70A14F80A20002BD6D122EA42
:100EE00005057A1C04F80A5092B20028D4D10131C9
:100EF00089B288458646DAD802F00701A4F858225C
:100F0000755C02F10807BFB2802111F07E0F4FEA35
:100F1000E20004D183F00103DBB284F86032F3B164
:100F2000215C0D43013292B2974202F00701255431
:100F30001AD0755C1CF8011FE7E783F00103D51098
:100F4000DBB202F0070284F86032605DB25C8BB104
:100F50001043BA1C92B260554FF0000EA3E7D010B8
:100F6000215C21EA0505DDE70020A4F858724DB0A8
:100F7000BDE8F08F20EA0200EBE740254FF0800E3D
:100F80003B4640E73A46BCE798480100A0480100CC
:100F9000F0B58DB0144F0DF106040DF12E060BE0E7
:100FA000AD10A0F85E32772B24F8025F84BF783B47
:100FB000A0F85E32B4420DD0B0F85E22931D9BB211
:100FC00037F912500029EBD102F10B039BB2A0F8C4
:100FD0005E32E8E70023009302AA14230B210348A2
:100FE00007F014FB0DB0F0BDA848010058A5FF1F85
:100FF000B0F8583283B31C4B1B7870B5044613B954
:10100000B0F85A324BB3194807F0C0FB1428054614
:1010100029D9B4F85A32164E01E0142D1BD9D91033
:1010200003F00702615CB25C01331142A4F85A324A
:1010300014BF012100212046FFF7AAFFB4F85A325D
:10104000B4F85822143D9A42ADB2E6D80023A4F871
:101050005A32A4F8583270BD70470648FFF750FE68
:101060000028D0D170BD70BD540EFF1F58A5FF1FC2
:101070009848010018F5FF1F01EB41018900A0F815
:101080005C127047B0F8580200280CBFFF20002007
:10109000704700BF30B400F10C052B4600F15C0432
:1010A000002223F8022B9C42FBD18B1DDBB2044AA9
:1010B000456052F8233083600923038030BC7047B9
:1010C0007C09FF1F11F0A4BE0346063110B4C9B25B
:1010D0000924054A23F80C4B52F821208260436012
:1010E0005DF8044B704700BF7C09FF1F10B4034636
:1010F00000F57A74002103F8011BA3424FF00002AF
:10110000F9D1A0F8E823A0F8EA2380F8EC235DF8F1
:10111000044B7047B0F8E83303B97047F0B50446A4
:1011200083B0224807F032FB182805463CD9B4F8B2
:10113000EA331F4E1CE0CDF800E007F067FA94F8A0
:10114000EC330133DBB2183D312B84F8EC33ADB214
:10115000B4F8EA3306D901339BB20022A4F8EA338B
:1011600084F8EC23B4F8E8239A4218D9182D1BD937
:10117000DA1003F00703A15CF75C0E4A0B480F403E
:101180004FF0000E4FF018034FF06101D3D10097DC
:101190001823094A0548612107F038FACFE70023F0
:1011A000A4F8EA33A4F8E83303B0F0BD58A5FF1F54
:1011B000C44B0100400AFF1F9C19FF1F2DE9F84F87
:1011C00004460E46154600214FF47A7212F09EFF37
:1011D0004FF0000E0822A4F8E823A4F8EAE384F80C
:1011E000ECE3002D63D0DFF8E880364F40F2E23CBC
:1011F00016F80EA0BAF1410F5FD00120422104E0A1
:101200008A451CD017F829101846431CDBB203EBA3
:1012100043090029F4D10EF1010E5FFA8EFEAE45AE
:10122000E6D3082A43D0053292B2A4F8E82326492F
:10123000264812B20DF02CFC0020BDE8F88F00EB20
:10124000400307EB83031F491B7A002BE3D000EB1D
:10125000400001EB8000013B02F1010959FA83F9DA
:10126000D0F804A01FFA89F94FF0004011E018F8F7
:1012700003B0635C23EA0B0302F1010B6245635484
:101280001FFA8BF24FEA500011D84A45A4F8E82320
:10129000C1D030EA0A0B4FEAE20102F00703E6D1BF
:1012A0009B46635C18F80BB04BEA0303E4E70023AA
:1012B000A4F8E8330420BDE8F88F02490823002091
:1012C000C5E700BFB449010098490100F04CFF1F79
:1012D000C44B01000023A0F8E833A0F8EA3380F8FB
:1012E000EC33704738B505460022083003462A70B3
:1012F0006A706A6005F12A0403F8012BA3424FF0DB
:101300000001F9D185F82A10222202490EF060FB73
:10131000284638BDC04C0100114AC1EBC101531829
:10132000F0B5515C867D9A79057F5C78C47522F0B2
:101330000F0201F00F0405F00F0526F00F01214305
:1013400093F802E0DF781E795C79817545EA020343
:1013500080F818E047768676C4760377F0BD00BF44
:10136000CC4B0100114AC1EBC1015318F0B5515CDF
:10137000867D9A79057F5C78C47522F00F0201F0B2
:101380000F0405F00F0526F00F01214393F802E04A
:10139000DF781E795C79817545EA020380F818E0F0
:1013A00047768676C4760377F0BD00BF4C4C0100CB
:1013B00010B50446304802F099FE2F4802F064FC54
:1013C00048B16378013B032B03D8DFE803F0182D05
:1013D00040050023637010BD274802F001FF6368D9
:1013E0001E339842F7D90021234802F0C5FB22485A
:1013F00002F0F0FE002384F82A30637010BD012152
:101400001D4802F0CFFE09221C491B4802F060FB78
:1014100022221B49184802F0F3FA0121164802F073
:10142000ABFB0223637010BD94F82A102046FFF72F
:1014300073FF222204F108010F4802F0E1FA94F848
:101440002A30052B0FD0013384F82A3010BD222218
:101450000C49094802F0D4FA074802F0C1FE0423FF
:101460006060637010BD2378002284F82A20002B6E
:10147000B1D10323637010BDB078FF1F404C010051
:101480009C4C0100F84B010010B504461F4801F0C8
:10149000D1F91E4801F06CFA50B16378022B08D0E4
:1014A000032B21D0012B17D00023637084F82A303E
:1014B00010BD94F82A102046FFF754FF222204F1B1
:1014C0000801124801F032F994F82A30052B13D0A4
:1014D000013384F82A3010BD22220D490B4801F057
:1014E00025F90223637010BD22220A49074801F042
:1014F0001DF90023637010BD2378002284F82A2090
:10150000002BD5D10323637010BD00BFA8FEFF1FC1
:101510001C4C0100784C010008B5124B1B785C3B59
:10152000062B18D8DFE803F013170F041717040071
:10153000017889B10C48012102F02CFB0A48BDE872
:10154000084002F0D3BDBDE80840FFF731BFBDE859
:101550000840FFF799BF08BD0348BDE8084002F006
:1015600019BB00BFAC78FF1FB078FF1F012A01D064
:10157000042070470A78012A0CBF0123002303705E
:1015800009D143783BB90649097801F0FD015C298E
:1015900003D01846704700207047427018467047C5
:1015A000AC78FF1F002210B402600271826000F16B
:1015B0000C0300F13C0423F8022BA3424FF000017E
:1015C000F9D180F83C105DF8044B7047F0B58368A2
:1015D00000294FEA4303B8BF43F001038360064686
:1015E00090F83C00421C06EB4000D2B286F83C204A
:1015F000172A8181334888BF002223F07F4388BFA8
:1016000086F83C2083B058400DF094FB022813D894
:101610002D4806F10A0306F13A014FF47A5433F9E2
:10162000022F9042B8BF10469442A8BF1446994278
:10163000F5D1031B052B32DCB368244823F07F432C
:1016400058400DF077FB022813D81F4D06F10A030E
:1016500006F13A014FF47A5433F9022F9542B8BF9C
:1016600015469442A8BF14469942F5D12B1B052B71
:1016700001DC03B0F0BD80232F122612052269463B
:1016800013488DF802508DF801708DF804408DF8E4
:1016900003608DF800300DF09DF903B0F0BD071226
:1016A000251200238DF802000522694608488DF8AE
:1016B00001708DF804408DF803508DF800300DF066
:1016C00089F9B9E768B4AA0080C1FFFF974B5500BC
:1016D000F04CFF1F6AB370B5561EB6B2044601EB5C
:1016E00046068D1E02E0B54223601FD035F9021F69
:1016F0002379C80F83421AD02368B3F5004F03F251
:10170000991224BF6FF4CC729A18226002F54C53E0
:101710003333B3F5803F2071E5D3A2F54C42CD3A87
:1017200022602046FFF752FFB542DFD170BD22682C
:10173000ECE77047002202704280704710B5044603
:1017400084B0C74803F00AFF23780BB904B010BD7A
:10175000C34803F0A9FE0428F8D9C24B01AA03F13B
:101760000B009E2101E013F8011F02F8011B8342C8
:10177000F9D16288BC48A2FB0001531A01EB530364
:101780001B0903EB4303C3EBC303D31A9BB2002B28
:1017900041D0012A5CD0022A50D0032A62D0042A08
:1017A0006AD0052A72D0062A7AD0072A00F08280F1
:1017B000082A00F08980012B00F09080022B00F0B5
:1017C0009780032B00F09E80042B00F0A580052B52
:1017D00000F0AC80062B00F0B380072B00F0B8803F
:1017E000082B00F0D480092A00F0AC80092B00F00F
:1017F000EC800A2A40F0C0800B2B00F0A7800C2B55
:1018000040F0CF803D210222D7238DF80D108DF8B6
:101810000E208DF80F3001A90C22914803F08AFCAC
:101820006188924B01314A08A3FB0232120A40F24E
:10183000762303FB1213638004B010BD34211922F8
:10184000DE238DF80D108DF80E208DF80F30E2E7B5
:1018500030210222DE238DF80D108DF80E208DF838
:101860000F30D8E731216F22DE238DF80D108DF86F
:101870000E208DF80F30CEE71F212B22F6238DF896
:101880000D108DF80E208DF80F30C4E73221222282
:10189000B3238DF80D108DF80E208DF80F30BAE7B8
:1018A00024212A22E0238DF80D108DF80E208DF8CA
:1018B0000F30B0E733213B22B3238DF80D108DF8A4
:1018C0000E208DF80F30A6E750216F22B3238DF83C
:1018D0000D108DF80E208DF80F309CE725214F223A
:1018E00093238DF80D108DF80E208DF80F3092E7B0
:1018F00070210B22DA238DF80D108DF80E208DF853
:101900000F3088E725211D22D6238DF80D108DF884
:101910000E208DF80F307EE733211B22B3238DF884
:101920000D108DF80E208DF80F3074E725216F22F1
:10193000D7238DF80D108DF80E208DF80F306AE743
:101940003921E0E70A2B0DD00B2B60D12521BCE714
:1019500025210C22C7238DF80D108DF80E208DF84F
:101960000F3058E721210C22C2238DF80D108DF87D
:101970000E208DF80F304EE70A2BF3D00B2A2ED114
:101980000C2B3FF43FAF0D2B3BD1252157E75021C6
:101990006F22D0238DF80D108DF80E208DF80F30AA
:1019A00039E70D2BF1D00E2A2BD10F2B39D0102B6C
:1019B00041D0112B49D016212922F5238DF80D1085
:1019C0008DF80E208DF80F3025E725211E22D0231B
:1019D0008DF80D108DF80E208DF80F301BE70B2BB6
:1019E000B4D00C2A13D10D2BCFD00E2B3FF46CAFFB
:1019F0000F2B16D0102ADCD0102B1CD0112AD8D1D6
:101A0000D9E70E2B3FF460AF0F2AD0D0F0E70C2BB4
:101A10003FF4F8AE0D2AC4D10E2B3FF455AF0F2B77
:101A2000EAD125211B22D6238DF80D108DF80E202A
:101A30008DF80F30EFE623211B223A238DF80D108D
:101A40008DF80E208DF80F30E5E621212522F523B3
:101A50008DF80D108DF80E208DF80F30DBE600BFED
:101A6000C01DFF1F104D010087611886D1000DD0E9
:101A7000012A01D00420704738B50B78012B0446A9
:101A80000CBF01250025037803D05BB92570002029
:101A900038BD002BFAD1438029220449044803F0C1
:101AA000F7FAF3E7024803F095FBEFE7E44C010097
:101AB000C01DFF1F00224FF4C061018102804280DF
:101AC00042608272C2720273704700BF2DE9F0411A
:101AD0003E4F027B3B789A4282B0054644D0663B3B
:101AE000052B70D8DFE803F05B5F63676B0340F69C
:101AF000BF11018040F6BF12914235484FF00003FC
:101B000006D00133062B31D030F833209142F8D182
:101B10002F4EDBB216EBC30628D0686873886B8043
:101B200010B110F07FFA6B88580010F079FA6B88CA
:101B30006860BBB10024A046404611F099FFB5F99A
:101B40000830726883FB0001C30F43EA41036968F0
:101B500003F30F0321F8143001346B88A4B2A342BD
:101B60009044E9D83B782B73AB7A13B902B0BDE847
:101B7000F081184806F00AFE6B8883420446F5D2CD
:101B800000266A6839781348009606F03FFD6B8896
:101B9000E41AA4B2A342F4D302B0BDE8F0814FF43A
:101BA0006F710180A6E740F20F410180A2E740F289
:101BB000DF4101809EE740F2616101809AE740F6D3
:101BC0001F01018096E70021018093E7AC78FF1F99
:101BD0001C4D010058A5FF1F012A01D004207047A9
:101BE0000B78A3F10103B3FA83F35B09837200203E
:101BF000704700BF00220270704700BF10B5044656
:101C0000084808F08BF9237803B910BD054808F09F
:101C100047FA0128F9D9312203490248BDE81040AA
:101C200008F0E2B8B073FF1F4C4D0100012A01D04B
:101C3000042070470B78A3F10103B3FA83F35B0927
:101C400003700020704700BF002202704270827053
:101C5000704700BF10B50446114809F099F81048C4
:101C600009F068F928B16378012B03D00023637071
:101C7000A37010BDA3780B490948C3EBC303C3EBA2
:101C8000C3031944312208F0D7FFA3782278013327
:101C900003F00303A370002AEBD1627010BD00BFF4
:101CA000B42AFF1F804D0100012A01D00420704793
:101CB0000A78012A0CBF01230023037004D1437862
:101CC00013B9427018467047002070470022027016
:101CD0004270704710B5044611480AF095F8104854
:101CE0000AF05AF860B16378012B0AD0022B10D1A8
:101CF000D9220C490A4809F06FFF237863B9637051
:101D000010BDD9220849064809F066FF0223637016
:101D100010BD00236370F3E70123637010BD00BFA3
:101D20009C79FF1F4C0BFF1F700AFF1F012A01D077
:101D3000042070470A78012A0CBF01230023037096
:101D400004D1437813B94270184670470020704799
:101D500000220270704700BF08B5037803B908BDC0
:101D6000054806F013FDA528F9D9AA210348BDE8C6
:101D700008400AF0B1B900BF58A5FF1F6471FF1FEA
:101D8000012A01D0042070470B78A3F10103B3FAB4
:101D900083F35B0903700020704700BF00224FF6F9
:101DA000FF7101810260426042817047002A48D081
:101DB0002DE9F043561EB6B283B0044601EB460649
:101DC0008D1E45F6BF5701E0AE4237D035F8022FE1
:101DD000618963689142218938BF628191421344CD
:101DE00088BF2281226863600132BA422260EBD947
:101DF000B3FBF2F3B4F80AC0B4F808E08DF805308C
:101E00004FEA1C29C3F307234FEA1E2806220D4878
:101E10008DF8043069468DF801C08DF800908DF87A
:101E200003E08DF802800CF001FE00234FF6FF72F4
:101E3000AE422360636063812281C7D103B0BDE8F5
:101E4000F0837047F04CFF1F034600F1140100229D
:101E500043F8042B8B42FBD130B400F654350024F8
:101E600023F8024BAB424FF00002F9D142F20F735C
:101E700000F5B554A0F85C3BA0F8542BA0F8562B05
:101E8000A0F8582BA0F85A2BC0F8602BA0F8642BB0
:101E9000A0F8662BA0F8682BA0F86A2BA0F86C2B92
:101EA000A0F86E2BA0F8702BA0F8722B80F8742B82
:101EB00080F8752B80F8762B80F8772B80F8782BBC
:101EC00080F8792B80F87A2B1C3400F67C3323F8C9
:101ED000022B9C42FBD130BC704700BF002342F272
:101EE0000F72A0F85C2BA0F8583BC0F8603B80F85C
:101EF000753B80F8763B80F8783BA0F85A3B7047FA
:101F00002DE9F047BDF82050BDF924C0BDF9288067
:101F1000002A6CD0013A05F1040ED2B2AE1C0EEBD1
:101F200042020135334F1FFA8CFC1FFA82FEB6B213
:101F3000ADB2C8F1000924E04FEAE20A02F007025C
:101F400013F80A40BA5C24EA020203F80A20EA10F5
:101F500005F0070A9C5C17F80AA04AEA04049C549E
:101F60004A1D92B2B2F5B46F06F1020628BFA1F283
:101F70009B51B6B22CBF89B211460235B645ADB2FF
:101F800035D000EB4104B21EA48ACCEB040424B289
:101F90004C4592B2D0DB002C1FDB444513DA4FEAEC
:101FA000E20A02F0070213F80A40BA5C224303F87F
:101FB0000A20EA1005F0070A9C5C17F80AA024EA38
:101FC0000A049C54CCE7D41002F0070213F804A0D2
:101FD000BA5C42EA0A021A55B9E74FEAE20A02F08D
:101FE000070213F80A40BA5C24EA0202DFE7BDE800
:101FF000F08700BFDC4F01002DE9F04F0546A348F4
:10200000B5F8543B55F8233089B023F07F4358404E
:1020100004910CF08FFEC31EDBB2122B40F207813D
:10202000B5F8569BDFF878E2994F09F22D5189B245
:10203000B1F5B46F0646974826BFA9F1730292B274
:102040000A4600F1180A4FF47A5C002405EB4203BB
:10205000B3F914309F42B8BF1F469C45A8BF9C46A9
:10206000022E94BF90F900B09EF900B0BBF1010FB1
:1020700000F0E080BBF1030F00F0DE80BBF1FF3F1A
:1020800001D003EB43031C44531D9BB2B3F5B46F63
:1020900028BFA2F29B5200F101002CBF92B21A4657
:1020A00082450EF1010ED1D1D5F8603B9C4240F340
:1020B000BE800CEB070A4FEA6A0ACAEB070844F62F
:1020C000314303FB08F848F3CF33B1F5B46F059300
:1020D00028BFA9F17301059B02934FF004020FFA88
:1020E0008AFA0DF1180928BF89B20092CDF804A030
:1020F0004B4618222846FFF703FF022E4FF0000838
:1021000043D94746DFF89CB1634E07204FF00F0ECE
:1021100003E01BF801EF16F8010F19F808100EEA9A
:10212000010148400CF000FE08F101083844B8F104
:10213000070FC7B2EDD1032F79D8049B002B00F015
:102140009280059AA5F8722B0023A5F8702BA5F8AC
:102150006E2BA5F86C2BA5F86AABA5F868ABA5F8B3
:1021600066ABA5F864AB85F8743BB5F8563BC5F88B
:10217000604B03F21A4292B22021B2F5B46FA5F877
:10218000583B85F8751B44D341E0DFF818B1434E46
:1021900047460D204FF00F0E03E01BF801EF16F835
:1021A000010F19F808100EEA010148400CF0BCFDBF
:1021B00008F101083844B8F1070FC7B2EDD1032F79
:1021C00035D8049B002B3BD0059AA5F8722B002331
:1021D000A5F8702BA5F86E2BA5F86C2BA5F86AABAB
:1021E000A5F868ABA5F866ABA5F864AB85F8743BB9
:1021F000B5F8563BC5F8604B03F21A4292B2402143
:10220000B2F5B46FA5F8583B85F8751B01D3A3F55B
:10221000C372A5F85A2B03F20D1292B2B2F5B46F45
:102220002ABFA3F29343A5F85C2BA5F85C3B09B049
:10223000BDE8F08FE41A27E703EB4303E41A23E732
:1022400095F8743BBDF8141005EB43020133DBB283
:10225000032B88BF9DF81030A2F86C1BA2F864AB6A
:1022600085F8743BC4E795F8743BBDF8141005EB92
:1022700043020133DBB2032B88BF9DF81030A2F874
:102280006C1BA2F864AB85F8743B6EE76E28760091
:1022900080C1FFFFE44F01004C4E0100544E01008D
:1022A0005C4E0100444E010080F8771B704700BF70
:1022B000B0F85A3B3C33F0B40A469BB24FF4077473
:1022C000002600EB43015D1CADB2B1F87C7B013C04
:1022D000B5F5B46FA3F29F53A4B23E442CBF9BB29A
:1022E0002B46002CEDD1084B0848A3FB06135B0AD4
:1022F000C3F3072182F8233082F82210242301211E
:10230000F0BC0BF0F7BE00BF49D6B9F2F04CFF1F8E
:10231000F0B5B0F8565B00EB450300299982A3F8AD
:102320007C2BB0F8542B50F822304FEA4303B8BF4F
:1023300043F0010340F8223090F8783B8FB0044618
:10234000002B00F0A380B0F8581B01F29F539BB202
:10235000B3F5B46F01F1010292B224BF01F1FF3372
:102360009BB2B2F5B46F24BFA1F29F5292B29342D6
:1023700022D3AB4224D9AA4222D2B4F85C3BAB426E
:1023800028D094F8780B003018BF01200135ADB289
:10239000B5F5B46F24BF0023A4F8563BB4F8543B02
:1023A00038BFA4F8565B01339BB2042B88BF0023CF
:1023B000A4F8543B0FB0F0BDAB42DED8AA42DCD348
:1023C00000212046FFF718FEB4F8565BB4F85C3BDA
:1023D000AB42D6D1B4F96E3BB4F96C7BB4F9662B41
:1023E000B4F9701BB4F9646BB4F9680B1F4416445C
:1023F000B4F9723BB4F96A2B0F4405F2123189B279
:102400000644B1F5B46F16441F4428BFA5F28E21CF
:1024100094F8753B8DF814304FF0080246F38F06A0
:1024200047F38F0728BF89B205AB00920297019648
:1024300084222046FFF764FD94F8753B402B55D06D
:10244000202B00F0E88094F8782BB2B394F8763B18
:102450000133DBB20C2B84F8763B1DD8012A35D131
:1024600094F8793B042B3AD80133DBB284F8793BFA
:102470008DF8143005AA2223012178480BF03AFE8A
:1024800094F8780B003018BF012017E00121FFF706
:10249000B3FDB4F8565B70E7012170480BF05EFEA7
:1024A000002342F20F72A4F8583B84F8763B84F87C
:1024B000783BA4F85A3BA4F85C2B00200023B4F826
:1024C000565BC4F8603B84F8753B5FE7022A04D191
:1024D00094F87A3B002B40F0B3800120EEE72022F5
:1024E00000238DF8142084F8793BC3E704A801F099
:1024F0002BF90DF113030DF1120204A80DF11501D2
:1025000001F03EF994F8772B9DF812309A42B7D13A
:102510009DF814209DF8133000211A438DF81420E3
:1025200084F8761B84F8791B0A2B6ED8DFE803F059
:102530006353346D6D6D2006066D060094F8780BBC
:1025400002289FD1B4F9582B454944480097334697
:102550000CF0F8FA204605A9FFF7AAFE94F8780BCC
:102560009DF8133084F87A3B003018BF0120A5E7AE
:10257000B4F9582B3B493948009733460CF0E2FA3E
:10258000204605A9FFF794FE0222002384F8782B49
:1025900084F87A3B012091E794F8780B01287FF4C6
:1025A00071AF3149B4F9582B009733462B480CF0E2
:1025B000C9FA204605A9FFF77BFE002042F20F73FF
:1025C000A4F8580B84F8760B84F8780BA4F85A0B0F
:1025D000A4F85C3B72E72549B4F9582B00973346C1
:1025E0001E480CF0AFFA05A92046FFF761FE012056
:1025F00084F8780B62E794F8783B012BF7D1B4F9B3
:10260000582B1B4900973346EAE7B4F9582B194970
:1026100000973346CAE7B4F9582B17490F4800977B
:1026200033460CF08FFA204605A9FFF741FE002340
:10263000012084F8780B84F8763B84F8793B3DE7F9
:1026400043F04003204605A98DF81430FFF730FE13
:1026500094F8780B003018BF01202FE7F04CFF1FD3
:10266000A84E0100744E0100484F0100DC4E0100ED
:10267000104F0100804F0100AC4F0100B3B1F8B51D
:102680005E1EF6B2074601EB46068C1E951E34F917
:10269000021F35F8022F3846FFF73AFEB442F6D152
:1026A0000146BDE8F840034806F098B819460148CD
:1026B00006F094B858A5FF1F70B5044600264FF4E5
:1026C000B970268166736681208026730FF0A8FC9E
:1026D00004F11C056060266131466661A6612B46E7
:1026E00004F13C0223F8021B9342FBD104F2EC40BC
:1026F000002203F8012B98424FF00001F9D1F0239A
:10270000A4F8EC14A4F8EE14C4F8F03420222846FF
:1027100011F0FCFC05210922034B2174A5616282A2
:102720006361204670BD00BF280CFF1F222AF0B451
:1027300002D00420F0BC70474289038992B29BB258
:102740009A4217D04289038992B29BB29A420BD225
:1027500004890288438912FA83F31B1B9BB29A42B5
:102760000CD20520F0BC70474389048902881B1BEA
:102770009BB2F4E7037B002BF3D10388202BF0D925
:102780004B1C0125223103E04573013399421CD0D3
:10279000027B02F0FF06002AF6D1446802891F7806
:1027A00092B2A7540289013292B20281048902884E
:1027B000A4B292B2944228BF068104894289A4B28D
:1027C00092B2944208BF0573DFE70020B2E700BF72
:1027D000F0B58FB002AC04AA4FF4E37E40F252573A
:1027E0004FF6AE264FF63A6501F0C003802B1CD0A1
:1027F000C02B18D0ABB12680023489009442C9B2F4
:10280000F2D102A92246103004230FF017FE002354
:102810000093224614230221054805F0F7FE0FB06D
:10282000F0BD2580E8E72780E6E7A4F800E0E3E7CD
:1028300058A5FF1FB0F8EC2438B51AB30446494830
:1028400005F0A4FF1428054640F28B80B4F8EE345E
:1028500001E0142D3DD95A1C2344A4F8EE2493F82A
:102860003C102046FFF7B4FFB4F8EE34B4F8EC2483
:10287000143D9A42ADB2ECD80023A4F8EE34A4F88B
:10288000EC3438BD4189038989B29BB2994229D081
:102890004189038989B29BB299421BD2038941893C
:1028A0005B1A9BB2ABB1304B1B7803BBD0F8F01472
:1028B00041B15F24C21801339BB28B4282F83C4085
:1028C000F8D38AB20023A0F8EC24A0F8EE34002A52
:1028D000B4D138BD44890388018913FA81F31B1BE5
:1028E0009BB2DFE7037B002BF3D00388DAE700F12C
:1028F0003C0100F15D05002413E0426843899BB26E
:10290000D35C0B700473438901339BB243814289CA
:10291000038892B29BB29A4200D344810131A9420A
:102920000BD00289438992B29BB29A42E5D1037BD4
:10293000002BE2D10131A942F3D10C4C00F15C0231
:102940006321002301E014F8011F02F8011F013385
:10295000272BF8D148220023A0F8EC24A0F8EE346D
:102960006CE738BD58A5FF1F50A5FF1FFC4F0100A5
:102970004289038992B29BB29A4220D0428903894C
:1029800092B29BB29A4208D34389018902885B1AAA
:102990009BB293420AD9002070470189028843897B
:1029A00012FA83F35B1A9BB29342F4D80A48A0FB55
:1029B00003201B1A00EB5303C3F347107047037B3C
:1029C000002BE8D10088044BA3FB0023C01A03EBC3
:1029D0005000C0F347107047D5411DD40C234FF46D
:1029E000167203FB0121B1F5966F8ABF4FF496630F
:1029F000C0F8F014C0F8F034704700BF034600F18F
:102A00001401002243F8042B8B42FBD130B400F2B6
:102A10003C55002423F8024B9D424FF00002F9D1AF
:102A200042F20F73A0F83C25A0F83E25C0F84425DB
:102A3000A0F84825A0F84A2580F84C25A0F8403594
:102A400030BC7047002342F20F72A0F84025A0F876
:102A50003E35A0F83C35C0F84435A0F84A35A0F81A
:102A6000483570472DE9F047BDF82050BDF924C026
:102A7000BDF92880002A6CD0013A05F1040ED2B2CB
:102A8000AE1C0EEB42020135334F1FFA8CFC1FFACD
:102A900082FEB6B2ADB2C8F1000924E04FEAE20A04
:102AA00002F0070213F80A40BA5C24EA020203F8B3
:102AB0000A20EA1005F0070A9C5C17F80AA04AEA07
:102AC00004049C544A1D92B2B2F5257F06F1020619
:102AD00028BFA1F28F21B6B22CBF89B211460235B0
:102AE000B645ADB235D000EB4104B21EA48ACCEBA2
:102AF000040424B24C4592B2D0DB002C1FDB4445C9
:102B000013DA4FEAE20A02F0070213F80A40BA5C4D
:102B1000224303F80A20EA1005F0070A9C5C17F824
:102B20000AA024EA0A049C54CCE7D41002F007025D
:102B300013F804A0BA5C42EA0A021A55B9E74FEA50
:102B4000E20A02F0070213F80A40BA5C24EA020221
:102B5000DFE7BDE8F08700BF605001002DE9F04FCE
:102B6000B0F83C2550F8223000294FEA4303B8BFA3
:102B700043F0010340F82230B0F83E25044604EB50
:102B800042028348918223F07F4391B058400CF079
:102B9000D1F80228B4F83EC57ED80CF2212189B2C2
:102BA000B1F5257F7B487C4F26BFACF173031FFA3C
:102BB00083F8884600F1170E6FF002034FF47A563F
:102BC000002504EB4802B2F914209742B8BF17461B
:102BD0009642A8BF1646012B19D0032B13D0013300
:102BE00001D002EB4202154408F105039BB2B3F594
:102BF000257F24BFA8F28F239BB2864509D0984633
:102C000010F9013FDDE702EB4202AD1AECE7AD1A25
:102C1000EAE7D4F844359D423EDD3E447610BF1BC2
:102C200044F6314909FB07F747F3CF33B1F5257F68
:102C3000059328BFACF17301059B02934FF004028A
:102C400036B20DF11C0A28BF89B2009220460196C7
:102C5000534618224FF00008FFF704FFDFF848B191
:102C60004E4FC1460D200F2103E01BF8011F17F83E
:102C7000010F1AF808200A4050400CF055F808F1EE
:102C800001084844B8F1070F5FFA80F9EDD1B9F1B6
:102C9000030F52D9B4F83EC5B4F840359C4518D05E
:102CA0000CF1010C1FFA8CFCBCF5257F24BF00231E
:102CB000A4F83E35B4F83C3538BFA4F83EC501331E
:102CC0009BB2042B88BF0023A4F83C3511B0BDE8AB
:102CD000F08F0CF1060189B2B1F5257F28BFACF267
:102CE0008E21B4F94A35B4F9480501904FF0080235
:102CF00028BF89B20293009207AB84222046FFF7D7
:102D0000B1FE06A800F020FD0DF11B030DF11A0223
:102D100006A80DF11D0100F033FD94F84C259DF837
:102D20001A309A4225D042F20F720023B4F83EC501
:102D3000A4F84025C4F84435B2E7059F184919485E
:102D40003B4632460BF0AAFEB4F83EC5C4F84455E3
:102D50000CF20D139BB2B3F5257FA4F84865A4F8D7
:102D60004A7503D36FF4C37363449BB2A4F8403530
:102D700094E79DF81B30032BD5D1C32507AA222346
:102D8000002108488DF81C500BF0B4F9CBE700BFC8
:102D90006E2876006850010080C1FFFF2C500100B2
:102DA00034500100F04CFF1F2450010072B170B587
:102DB000551EEDB2064601EB45058C1E34F9021F87
:102DC0003046FFF7CBFEAC42F8D170BD704700BF74
:102DD00080F84C15704700BF10B50021044600F084
:102DE00063F804F65460012100F05EF8204610BD3F
:102DF0002DE9F0479DF820407CB30746601E80B265
:102E000001EB40095E1E8C1E951E07F6546814E007
:102E1000082B384601D100F095F834F9021F35F837
:102E2000022F384600F0C0FA2A88B4F90010824612
:102E3000404600F0B9FA4C4505D016F8013F042B86
:102E4000E6D14046E7E7BAF1000F0CBF0146012189
:102E50000348BDE8F04705F0C1BC2146F8E700BFD4
:102E600058A5FF1F38B504460D4600F06BFA2946F9
:102E700004F65460BDE8384000F064BA38B5044642
:102E80000D4600F063FA294604F65460BDE8384068
:102E900000F05CBA10B5044600F060F804F6546027
:102EA000BDE8104000F05AB8034630B403F8041BE4
:102EB00000F11804002243F8042BA342FBD100F5D3
:102EC000E465002423F8024BAB424FF00002F9D135
:102ED00042F20F73A0F82837A0F82027A0F8222785
:102EE000A0F82427A0F82627A0F82A27C0F82C2726
:102EF000A0F83027A0F83227A0F83427A0F836270A
:102F0000A0F83827A0F83A27A0F83C27A0F83E27D9
:102F100080F8402780F8412780F8422780F843272F
:102F2000A0F8442780F8462780F8472780F84827EC
:102F300000F24A7300F6526123F8022B9942FBD14A
:102F400030BC70470023A0F82237A0F82A37A0F839
:102F50002037C0F82C3780F841377047002342F201
:102F60000F72A0F82827A0F82437A0F82237A0F87D
:102F70002A37A0F82037C0F82C3780F8413780F87E
:102F8000423780F84637A0F8263770472DE9F04FD2
:102F900087B08146BDF94840BDF84000BDF9447096
:102FA0000494002A00F08A80013A2646D2B2041D19
:102FB00004EB4202851C01301FFA82FB82B2704290
:102FC000019048461FFA87FAD946ADB2834618E009
:102FD0003C483C4E10F8084013F80E0016F80CC0A0
:102FE00020EA040003F80E00D85D4CEA000C03F858
:102FF00007C00235ADB205310232A94589B292B29D
:103000005CD001F10C00019E3BF81040CAEB0404B7
:1030100024B2A81E80B2B4424FEAE20702F0070CC5
:103020004FEAE00E00F00708D2DB002C34DB00F0A2
:1030300007064FEAE00802963046049E4FEAE20C8B
:1030400002F00707B442C6460397CDF814C010DA61
:1030500006461C48845D13F808001A4E204303F806
:103060000800F75D13F80C0020EA070703F80C705E
:10307000BFE7144C245C13F80800204303F8080051
:103080003E46D0100F4F185C17F806C04CEA000CF3
:10309000D01003F800C0ACE7C7100A4EDC5D00F0AA
:1030A0000700305C24EA0000D855D01002F0070772
:1030B0001C5CF75D24EA07041C549AE707B0BDE8DE
:1030C000F08F00BF385201002DE9F04F05469648B9
:1030D000B5F8203705EB830389B05B6823F07F43A5
:1030E00058400F460BF026FEC31EDBB2122B3AD916
:1030F000B5F822878D49DFF844C2A8F17309064666
:103100001FFA89F908F1050889481FFA88F84B4623
:103110004FF47A5E002403F10C0235F91220944535
:10312000B8BF94469645A8BF9646022E94BF91F923
:1031300000A090F900A0BAF1010F17D0BAF1030F67
:1031400016D0BAF1FF3F01D002EB4202144405331E
:103150009BB2434501F1010100F10100DBD1D5F83B
:103160002C379C4208DC09B0BDE8F08FA41AEEE7CA
:1031700002EB4202A41AEAE70EEB0C035B10C3EB6E
:103180000C0C44F6314B0BFB0CFC4CF3CF321BB256
:10319000104605920DF1180A04220493019302903F
:1031A00000924946534618222846FFF7EFFE022EAA
:1031B0004FF0000B45D8DFF888915E4ED8460D20C1
:1031C0004FF00F0E03E019F801EF16F8010F1AF88F
:1031D0000B100EEA010148400BF0A6FD0BF1010BAC
:1031E0004044BBF1070F5FFA80F8ECD1B8F1030F50
:1031F000B9D8002F6BD195F84037BDF8141005EB06
:1032000043020133DBB2A2F83817032BBDF81010CC
:10321000A2F8301794BF85F8403785F84077B5F8A5
:103220002237C5F82C47A3F5C37003F20D114022D5
:10323000A5F82437A5F82607A5F8281785F841270B
:1032400091E7D846DFF8F8903B4E07204FF00F0E7D
:1032500003E019F801EF16F8010F1AF80B100EEA47
:10326000010148400BF060FD0BF1010B4044BBF144
:10327000070F5FFA80F8ECD1B8F1030F3FF673AF98
:10328000DFBB95F84037BDF8141005EB430201335E
:10329000DBB2A2F83817032BBDF81010A2F83017D4
:1032A00094BF85F8403785F84077B5F82237C5F8E0
:1032B0002C47A3F5C37003F20D112022A5F8243783
:1032C000A5F82607A5F8281785F841274BE7059AA2
:1032D000A5F83E270023A5F83C27A5F83A27A5F82E
:1032E0003827049AA5F83627A5F83427A5F83227F9
:1032F000A5F8302785F8403791E7059AA5F83E27CD
:103300000023A5F83C27A5F83A27A5F83827049A02
:10331000A5F83627A5F83427A5F83227A5F83027D1
:1033200085F84037C1E700BF6E28760040520100A3
:1033300098500100905001008850010080C1FFFFAB
:103340008050010080F84317704700BFA0F8441771
:10335000704700BF0A46B0F8261701F13C0301F59B
:10336000167130B49BB28CB20546002105EB4300C8
:103370000133B0F84A079BB2A3420144F6D1084B8F
:103380000848A3FB01135B0AC3F3072182F823302B
:1033900082F822102978242330BC0AF0ABBE00BF8B
:1033A00049D6B9F2F04CFF1FF0B5B0F82A37B0F8A3
:1033B000444701339BB29C428FB0A0F82A3738D8DB
:1033C000B0F82237B0F82857AB4232D8B3F5617F56
:1033D0002FD200EB430400292183A4F84A27B0F838
:1033E000202700EB820254684FEA4404B8BF44F03F
:1033F0000104546090F8462704460ABBA3F5C8723E
:103400005A2A2FD9AB4235D094F84607003018BF5E
:103410000120B4F82027013292B20133042AA4F823
:1034200022378ABF0023A4F82027A4F820370FB042
:10343000F0BD90F84607003018BF01200FB0F0BD76
:10344000B0F82427511E89B28B42DBD3013292B2ED
:103450009342D7D80021FFF737FEB4F82237B4F8EB
:103460002857CFE70121FFF72FFEB4F82237B4F831
:103470002857C7E7B4F930E7B4F93257B4F93A2717
:10348000B4F93477B4F93867B4F93C07B4F93617AE
:10349000754416443D44B4F93E2794F841E70EAF15
:1034A000064407F824ED0D441644A3F28E210822A9
:1034B00045F38F0546F38F063B46009289B201958E
:1034C000029684222046FFF761FD94F84137402B95
:1034D0004DD0202B31D094F8462762B394F8423770
:1034E0000133DBB20C2B84F8423719D8012A5DD1A5
:1034F00094F84737042B52D9202200238DF814204A
:1035000084F847377C4821783A4622230AF0F2FDB6
:1035100094F84607003018BF0120B4F8223778E746
:10352000217875480AF01AFE002242F20F7384F8DF
:103530004627A4F828370020EFE72278B4F924378B
:103540006E496D480196002A0CBF012202220095A7
:103550000BF064FB20463946FFF7FCFE00230120F8
:1035600084F8460784F8423784F84737D5E704A83B
:1035700000F0EAF80DF113030DF1120204A80DF1A9
:10358000150100F0FDF894F843279DF812309A4297
:1035900015D094F84607003018BF0120BDE701336D
:1035A000DBB284F847378DF81430ABE7022A04D138
:1035B00094F84837002B40F096800120ADE79DF845
:1035C00014209DF8133000211A438DF8142084F83C
:1035D000421784F847170A2B7AD8DFE803F06A55B8
:1035E0003879797920060679060094F8460702288A
:1035F000D1D12278B4F9243741493F480196002AB5
:103600000CBF0122022200950BF008FB3946204630
:10361000FFF7A0FE9DF8133084F84837B9E7227809
:10362000B4F92437374934480196002A0CBF0122E7
:10363000022200950BF0F2FA20463946FFF78AFE87
:103640000220002384F8460784F84837A3E794F85B
:10365000460701289FD122782B49B4F924370196D7
:10366000002A00950CBF0122022223480BF0D6FA53
:1036700020463946FFF76EFE002042F20F7384F8B1
:103680004607A4F8283786E722782049B4F924377A
:103690000196002A00950CBF0122022216480BF069
:1036A000BDFA39462046FFF755FE012084F846074B
:1036B00071E794F84637012BF7D12278B4F9243713
:1036C00013490196002A00950CBF01220222E5E76A
:1036D0002278B4F924370F490196002A00950CBFCF
:1036E00001220222C1E743F04003394620468DF80B
:1036F0001430FFF72FFE4CE7F04CFF1F0052010083
:10370000E8500100B0500100945101002051010027
:1037100058510100D051010020F4FF6323F007034A
:103720008BB14FF4802340F67541034208BF5B081C
:10373000FBD0DA0A01FB02F2504020F4FF6222F0D3
:103740000702002AF1D17047704700BF4B78887894
:1037500010B50C78DB0003EBC42303EB5014B4F575
:10376000006F204606DA054B53F820006040C0F396
:10377000C72010BDFFF7D0FFF5E700BF5854010088
:10378000F0B517464E7BCA7C0C7D91F80CE0B50075
:10379000910025F03F0501F03C0183B02943A200D0
:1037A000B60946EA8E0641EA941422F00F0201A9F6
:1037B0001D468DF804608DF805408DF80620FFF752
:1037C000C5FF030900F00F003B70287003B0F0BD87
:1037D00002F00F0242EA0111C9B2144AF0B532F800
:1037E00011701D7D5E7B1C7B93F813E0F8B205F031
:1037F000030545EA801506F00F068008BF0A46EA71
:10380000811600F0300224F03F0407F03C072EF050
:103810000F0E00F00F0044EA910116434EEA00003B
:103820003D4319735E73D8741D75F0BD5852010085
:10383000F8B500264FF4B975044606810580468127
:103840004673067328460EF0EBFB268360606683A2
:1038500025822846267766770EF0E2FB04F12C05D8
:103860006061266230466662A6622B4604F14C0116
:1038700023F8020B8B424FF00002F9D184F84C2060
:1038800004F14D0304F16E00002103F8011B98427E
:103890004FF00002F9D104F16F0684F86E20334630
:1038A00004F17B0703F8012BBB42FBD13B4604F13B
:1038B0008701002203F8012B8B42FBD104F1AF01F9
:1038C000002203F8012B8B42FBD104F1D700002228
:1038D00003F8012B98424FF00001F9D1A4F8D81059
:1038E000A4F8DA10C4F8DC10C4F8E010C4F8E4104E
:1038F00084F8E81084F8E9102022284610F006FC2D
:10390000094B63620521092284F820106284A562B4
:1039100038460C2205490CF05BF830460C2203496E
:103920000CF056F82046F8BD840CFF1F9C74010073
:10393000222AF0B402D00420F0BC7047034640892C
:103940001A8980B292B2904217D058891A8980B2EF
:1039500092B290420BD21C8918885A8910FA82F2CE
:10396000121B92B290420CD20520F0BC70475A89CB
:103970001C891888121B92B2F4E71A7B002AF3D133
:103980001A88202AF0D993F8E820002A2BD14A1C63
:103990000125223103E05D7301328A421CD0187B7D
:1039A00000F0FF060028F6D15C681889177880B20D
:1039B00027541889013080B218811C891888A4B254
:1039C00080B2844228BF1E811C895889A4B280B26B
:1039D000844208BF1D73DFE7084A107858B90122F6
:1039E00083F84C20A8E700221A815A735A8183F881
:1039F000E8201A73CBE700209EE700BF50A5FF1F09
:103A0000222AF0B402D00420F0BC70470346408B59
:103A10001A8B80B292B2904217D0588B1A8B80B218
:103A200092B290420BD21C8B188A5A8B10FA82F2F7
:103A3000121B92B290420CD20520F0BC70475A8BF8
:103A40001C8B188A121B92B2F4E71A7F002AF3D15A
:103A50001A8A202AF0D993F8E920002A2BD14A1C8F
:103A60000125223103E05D7701328A421CD0187FA4
:103A700000F0FF060028F6D15C69188B177880B239
:103A80002754188B013080B218831C8B188AA4B27B
:103A900080B2844228BF1E831C8B588BA4B280B294
:103AA000844208BF1D77DFE7084A107858B9012221
:103AB00083F84C20A8E700221A835A775A8383F8A8
:103AC000E9201A77CBE700209EE700BF50A5FF1F33
:103AD000092A01D004207047F8B50C220E4605468D
:103AE00000217B3010F012FB154FDFF858E0002268
:103AF000402401204FF0800C12E091F87B301C43F1
:103B0000531C1A46442ADBB281F87B4003F00703BA
:103B100014D01EF8010F17F803C000F00703FC5C77
:103B2000D31005EBD001F35C1CEA030FE5D105EBE4
:103B3000D00191F87B3023EA0404E1E70020F8BDCE
:103B4000CC74010058740100012A01D00420704790
:103B50000978012908D00229F8D1002380F8E9204A
:103B6000C0F8E43018467047002380F8E810C0F829
:103B7000E0301846704700BF002380F84C10C0F8B2
:103B8000DC30C0F8E030C0F8E43080F8E83080F88D
:103B9000E9307047002914BF0523002380F84C301A
:103BA000704700BFF0B595B0164603AC05AA4FF4B8
:103BB000E37C40F2525E4FF6AE274FF63A6501F0D5
:103BC000C003802B24D0C02B1FD0E3B12780023448
:103BD00089009442C9B2F2D1002503A90AAA203073
:103BE000042305956560A560E56025618DF81E607C
:103BF0000EF024FC0AAA009414230221064804F0C3
:103C000005FD15B0F0BD2580E1E7A4F800E0DEE792
:103C1000A4F800C0DBE700BF58A5FF1F4289038955
:103C200092B29BB29A4220D04289038992B29BB24F
:103C30009A4208D34389018902885B1A9BB2934256
:103C40000AD90020704701890288438912FA83F358
:103C50005B1A9BB29342F4D80A48A0FB03201B1ABC
:103C600000EB5303C3F347107047037B002BE8D1ED
:103C70000088044BA3FB0023C01A03EB5000C0F3E1
:103C800047107047D5411DD4428B038B92B29BB233
:103C90009A4220D0428B038B92B29BB29A4208D3B5
:103CA000438B018B028A5B1A9BB293420AD9002094
:103CB0007047018B028A438B12FA83F35B1A9BB223
:103CC0009342F4D80A48A0FB03201B1A00EB5303CD
:103CD000C3F347107047037F002BE8D1008A044BE1
:103CE000A3FB0023C01A03EB5000C0F3471070473A
:103CF000D5411DD40B01C218F0B455891489ADB259
:103D0000A4B2A54267D055891489ADB2A4B2A54228
:103D100046D35589C65A148916FA84F2521B92B2B8
:103D2000202A43D9D0F8DC20132A3FD901F13802E8
:103D300050F82220052A39D9034400EB011600F17E
:103D4000860400F1A707002515E071685A8992B230
:103D50008A5C84F829201D735A89013292B25A81F3
:103D60005989328889B292B2914200D35D8104F8B8
:103D7000015FA7420CD019895A8989B292B2914247
:103D8000E3D11A7B002AE0D104F8015FA742F2D107
:103D900021220023A0F8D820A0F8DA30F0BC704728
:103DA00014895289A21A92B2202ABBD80144002554
:103DB00081F8E85000F14C0300F1AE0100F18602F9
:103DC00000F16D0613F8014F01F8014FB34202F8FC
:103DD000015FF7D1DCE7127B002AE7D0C25A9FE7E8
:103DE000214B1B78622B30B427D05F2B20D100F100
:103DF000AE0300F1860200F1B5055524002103F859
:103E0000014FAB4202F8011FF9D103465F2203F8CC
:103E1000B62F00F1BD0500F18E02FF24002103F84A
:103E2000014FAB4202F8011FF9D10F23A0F8D8309F
:103E30000023A0F8DA3030BC704700F1AE0300F187
:103E4000860200F1CF055F24002103F8014F9D4257
:103E500002F8011FF9D12123A0F8D8300023A0F8DF
:103E6000DA3030BC704700BFAC78FF1F2DE9F84353
:103E700004460F46D0F8E000D4F8E410D4F8DC3063
:103E800094F86E600130013103F101090B2E904668
:103E9000C4F8E000C4F8E410C4F8DC9024D900238E
:103EA00084F86E306289238992B29BB29A4200F004
:103EB000E5806289238992B29BB29A4280F0B380F6
:103EC000238962899B1A9BB2002B00F0B68004F113
:103ED0006F0318460C2204F17B010BF079FD0021E1
:103EE00003460E46032506E0002EDBD0F51CEDB29E
:103EF00004F16F0331460322194404F1AF000BF0C3
:103F000067FDB8F1010F14BF042208220023B9F1A4
:103F1000130F84F8892084F8873084F8883025D9F5
:103F20004FEA081804EB08014A890B8992B29BB248
:103F30009A4200F0A8804A890B8992B29BB29A42B9
:103F4000C0F09480488934F808300A8913FA82F363
:103F50009AB283B2D31A18BF0123A7F10102B2FAB1
:103F600082F252094EB9B64601270CE0A7F10102D0
:103F7000B2FA82F25209002E4AD0B6F1090718BFF0
:103F800001274FF0010E002B8EEA020194F8AFC01A
:103F900082EA03000CBF00268026C9B246EA0C0C58
:103FA000002A3ED10023BEF1000F94F8B02043EA6E
:103FB0000C0C0CBF00238023002F84F8AFC043EA11
:103FC00002030CBF0026082694F8B12084F86E5036
:103FD0008F4214BF202100211143704514BF4FF0C0
:103FE000020E4FF0000E3343874214BF0227002712
:103FF00047EA01004EEA03030321002284F8B030AF
:1040000084F8B100A4F8D810A4F8DA20BDE8F88349
:10401000012F94F8AFC040D01146B6461046012794
:10402000C0E70823BFE761892388228913FA82F356
:104030005B1A9BB2002B7FF44AAF628B238B92B248
:104040009BB29A423CD0628B238B92B29BB29A4233
:104050002ED2238B628B9B1A9BB2002B7FF437AF3F
:1040600004F16F0318460C221F4936E70B89488973
:104070009AB283B2D31A18BF01236EE7237B002BB9
:10408000DBD0238820E70A7B02F0FF03EAB134F893
:104090000830003318BF01235FE74CF0080CB64628
:1040A000114684F8AFC0104694F8B03008268BE76C
:1040B000618B238A228B13FA82F35B1A9BB2CCE7C3
:1040C000237F002BCCD0238AC7E7A7F10102B2FAE5
:1040D00082F25209002E7FF450AF94F8AFC011461F
:1040E0001046B646012759E79C74010038B590F890
:1040F0004C3033B3B0F8D82004461AB3284804F043
:1041000045FB142805464AD9B4F8DA3001E0142DED
:1041100017D9E218013392F8AF1092F88720A4F86B
:10412000DA302046FFF73EFDB4F8DA30B4F8D82094
:10413000143D9A42ADB2EAD80023A4F8DA30A4F8CC
:10414000D83038BD013B042B21D8DFE803F019201B
:10415000120A0300FFF744FEB4F8D830002BCDD18B
:1041600038BD00220121FFF781FE032384F84C3083
:10417000F2E70121FFF7BEFD022380F84C30EBE7A8
:104180000021FFF7B7FD042380F84C30E4E701225B
:104190000021FFF76BFE012384F84C30DCE738BDCB
:1041A00058A5FF1F30B500F14D0483B00D46212204
:1041B000074920460BF00CFC01A8FFF7C5FA23467F
:1041C000294601A80922FFF703FB03B030BD00BF59
:1041D000A874010000230383437743830377704768
:1041E000D0F8DC00704700BF03460022F0B503F8AA
:1041F000082B002400F130020025E3E80245934239
:10420000FBD100F5D0520C32002123F8021B93425F
:10421000FBD100F5EE510C31002523F8025B8B42F7
:104220004FF00002F9D141F6CC5741F6CE5641F697
:10423000D05341F6D25541F6D451C2538253C252A3
:1042400042F20F73435341F6D657435241F6D856C4
:1042500041F6DC5500F5EF51C35341F6E45C83535E
:1042600041F6E65E425141F6F8530A6041F6E857DE
:1042700041F6F45141F6EC5641F6F05520F80C2089
:1042800000F80E20C251825142514250C25000F5F6
:10429000F55100F5EF531C33043143F8042B8B42E6
:1042A000FBD100F5FA520C32002143F8041B934273
:1042B000FBD100F5FF521432002143F8041B934256
:1042C000FBD100F502521C32002143F8041B93423B
:1042D000FBD100F503520632002403F8014B934250
:1042E0004FF00001F9D142F2C80242F2CC038150F2
:1042F000C152F0BDF0B441F6D05141F6CE54002386
:1043000041F6CC5741F6DC5600F5EF52035341F627
:10431000D255037041F6D454435241F6D651C3539B
:104320008351136042F20F72425341F6D857025341
:1043300041F6E456425241F6E65542F2C80442F2D2
:10434000CC01C2538353435503514352F0BC7047D1
:1043500038B542F2CC030446C35A5BB929220D4852
:1043600009F020FE42F2C80142F2CC020023635061
:10437000A35238BD42F2C8002B222058B0FBF3F301
:10438000C3F3072081F8290081F82A30014809F099
:1043900009FEE7E7F04CFF1F38B542F2CC030446B4
:1043A000C35A5BB90C220C4809F02EFE42F2C80138
:1043B00042F2CC0200236350A35238BD42F2C8003F
:1043C0000E222058B0FBF3F3C3F3072008734B739E
:1043D000014809F019FEE9E7F04CFF1FFFFFFFFF5E
:1043E00070B541F6CC53044626A1D1E90001E35A49
:1043F00004EBC303D3E90223002322F07F425040A1
:1044000059400AF0B1FC02282ED841F6D0531C497D
:10441000E25A02F26D139BB2B3F5F07F24BFA2F112
:1044200073039BB2002001F118060CE0801A5A1D9C
:1044300092B26FF4ED75B2F5F07F2B442CBF9BB2B6
:104440001346B1420BD003F6045204EB420211F8BA
:10445000015FB2F90420002DE8D11044E7E741F6EE
:10446000DC53E258824201DB002070BD41F6CE529F
:104470000021E050A152012070BD00BFAFF30080C9
:10448000437B01005076550000000000FFFFFFFF56
:10449000F8B5044641F6CC5346A1D1E90001E35AF0
:1044A000257804EBC303D3E90223002322F07F42E3
:1044B000022D80EA020081EA030114BF00250225D3
:1044C0000AF052FC85422ED341F6D0533849E65AC1
:1044D00006F26D139BB2B3F5F07F24BFA6F1730310
:1044E0009BB2002001F118070CE0801A5A1D92B20D
:1044F0006FF4ED75B2F5F07F2B442CBF9BB21346E1
:10450000B9420BD003F6045204EB420211F8015FEA
:10451000B2F90420002DE8D11044E7E704F5EF528A
:104520001368834201DB0020F8BD731D41F6E4559A
:1045300041F6D4519BB20027B3F5F07F106067536A
:10454000665216D241F6D252A352731C9BB2B3F5F7
:10455000F07F19D241F6D852A35206F2DF139BB274
:10456000B3F5F07F1CD341F6D653013EE65201204D
:10457000F8BD41F6D2536FF4ED717218E252731C1C
:104580009BB2B3F5F07FE5D341F6D8536FF4EF72E9
:10459000B218E25206F2DF139BB2B3F5F07FE2D21B
:1045A00041F6D6520120A352F8BD00BFAFF3008000
:1045B000577A010068B4AA0000000000F8B50D4663
:1045C0000446FFF70DFFB0B141F6CE5041F6E6527A
:1045D000235A052603F11801A65442F2C80742F2F5
:1045E000CC0624F811500022013301212352E2515C
:1045F000A2532170F8BD2046FFF74AFF68B1074972
:1046000007480AF03FFA0121064804F0E7F80121C3
:10461000044804F0EFF802232370F8BD907A0100FB
:10462000F04CFF1F58A5FF1F2DE9F043079EBDF872
:1046300020704BB30020DFF854E0DFF854C004468C
:1046400011E0745D1EF8098008EA0404745505320F
:1046500092B2BA4200F1010028BFD21B84B228BF37
:1046600092B2A34210D931F91280B8F1000F4FEA8B
:10467000E00504F00709E4DA2C461CF80980755DB2
:1046800048EA05053555E2E7BDE8F083807A010088
:10469000887A0100FFFFFFFF2DE9F04141F6CC537E
:1046A000044661A1D1E90001E35A04EBC30386B0DB
:1046B0009B6858400AF058FB012879D941F6D65337
:1046C00041F6D852E35AA25A41F6D0519342615A68
:1046D00014D38B4216D98A4214D241F6E45834F8E6
:1046E0000830952B17D841F6D05341F6D855E25AE9
:1046F000635B9A4229D006B0BDE8F0818B42ECD8CA
:104700008A42EAD341F6E4582046FFF7C1FE34F866
:104710000830952BE7D93E493E480AF0B3F900210D
:104720003D4804F05BF83C48002104F063F8394848
:1047300009F09CFC41F6DC5104F5EF520023635074
:104740001360237006B0BDE8F08141F6D2574FF4F4
:10475000F07302AE04F5D051E25B01930C3160239B
:1047600020460096FFF760FF34F808202B48A2FB94
:104770000001531A01EB53031B0903EB4303C3EB83
:10478000C303D31A9BB21BBB42B331462046FFF78B
:1047900003FE41F6E45141F6DC55635A04F5EF504F
:1047A0000022013363526251026006B0BDE8F0811D
:1047B0001B4918480AF066F90021174804F00EF862
:1047C0000021154804F016F8124809F071FCB1E711
:1047D00031460C220F4809F017FCDAE741F6D651B2
:1047E000605F615EE25F41F6D4532D27E35E8DF892
:1047F00012708DE80300552016258DF81100094927
:1048000004488DF813500AF009FABEE7AFF30080B0
:10481000D47A0100F04CFF1F58A5FF1F876118864E
:10482000B47A0100FC7A01005E13AAAA000000001D
:104830002DE9F04341F6F45241F6EC5441F6E853C9
:1048400050F804C050F802E00D680F69C258654482
:104850007744BD4285B04FEAD20302F0070461DA23
:104860009B0000EB030941F6FC584A4E59F80870CA
:10487000365D0095374049F808704E684D696644CA
:104880007544AE4261DA00EB030C41F6A46E414D73
:104890005CF80E702D5D01963D404CF80E5041F6CF
:1048A000F05641F6F85550F806E08F6850F805C00C
:1048B0008E6977446644B7425FDA00EB030941F63C
:1048C0004C78344E59F80850365D0297354049F817
:1048D0000850CD68CE690EEB05010CEB0605A94228
:1048E00041DA034441F6F4752A4F5E593C5D039169
:1048F00006EA0401595141F6E85441F6EC570132F9
:104900000251009AC25141F6F05541F6F45141F678
:10491000F853019E029C039A46514450C25005B080
:10492000BDE8F0839B0000EB030941F6FC581A4EEA
:1049300059F80850365D0097354349F808504E68DD
:104940004D6966447544AE429DDB00EB030C41F6B5
:10495000A46E114E5CF80E70365D019547EA0605AF
:104960004CF80E509BE7034441F6F4760A499F59F0
:10497000095D039539439951BDE700EB030941F601
:104980004C78054D59F808702D5D02962F4349F873
:1049900008709EE7707A0100787A010070B50B46C6
:1049A00028CB88B085F0010483F00102A61869467F
:1049B0001C442A442B4401960496029407940392C3
:1049C000069200930593FFF733FF08B070BD00BF58
:1049D0002DE9F043654D664E2F464FF07F0C4FF0AA
:1049E000400E40F24911002315E092F81CE0013915
:1049F0000CEA0E0414774A1C03F1010300F0A080B6
:104A0000DFF868E15A4C01F0070C03F007021EF8CA
:104A10000CE014F802C0CA1002F27E7200EB8202AF
:104A200052681EEA020F00EBD30202F50252DCD0FC
:104A3000147F0CEA0404147701334A1E002900F0A5
:104A40008F80DFF828E14A4CD11001F2D27100EBDF
:104A5000810102F0070C496815F80CC01CEA010F2F
:104A600000EBD30101F5025103F0070891F81CC0D7
:104A700016F8088008EA0C0C81F81CC003F1010349
:104A800028D002F1FF3C002A6CD04FEAEC0101F281
:104A9000FC7100EB81010CF00708496815F80880EB
:104AA00000EBD30202F5025218EA010F02F11C02D8
:104AB00003F0070932D0117815F809800CF1FF3C9A
:104AC00048EA0101BCF1FF3F03F101031170DCD1A1
:104AD000BDE8F08302F1FF38002A45D04FEAE80232
:104AE00002F5F56200EB820208F007015268695C8A
:104AF000114200EBD30202F5025203F0070C117FC2
:104B000020D015F80CC04CEA01011177013308F1EF
:104B1000FF32B8F1000F97D1BDE8F08300EBD3026C
:104B200002F5025203F00708117F17F8088048EADF
:104B30000101117701330CF1FF38BCF1000FCDD129
:104B4000BDE8F08317F80CC04CEA0101117701337E
:104B500008F1FF31B8F1000F7FF455AFBDE8F083E5
:104B6000BDE8F083BDE8F083BDE8F083787A01000A
:104B7000707A010030B4134D481E01F126044FF045
:104B8000FF3210F8013F5340DBB2C2F3072235F881
:104B90001330844283EA02031A46F2D1DA4391F8D1
:104BA0002700D3B2984202D0002030BC704791F861
:104BB0002800C2F30723181AB0FA80F0400930BC6D
:104BC000704700BF5C7B01002DE9F0434E1E054697
:104BD000144699B0DFF838E230467027002201E031
:104BE0001EF8017F10F8013F01327B40532A06F87E
:104BF000013FF5D10DF10B030DF15F00002203F829
:104C0000012F8342FBD1DFF80CC2042763464FF02B
:104C1000000E80264FEAEE02885CC2070ED51CF813
:104C20001E2093F801800DF160094A4426FA08F924
:104C300012F8548C49EA080802F8548C82070DD502
:104C40009A7893F803800DF160094A4426FA08F92E
:104C500012F8548C49EA080802F8548C42070DD522
:104C60001A7993F805800DF160094A4426FA08F98B
:104C700012F8548C49EA080802F8548C020774D5DB
:104C80009A7993F807800DF160094A4426FA08F9E9
:104C900012F8548CB7F5257F49EA080802F8548CBD
:104CA00066D141F6EC5741F6F05641F6F45041F624
:104CB000F85141F6E8520023EB51AB512B506B50A9
:104CC000AB5099464FF080080127402618AA02EB06
:104CD000E90209F0070312F8542C28FA03F11140F5
:104CE00026FA03F30CBF0291029709F1020913405F
:104CF00001A9284614BF01970193FFF74FFEB9F5AC
:104D0000257FE3D12846FFF763FE631E04F12801E7
:104D1000002203F8012F9942FBD13C4F402040F282
:104D20004912012601E017F80C0005EBE20101F53C
:104D30000251C2F5A47391F81CE00133013AD9087D
:104D400010EA0E0F03F0070302F0070C06FA03F354
:104D500002D0605C03436354531CE4D121462846CF
:104D6000FFF708FF19B0BDE8F083B7F5257F98D0AD
:104D7000C2060DD51A7A93F809800DF160094A44EC
:104D800026FA08F912F8548C49EA080802F8548CFB
:104D900082060DD59A7A93F80B800DF160094A448A
:104DA00026FA08F912F8548C49EA080802F8548CDB
:104DB00042060CD402061AD40EF1080EBEF5267F68
:104DC00003F1100307F108077FF424AF69E71A7BAA
:104DD00093F80D800DF160094A4426FA08F912F89B
:104DE000548C49EA080802F8548C0206E4D59A7BF0
:104DF000D87B0DF16008424426FA00F812F8540CF2
:104E000048EA000002F8540CD6E700BF787A0100A7
:104E1000FC790100D4740100F0B541F6E655A3B069
:104E2000435D04460E469BB941F6CE5240F6E9403A
:104E3000A35A03F1180501339BB2834224F815608D
:104E4000A35230D040F6EE42934207D023B0F0BDDB
:104E5000FFF7C6FA635D013B6355E5E741F6E452AF
:104E6000002341F6D05041F6D251A35241F6D45717
:104E70004FF4EE7241F6D85641F6D655235262529F
:104E800040F2D7134FF4EC704FF4EB71E353A0539F
:104E90000090615319480191194909F0BFFE02239E
:104EA000237023B0F0BD40F6E4430DAD019305221D
:104EB00004F13001204600954FF42573FFF7B4FB51
:104EC000294602AA2046FFF77FFE50B941F6DC5280
:104ED00004F5EF532070A050186041F6CE53E35A0A
:104EE000B0E70121074803F079FC0121054803F0F0
:104EF00081FC02A92046FFF72BFAEEE7F04CFF1FDA
:104F0000207B010058A5FF1F002B6BD02DE9F04F2F
:104F1000013B00F5035B00F5EE5983B09BB2DA4626
:104F2000C84602EB4303971E064600938A1E0BF108
:104F3000080B0AF10C0A09F10C0908F110081AE033
:104F400030460192FFF7A8FB019AB8F80030013310
:104F50009BB2B3F5F07F28BF0023A8F80030B9F862
:104F6000003001339BB2042B88BF0023A9F8003026
:104F7000009BBB4233D037F8024FDBF80000BAF891
:104F80000010B9F8003020440131CBF8000006EBE6
:104F9000C303AAF80010D3E9024532F9021F24190D
:104FA0006D410029B8BF44F00104C3E90245B8F8D7
:104FB0000030307803F6045306EB43030128998050
:104FC00007D00228BCD030460192FFF7F7FA019AC9
:104FD000BBE730460192FFF71FFF019AB5E703B028
:104FE000BDE8F08F704700BF426803899BB2D1547F
:104FF000038901339BB203810289038892B29BB279
:105000009A4224BF002303810289438992B29BB252
:105010009A4204BF012303730120704770B5044610
:1050200000264FF4B970268166736681208026734E
:105030000CF0F6FF04F11C056060266131466661E4
:10504000A6612B4604F1440223F8021B9342FBD1D4
:1050500004F52770002203F8012B98424FF000015D
:10506000F9D13C23A4F89C12A4F89E12A4F8A03213
:10507000282228460FF04AF805210322034B217409
:10508000A56162826361204670BD00BFE00CFF1F16
:10509000292A01D004207047F8B54289038992B2C9
:1050A0009BB29A420C4607461BD04289038992B2B2
:1050B0009BB29A420FD201890288438912FA83F384
:1050C0005B1A9BB2934210D900221849184809F084
:1050D000DFFC0520F8BD4389018902885B1A9BB279
:1050E000F0E7037B002BEFD10388292B1BD93B7BF7
:1050F00003F0FF019BB101237B7304F12905012615
:1051000003E07E730134A54207D03B7B002BF8D12E
:1051100021783846FFF768FFF4E70020F8BD3846ED
:10512000FFF762FFE9E71AB2CFE700BFE0820100B4
:10513000F04CFF1F0C2A01D004207047F8B54289BB
:10514000038992B29BB29A420C46054615D0428919
:10515000038992B29BB29A422BD201890288438979
:1051600012FA83F35B1A9BB293420AD900221749C1
:10517000174809F08DFC0520F8BD037B002BF5D105
:1051800003880C2B20D92B7BCBB101236B7304F14B
:105190000C06012703E06F730134A64207D02B7B76
:1051A000002BF8D121782846FFF71EFFF4E70020F6
:1051B000F8BD4389018902885B1A9BB2D4E70121BB
:1051C0002846FFF711FFE2E71AB2D0E7008301009B
:1051D000F04CFF1F4289038992B29BB29A4210B5EC
:1051E00026D04289038992B29BB29A420DD3438959
:1051F000018902885B1A9BB293420FD900221149A0
:10520000114809F045FC052010BD01890288438939
:1052100012FA83F35B1A9BB29342EFD8002BEDD0C6
:10522000037B03F0FF0443B101234373002010BD4F
:10523000037B002BE2D10388F0E70221FFF7D4FEC5
:10524000204610BD20830100F04CFF1F2DE9F04FD8
:105250009BB0531E0392029318460DF166040DF1A4
:105260001303002203F8012F9C4200F8012FF9D10B
:1052700000234A1EDFF8C0A1009301921E461C467F
:105280004FF00109019A12F8018F0192009A3346FA
:105290000020264609FA00F118EA010F18BF012480
:1052A00002F1010108BF00241AAD05EBD20E05EB97
:1052B000D1071D193344234413F0010F02F0070CEA
:1052C00001F0070100F1010005F00105334602F18C
:1052D000020207D01AF80CB01EF854CC4BEA0C0CA2
:1052E0000EF854CC35B11AF8015017F8541C294364
:1052F00007F8541C082801D02646CBE7009B103342
:10530000B3F5287F0093BDD1494F039B042539464F
:10531000002601241AAA02EBD60212F8542C100619
:105320000BD517F8160091F801C013F800E004FA45
:105330000CFC4CEA0E0E03F800E050060AD591F87A
:1053400002C0C87813F80CE004FA00F040EA0E003E
:1053500003F80C0090060AD591F804C0487913F8B8
:105360000CE004FA00F040EA0E0003F80C00D0064E
:1053700020D591F806C0C87913F80CE004FA00F0C3
:1053800040EA0E00B5F5257F03F80C0015D1029D0B
:10539000284C00231946284601E014F8013F10F874
:1053A000012F01315340532905F8013FF5D11BB0BE
:1053B000BDE8F08FB5F5257FE9D010070BD591F842
:1053C00008C091F809E013F80C0004FA0EFE4EEA4A
:1053D000000003F80C0050070BD591F80AC091F8B3
:1053E0000BE013F80C0004FA0EFE4EEA000003F87E
:1053F0000C0090070BD591F80CC091F80DE013F854
:105400000C0004FA0EFE4EEA000003F80C00D2076E
:1054100009D591F80EE0C87B13F80E2004FA00F0CD
:10542000024303F80E2008361031083572E700BF3A
:105430005C7D0100848201004C83010070B59AB04C
:1054400002AC06AA012340F249354FF6B74633EACB
:10545000010E0CBF2680258002345B009442DBB233
:10546000F5D102A92246103008230CF0E7FF0023F3
:105470000093224628230121024803F0C7F81AB0FE
:1054800070BD00BF58A5FF1F01EB4101490001F5A8
:10549000967189B2B1F5167F8ABF4FF41673A0F8E2
:1054A000A012A0F8A03270474289038992B29BB241
:1054B0009A421DD04289038992B29BB29A4208D384
:1054C0004389018902885B1A9BB293420AD9002062
:1054D000704701890288438912FA83F35B1A9BB2F1
:1054E0009342F4D80748A0FB0330C0F3870070470D
:1054F000037B002BEBD103880248A0FB0330C0F3F1
:10550000870070474FECC44E034600895A8980B229
:1055100092B2904210B419D05C685A8992B20020BD
:10552000A25C0A7018735A89013292B25A81598961
:105530001A8889B292B2914204D358815DF8044B23
:105540000120704701205DF8044B70471A7B02F080
:10555000FF00002AE0D15DF8044B704770B5428926
:10556000038992B29BB29A42A2B004467ED042898D
:10557000038992B29BB29A4225D2038942899B1A2F
:105580009BB24BB362896168B4F89C3292B28A5C78
:10559000002A4DD14BBB634A1278002A40F090801C
:1055A000B4F8A0524DB1AA21E21801339BB2AB422C
:1055B00082F84410F8D1A4F89C520023A4F89E323B
:1055C0009DB922B070BD41890388028913FA82F324
:1055D0005B1A9BB2002BD5D1B4F89C32002BF0D0D3
:1055E0006289616892B28A5C12BB4F4803F0CEF8C0
:1055F00028280546E5D9B4F89E3201E0282DE0D9E7
:105600005A1C2344A4F89E2293F844102046FFF726
:1056100015FFB4F89E32B4F89C22283D9A42ADB2F0
:10562000ECD80023A4F89E32A4F89C3222B070BDBE
:10563000012A20D1002BD8D10CA92046FFF764FF06
:105640000C25B4F89C124B1C2144A4F89C32443124
:105650002046FFF759FF6B1E13F0FF05F1D1A4F8A8
:105660009E52B4F89C52002DABD0BEE7037B002BBA
:10567000B2D0038885E7022A4ED1002BB5D10CA900
:105680002046FFF741FFB4F89C3203F11205ADB29A
:10569000981D264E80B2552201E016F8012FE11820
:1056A00001339BB2834281F84420F6D1AB42EFD163
:1056B0000023A4F89C52A4F89E32002D81D094E7D8
:1056C0000DF103012046FFF71FFF01AD0DF12D067F
:1056D000294620460135FFF717FFAE42F8D101A950
:1056E0000DF132022046FFF7B1FDB4F89C32EA22F8
:1056F00003F15505A620ADB20CA98DF830208DF828
:10570000310001E011F8012FE01801339BB2AB42E8
:1057100080F84420F6D14EE71D46002D3FF451AFEE
:1057200063E700BF50A5FF1F58A5FF1F408301007E
:1057300038B50B4D04460021284603F04FF82846A3
:10574000002103F057F80748074909F09BF90523A2
:1057500084F84C3C04F67840BDE8384002F060BC68
:1057600058A5FF1FF04CFF1F5483010042680389B6
:105770009BB222F81310038901339BB20381028983
:10578000038892B29BB29A4224BF0023038102890C
:10579000438992B29BB29A4204BF01230373012052
:1057A000704700BF2DE9F843054602F0ADF905F555
:1057B000806002F0A9F905F5006002F0A5F905F591
:1057C000406001F0E9FF05F5426002F08FF805F650
:1057D0002840002702F02AFB05F5446002F0C8FBD0
:1057E00085F84C7C85F84D7C85F84E7C85F84F7C9F
:1057F00005F5456002F0FEFB05F6584002F0FAFBA5
:1058000005F5466002F0F6FB05F6684002F0F2FB93
:1058100005F5476002F0EEFB05F6784002F0EAFB82
:1058200005F6884905F5486002F0E4FB05F549688E
:10583000484602F0DFFB404602F0DCFB4FF4B56067
:10584000564B5749574AC5F8B00CC5F8B83C45F215
:10585000683044F66C23544CC5F8BC0CC5F8D81C11
:105860005248C5F8DC2C47F6E4214FF43572C5F8F0
:10587000E03C4FF40043C5F8AC2CC5F8B42C01262D
:10588000C5F8D03CC5F8F43CC5F8FC3C85F8987CDC
:10589000C5F8A47CC5F89C7CC5F8A87CC5F8A07C9C
:1058A000C5F8D47CC5F8C87CC5F8C07CC5F8CC7CEC
:1058B000C5F8C47CC5F8EC7CC5F8E47CC5F8F07C80
:1058C000C5F8E87CC5F8F84CC5F8000DC5F8041D0E
:1058D00005F6085001F012FF4FF4C87185F8197DE4
:1058E00085F81A7D85F81B7D85F8186DA5F81C6D67
:1058F000A5F81E6D05F5526002F05EF840F66113E2
:10590000A5F8403DA5F8487D85F83C7DA5F84A7D81
:1059100085F84D7D85F84C7DA5F83E6D41F2C2209D
:105920000CF07EFB4FF41664A5F8587DC5F8440DC5
:10593000A5F85A7D85F85D7D85F85C7DA5F8504D0C
:105940004FF496500CF06CFBC5F8540D05F55660FD
:1059500002F08AFB3A46484685F8807D85F8817DCD
:10596000314602F04BFB39464046962202F046FB98
:1059700005F5546703E0013C85F84D6D0AD095F8B4
:105980004C3D03F0FF01002BF5D13846FFF7EEFE4A
:10599000013CF4D12846BDE8F88300BFF96BFFFF56
:1059A0000080FFFF5D3BFFFF0000FFFFB505FFFF2D
:1059B00038B50025044680F84C5C00F5456002F0DF
:1059C00035FB04F6584002F031FB04F6684002F063
:1059D0002DFB04F5476002F029FB04F6784002F045
:1059E00025FB04F5486002F021FB04F6884002F034
:1059F0001DFB04F5496002F019FB04F5406001F05D
:105A00006FFF04F5806002F0F7F904F5006002F022
:105A1000F3F9204602F0F0F904F5446002F0E6FAEA
:105A2000A4F8585D04F55660A4F85A5D84F85D5DED
:105A300084F85C5D02F030FB04F5526002F060F81F
:105A400004F6284002F08EFA84F8985C84F8805DB1
:105A500084F8815D38BD00BF2DE9F04F83B000F5BB
:105A600046679DF834409DF840B09DF838609DF839
:105A700044C09DF848E09DF8305080F84DBCC4EB20
:105A80000414A400A4B2019680F84ECC064680F817
:105A90004FEC884638462146914600229DF83CA0AE
:105AA0009B4602F0ABFAC5EB0511890089B206F5F9
:105AB0004560002202F0A2FA14B1384602F0B0FAB2
:105AC000019B0C934A465B4641463046CDF834A0D4
:105AD00003B0BDE8F04F02F039B800BF2DE9F04740
:105AE000BDF824709DF820609DF828500446884633
:105AF000914600F678403A4600219A4602F07EFA36
:105B00002EB13A46314604F5476002F077FA09951E
:105B1000089553464A46414604F58060BDE8F04783
:105B200002F014B82DE9F04F85B083469DF84C7013
:105B30009DF858409DF864E09DF850609DF85450E1
:105B40009DF844008BF8187D8BF81B4D17469DF887
:105B500040409DF83820ABF81CED01908BF8196D92
:105B60008BF81A5D0BF658409DF848A000920394FC
:105B700000229DF860409DF83C509DF85C600294C6
:105B80009DF868909DF86C801C4602F037FA0199E8
:105B90000BF66840002202F031FA002251460BF564
:105BA000486002F02BFA39460BF5446002F0E8F940
:105BB0003A4649460BF6085001F0AAFD029AABF8A6
:105BC0003E8D31460BF6284002F03AF92B46009AFA
:105BD00021460BF5406001F0EDFD10B105B0BDE8C8
:105BE000F08F039A21460BF5426005B0BDE8F04FF7
:105BF00001F082BE70B4BDF80C509DF81040A0F8C2
:105C00001E2D012680F83C6D1A4604942B46039401
:105C100000F5006070BC01F099BF00BF70B504468C
:105C20000D4600F5456002F005FA294604F6584095
:105C300002F000FA294604F5466002F0FBF9294615
:105C400004F6684002F0F6F9294604F5476002F0D0
:105C5000F1F9294604F6784002F0ECF904F688469A
:105C6000294604F5486002F0E5F93046294602F07D
:105C7000E1F904F54960294602F0DCF9304602F00A
:105C8000E1F900B970BD304602F0E2F90028F9D020
:105C900094F84C1C034808F0B1FC3046BDE8704055
:105CA00002F0BEB9F04CFF1FF8B5054681BB02B942
:105CB000F8BD1F491F4808F0E5FE072385F84C3C56
:105CC00005F555674FF49664012603E0013C85F81D
:105CD0005D6D0AD095F85C3D03F0FF01002BF5D116
:105CE0003846FFF743FD013CF4D105F6584002F079
:105CF00097F905F5496002F099F905F6884002F038
:105D00008FF995F84C1C0B48BDE8F84008F076BCBC
:105D10000949084808F0B6FE022385F84C3C0121E9
:105D2000064802F05BFD0121044802F063FDDCE758
:105D300088830100F04CFF1F7083010058A5FF1FEE
:105D400038B5044631B100F65845284602F07AF9D4
:105D5000E0B938BD0D46174802F040FD2946154808
:105D600002F048FD1449154808F08CFE032384F81E
:105D70004C3C04F6784002F053F994F83C3D002B7B
:105D8000E7D00E48BDE8384008F05EBC284602F077
:105D90005FF900B938BD0A49084808F073FE0423CA
:105DA00084F84C3C284602F041F994F83C3D002B25
:105DB000E7D138BD58A5FF1FA0830100F04CFF1F9D
:105DC000BC83010070B5044639B900F67846304608
:105DD0000D4602F037F9A8B970BD0121134802F051
:105DE000FDFC0121114802F005FD1148114908F0A0
:105DF00049FE022384F84C3C04F67840BDE870402C
:105E000002F014B9304602F023F90028E4D00A4920
:105E1000074808F037FE304684F84C5C02F006F97B
:105E200004F65840BDE8704002F000B958A5FF1FC5
:105E3000F04CFF1F70830100D083010038B5044689
:105E400031B100F65845284602F0FCF868B938BD73
:105E50000E480F4908F016FE082384F84C3C04F65F
:105E60007840BDE8384002F0DBB8284602F0F0F890
:105E700000B938BD0548074908F004FE0923284643
:105E800084F84C3CBDE8384002F0D0B8F04CFF1F1D
:105E9000E48301000084010070B5044639B900F6BE
:105EA000784630460D4602F0CDF868B970BD11480D
:105EB000114908F0E7FD072384F84C3C04F67840CC
:105EC000BDE8704002F0B2B8304602F0C1F80028D8
:105ED000ECD00A49074808F0D5FD304684F84C5C00
:105EE00002F0A4F804F6584002F0A0F8012384F868
:105EF000983C70BDF04CFF1F88830100D0830100E7
:105F000070B5044639B900F6784630460D4602F0C1
:105F100099F868B970BD1148114908F0B3FD09231B
:105F200084F84C3C04F67840BDE8704002F07EB83E
:105F3000304602F08DF80028ECD00A49074808F0F6
:105F4000A1FD304684F84C5C02F070F804F658402D
:105F500002F06CF8012384F8983C70BDF04CFF1FF0
:105F600000840100D083010038B590F84C3C044611
:105F70000A2B0DD8DFE803F0530C5B6325250C2FAB
:105F80003841060011462046FFF7BAFF94F84C3C12
:105F900003B138BD04F54965284602F053F828B925
:105FA00094F8983C13B1284602F03AF8284602F0DB
:105FB00049F80028EDD0284602F04AF8002846D1DA
:105FC00038BD0029E5D12046FFF7B2FB94F84C3CE0
:105FD000002BDED1DEE711462046FFF72FFF94F8B5
:105FE0004C3C002BD5D1D5E711462046FFF754FF96
:105FF00094F84C3C002BCCD1CCE7002AC9D11749EE
:10600000174808F03FFD0A2384F84C3C04F678401A
:1060100002F006F894F84C3C002BBAD1BAE72046BF
:10602000FFF742FE94F84C3C002BB2D1B2E7204679
:10603000FFF786FE94F84C3C002BAAD1AAE7204635
:10604000FFF7C0FE94F84C3C002BA2D1A2E72846F3
:1060500001F0ECFF002384F8983C38BD188401005F
:10606000F04CFF1F2DE9F843054691468846A9B13B
:1060700090F8803D002B3ED090F8813DB9F1000FA3
:106080000FD1CBB195F8804D002C73D001220023A5
:1060900085F8982C85F8813DBDE8F88332B190F8F9
:1060A000813D5BB1B8F1000F40F08D8095F8803DE7
:1060B000A3BBB9F1000F49D0BDE8F88395F8803D46
:1060C000002B46D005F555674FF49664012603E092
:1060D000013C85F85D6D0AD095F85C3D03F0FF0149
:1060E000002BF5D13846FFF741FB013CF4D10123E9
:1060F00085F8813DD6E70121344802F06FFB01218C
:10610000324802F077FB95F8813D002B48D0012200
:1061100085F8802DB9F1000FB3D0C2E700212B48DC
:1061200002F05CFB0021294802F064FB95F8814DE8
:106130005CB395F83C3D002285F8802D002BB8D04B
:10614000234808F081FAB9F1000FB5D195F8813DE7
:1061500097E720491E4808F095FC072305F688407C
:1061600085F84C3C01F05CFF95F84C1C184808F091
:1061700045FAA7E71849164808F084FC85F84C4C06
:1061800005F6884001F052FF80E71349104808F0F7
:1061900079FC85F84C4C05F6884001F047FFC8E7CC
:1061A0000E490B4808F06EFC022385F84C3C05F6BE
:1061B000884001F035FF95F84C1C054808F01EFAA0
:1061C00095F8813DA3E7BDE8F88300BF58A5FF1F00
:1061D000F04CFF1F88830100D08301007083010011
:1061E00038B500F546650446284601F02BFF20B17E
:1061F000284601F02DFF48B938BD0A480A4908F081
:1062000041FC2046BDE8384001F0E4BD06490548A0
:1062100008F038FC204601F0DDFD2846BDE8384096
:1062200001F0FEBEF04CFF1F3484010038B5044677
:1062300031B100F66845284601F00AFF70BB38BD51
:106240000D46244802F0CAFA2946224802F0D2FA42
:106250002149224808F016FC04F6684084F84C5C9A
:1062600001F0E4FE04F6584001F0E0FE04F547605A
:1062700001F0DCFE04F5456001F0D8FE04F688402C
:1062800001F0D4FE94F83C3D012284F8982C002BB8
:10629000D5D01248BDE8384008F0D6B910490F48AB
:1062A00008F0F0FB022384F84C3C284601F0BEFEC7
:1062B00094F84D3C002BC2D094F84F3C002BBED03C
:1062C0002046FFF78DFF04F54560BDE8384001F03A
:1062D000A7BE00BF58A5FF1FD0830100F04CFF1FD1
:1062E0007083010038B5044661B100F65845284670
:1062F00001F0A8FEA0BB04F54565284601F0A2FE0A
:1063000008BB38BD0D46244802F068FA29462248E9
:1063100002F070FA2149224808F0B4FB032384F804
:106320004C3C04F6784001F07BFE94F83C3D002B99
:10633000E1D01B4804F5456508F086F9284601F0D0
:1063400081FE0028DDD0284601F082FE38B12046CB
:10635000FFF746FF2846BDE8384001F061BE38BD72
:10636000284601F075FE0028C5D00E490C4808F0FB
:1063700089FB042384F84C3C04F5476001F056FE89
:10638000284601F053FE04F5446001F029FE94F81C
:106390003C3D002BAFD0CCE758A5FF1FA0830100E8
:1063A000F04CFF1FBC83010070B50446C9B1012148
:1063B000304802F013FA01212E4802F01BFA2E4851
:1063C0002E4908F05FFB022384F84C3C04F6784029
:1063D00001F02CFE04F54565284601F033FE78BB3C
:1063E00070BD00F67845284601F02CFE0028F1D05B
:1063F000284601F02DFE0028ECD01F48204908F067
:1064000041FB04F547660B2384F84C3C304601F011
:1064100019FE10B3304601F01BFEF0B9284601F01A
:1064200005FE04F6584001F001FE04F5456504F54B
:10643000486001F0F5FD284601F004FE0028CFD0A9
:10644000284601F005FE38B12046FFF7C9FE284670
:10645000BDE8704001F0E4BD70BD0A49064808F08F
:1064600011FB04F5806001F0B5FC304601F0DEFD63
:10647000D4E700BF58A5FF1FF04CFF1F7083010039
:10648000508401004484010038B5044631B100F65F
:106490006845284601F0DCFDF8B938BD0D461C48BA
:1064A0001C4908F0EFFA04F6684084F84C5C01F0EF
:1064B000BDFD04F6584001F0B9FD04F5476001F058
:1064C000B5FD04F5456001F0B1FD04F6884001F02A
:1064D000ADFD012384F8983C38BD0F490C4808F005
:1064E000D1FA072384F84C3C284601F09FFD94F82C
:1064F0004D3C002BD1D094F84F3C002BCDD0204602
:10650000FFF76EFE04F54560BDE8384001F088BD38
:10651000F04CFF1FD08301008883010038B504468A
:1065200061B100F65845284601F08CFD28BB04F502
:106530004565284601F086FD90B938BD1B491C48C9
:1065400008F0A0FA082304F6784084F84C3C04F5DF
:10655000456501F065FD284601F074FD0028ECD08A
:10656000284601F075FD38B12046FFF739FE284670
:10657000BDE8384001F054BD38BD284601F068FD43
:106580000028D4D00B490A4808F07CFA092384F883
:106590004C3C04F5476001F049FD284601F046FDFA
:1065A00004F5446001F01CFDC1E700BFE483010075
:1065B000F04CFF1F0084010070B5044689B12D48DE
:1065C0002D4908F05FFA072384F84C3C04F6784024
:1065D00001F02CFD04F54565284601F033FD78BB3C
:1065E00070BD00F67845284601F02CFD0028F1D05A
:1065F000284601F02DFD0028ECD01E481F4908F068
:1066000041FA04F547660B2384F84C3C304601F010
:1066100019FD10B3304601F01BFDF0B9284601F01A
:1066200005FD04F6584001F001FD04F5456504F54B
:10663000486001F0F5FC284601F004FD0028CFD0A9
:10664000284601F005FD38B12046FFF7C9FD284670
:10665000BDE8704001F0E4BC70BD0949054808F090
:1066600011FA04F5006001F0B5FB304601F0DEFCE4
:10667000D4E700BFF04CFF1F888301005084010065
:106680006084010038B5044631B104F545652846FB
:1066900001F0D8FCE8B938BD0D46164802F09EF866
:1066A0002946144802F0A6F81349144808F0EAF9FC
:1066B00094F84E3C052284F84C2CBBB904F6784083
:1066C00004F5456501F0ACFC284601F0BBFC002850
:1066D000E1D0284601F0BCFC0028DCD02046FFF7C2
:1066E0007FFD2846BDE8384001F09ABC2046FFF700
:1066F00077FDE3E758A5FF1F54830100F04CFF1F0F
:1067000038B50446D1B101212D4802F067F80121C6
:106710002B4802F06FF82B482B4908F0B3F90423FB
:1067200084F84C3C04F6784001F080FC04F54565A3
:10673000284601F087FC002835D138BD00F67845A1
:10674000284601F07FFC0028F0D0284601F080FCAC
:106750000028EBD01D491B4808F094F90B2384F85E
:106760004C3C04F5446001F041FC1949154808F01F
:1067700089F904F5806001F02DFB284601F056FCF4
:1067800004F5476001F052FC04F6584001F04EFC5D
:1067900004F5456504F5486001F042FC284601F027
:1067A00051FC0028C9D0284601F052FC38B12046DF
:1067B000FFF716FD2846BDE8384001F031BC38BD72
:1067C00058A5FF1FF04CFF1FBC830100508401003F
:1067D0004484010038B5044631B104F545652846C6
:1067E00001F030FC90B938BD0F49104808F04AF963
:1067F0000A2304F6784084F84C3C04F5456501F022
:106800000FFC284601F01EFC0028ECD0284601F0C1
:106810001FFC0028E7D02046FFF7E2FC2846BDE831
:10682000384001F0FDBB00BF18840100F04CFF1F91
:1068300038B5044691B12A482A4908F023F90923BA
:1068400084F84C3C04F6784001F0F0FB04F5456513
:10685000284601F0F7FB002835D138BD00F6784511
:10686000284601F0EFFB0028F0D0284601F0F0FBAD
:106870000028EBD01C491A4808F004F90B2384F8CF
:106880004C3C04F5446001F0B1FB1849144808F091
:10689000F9F804F5006001F09DFA284601F0C6FB06
:1068A00004F5476001F0C2FB04F6584001F0BEFB5E
:1068B00004F5456504F5486001F0B2FB284601F097
:1068C000C1FB0028C9D0284601F0C2FB38B12046E0
:1068D000FFF786FC2846BDE8384001F0A1BB38BD73
:1068E000F04CFF1F0084010050840100608401000F
:1068F00070B5044659BB15466AB900F5486630467E
:1069000001F0A0FB00283DD104F54565284601F0C3
:1069100099FB50BB70BD2C492C4808F0B3F80723F5
:1069200084F84C3C2A49294808F0ACF804F580600A
:1069300001F062FA04F5006001F05EFA04F65840D6
:1069400001F06EFB04F5476001F06AFBDCE7012112
:10695000204801F043FF01211E4801F04BFF1E4972
:106960001A4808F08FF80223DAE7284601F070FB96
:1069700038B12046FFF734FC2846BDE8704001F0EE
:106980004FBB70BD304601F063FB0028BCD01349FB
:106990000E4808F077F8304684F84C5C01F046FB6E
:1069A00004F6884001F042FB94F84E3C43B904F5EC
:1069B0004565284601F03AFB012384F8983CA5E799
:1069C0002046FFF70DFCF2E788830100F04CFF1F23
:1069D0007084010058A5FF1F70830100D08301005F
:1069E000F8B5044600293BD102B9F8BD00F6684568
:1069F000284601F00DFB002840F092805849594884
:106A000008F040F894F84D3C072284F84C2C002BF9
:106A100040F09D8004F555674FF49665012603E02C
:106A2000013D84F85D6D0AD094F85C3D03F0FF01F0
:106A3000002BF5D13846FEF799FE013DF4D104F65E
:106A4000584001F0EDFA04F5476001F0E9FA04F569
:106A5000456001F0E5FA04F5496001F0E7FA3EE02F
:106A600000F66845284601F0D3FA002842D13E4995
:106A70003C4808F007F894F84D3C022284F84C2C6E
:106A8000002B68D104F555674FF49665012603E0A5
:106A9000013D84F85D6D0AD094F85C3D03F0FF0180
:106AA000002BF5D13846FEF761FE013DF4D104F626
:106AB000584001F0B5FA04F5476001F0B1FA04F569
:106AC000456001F0ADFA04F5496001F0AFFA01212B
:106AD000264801F083FE0121244801F08BFE04F6D4
:106AE000884001F09DFA94F84C1C1E48BDE8F8401F
:106AF00007F084BD1E491B4807F0C4FF012384F83A
:106B00004C3C284601F08CFA94F84D3C13B194F8B3
:106B10004F3C03B394F84C3C013B012BB2D9F8BD78
:106B20001449104807F0AEFF062384F84C3C284671
:106B300001F076FA94F84D3C13B194F84F3C33B120
:106B400094F84C3C063B012B7FF664AFF8BD204621
:106B5000FFF746FBF4E72046FFF742FBDAE700BF0A
:106B600088830100F04CFF1F7083010058A5FF1FB0
:106B70007C8401009484010038B590F84C3C0446B4
:106B80000B2B0DD8DFE803F0363C42484E545A61D7
:106B900068066F7611462046FFF71CFE94F84C3CC1
:106BA00003B138BD04F5806001F030F90028F8D158
:106BB00004F5006001F02AF90028F2D1204601F026
:106BC00025F90028EDD104F54965284601F03AFA87
:106BD00028B994F8983C13B1284601F021FA2846C8
:106BE00001F030FA0028DCD0284601F031FA002804
:106BF00046D138BD2046FFF7F3FE94F84C3CCFE772
:106C00002046FFF713FB94F84C3CC9E72046FFF7FA
:106C100069FB94F84C3CC3E72046FFF7C5FB94F8AA
:106C20004C3CBDE72046FFF72DFD94F84C3CB7E700
:106C30002046FFF765FD94F84C3CB1E7114620462D
:106C4000FFF722FC94F84C3CAAE711462046FFF7D8
:106C500065FC94F84C3CA3E711462046FFF7ACFCDA
:106C600094F84C3C9CE711462046FFF7E1FD94F870
:106C70004C3C95E72046FFF73BFE94F84C3C8FE7F1
:106C8000284601F0D3F9002384F8983C38BD00BFB2
:106C900090F8193D33B9044B1B780BB9FFF764B971
:106CA000FFF76ABFFFF7DEB9540EFF1F08B500F506
:106CB000566001F0C5FA034BA3FB0030C0F3C710C8
:106CC00008BD00BF8988888808B500F5566001F0C6
:106CD000EDF9002008BD00BF034600895A8980B243
:106CE00092B2904210B41AD05C685A8992B20020D5
:106CF00034F912200A8018735A89013292B25A81EB
:106D000059891A8889B292B2914204D358815DF8A8
:106D1000044B0120704701205DF8044B70471A7B3B
:106D200002F0FF00002ADFD15DF8044B704700BF7E
:106D30002DE9F04F894690F81A1D85B00446154696
:106D40001E4609B189F0010931462046FEF766FF6B
:106D5000002E00F02081013EF6B205EB4606DFF87A
:106D60004884023D04F5566AA3464F4628E09BF846
:106D70003C2D002A3BD09BF8182D012A00F0CF8033
:106D800055D3022A00F01C81BDF90C100BF54060B0
:106D900000F038FD98F800200A2A48D0002814BFD7
:106DA0003946002122465846FFF772FF9BF84C2CCB
:106DB0001AB198F800100A2947D0B54200F0EB80CC
:106DC00035F9021F9BF81B2DBBF93E0D090291FB03
:106DD000F0F109B2ADF80C10002A40F099800DF1E5
:106DE0000E01504601F0DCF904460028BFD19BF8A3
:106DF000182D012A00F09280C0F0B480022A40F0E1
:106E0000CD80BDF90C100BF5406000F0FBFC0028B4
:106E100000F0F280002F00F0C28198F800200A2ACA
:106E20004FF000044FF00101BCD1D8E0002422460D
:106E300039465846FFF72CFF98F800200A2ABCD1A3
:106E40009BF84C2C002A00F0E680911FC9B2012962
:106E500040F2EF80D34BBDF90C101878BBF91C4DF4
:106E6000002800F0A381013AD2B2012A00F2EE809C
:106E70000BF6085000F054FC9BF83C2D81462AB1DB
:106E80009BF84C2C013A012A40F2D38119FB04F4FF
:106E9000584624B200F0BCFF002840F0DE800BF51D
:106EA000006000F0B5FF002840F0D7800BF580634C
:106EB0001846009300F0F2FE204404B2584600F059
:106EC000A7FF002840F0D280009800F0A1FF002822
:106ED00040F0CC800BF5006000F0E0FE204404B2EE
:106EE000009800F095FF002840F0C6800BF5006088
:106EF00000F08EFF002840F0BF809BF84C2C002A49
:106F000040F09181584600F0C9FE204404B2B3E03D
:106F10000BF6284000F098FF074660E70024BDF913
:106F20000C100BF5406000F06DFC9BF84C2D814679
:106F30000BF55463002A57D001228BF84D2D1846CB
:106F400003A9FFF7C9FE98F80020ACB9B9F1000F0A
:106F500012D10A2A7FF431AF224649465846FFF73C
:106F600097FE69E7002F7FF461AF98F800200A2AA6
:106F70007FF423AF3C465AE70A2AEDD02246494621
:106F80005846FFF785FE9BF84C2C002A7FF411AF82
:106F9000B5427FF415AF05B0BDE8F08FBDF90C1018
:106FA0000BF5406000F02EFC70B3002FE2D098F893
:106FB00000200A2A4FF000043FF439AF0121F1E626
:106FC000BDF90C100BF5406000F01CFC98F8002097
:106FD0000A2A7FF4E3AE002814BF39460021224676
:106FE0005846FFF755FE27E71846BDF90C100093E9
:106FF000FEF7BCFB009BA2E798F800200A2A7FF46A
:10700000DCAE04460146EAE798F800200A2A7FF43D
:10701000D4AE04460BE70BF5806000F0F7FE0028C5
:1070200000F0D3809BF84C2C911FC9B201293FF688
:1070300011AF5C4BBDF90E101A78BBF91E4D002A3A
:107040007FF416AF11FB04F424B200E0002458468C
:1070500000F0DEFE00283FF422AF0BF580635846B7
:10706000009300F0D5FE00283FF42EAF009800F00A
:10707000CFFE00283FF43AAFDBF8A42CDBF8B00CCD
:10708000DBF8AC1CDBF89C3CCBF89C2C00FB02F042
:10709000DBF8B42CCBF8A44C01FB0401DBF8A80C02
:1070A000DBF8B84C03FB021EDBF8BC3CDBF8A01C91
:1070B000DBF8C82CCBF8A00C04FB10EEDBF8D44CAA
:1070C000DBF8D00C01FB13E104FB02F4DBF8C03C5D
:1070D000CBF8C02CC913DBF8D82C01F30E0109B290
:1070E00000FB014CDBF8CC4CDBF8DC0CCBF8A81C2B
:1070F00003FB02CC00FB14CCDBF8C42CDBF8E00C67
:10710000DBF8EC3CCBF8C81CDBF8F81CCBF8C44C23
:1071100002FB10CCDBF8E42CDBF8F40C019201FB51
:1071200003F14FEAEC3C0CF30E0C0FFA8CF200FB6F
:107130000219DBF8FC4CCBF8CC2CDBF8F01CCBF8BC
:10714000EC2C019ACBF8E43CDBF8003D02FB0499FF
:10715000DBF8E84CDBF8042DCBF8E81C03FB1199B5
:1071600004FB12994FEAE93909F30E090FFA89F481
:10717000CBF8F04C584600F04BFE002841D00BF500
:10718000496000F05FFF01460BF5426000F0FEFB36
:107190009BF85C2D72B301228BF85D2D0DE63C4609
:1071A00039461CE7540EFF1FAC78FF1F9BF83C0DBF
:1071B00000283FF402AE013AD2B2012A3FF6FDADFB
:1071C0000BF5526000F00CFCF7E50BF5006000F0E9
:1071D0001DFE00287FF426AF584600F017FE002859
:1071E0007FF420AF0BF5496000F02CFF00283FF43E
:1071F000E4AD17E7211809B20BF55560FEF7B6FAB2
:10720000DBE5009800F004FE0028B8D10BF5006023
:1072100000F0FEFD0028B2D10BF5446000F0B4FE92
:10722000484404B2ABE7584600F086FD204404B25F
:1072300022E701460BF5526000F0D2FB26E600BFC4
:107240002DE9F04F884690F81A1D85B00446154682
:107250001E4609B188F0010831462046FEF7DEFCE3
:10726000002E00F01A81013EF6B204F6284305EB29
:107270004606D64F0093023D04F5566926E094F881
:107280003C3D002B39D094F8183D012B00F00F81C4
:1072900054D3022B00F05D81BDF90C1004F5406061
:1072A00000F0B0FA3B780A2B48D0002814BF4146C2
:1072B000002152462046FFF7EBFC94F84C3C13B1FA
:1072C0003B780A2B42D0B54200F0E78035F9021F27
:1072D00094F81B3DB4F93E2D090291FBF2F109B27D
:1072E000ADF80C10002B40F0DB800DF10E0148468C
:1072F00000F056FF82460028C1D194F8183D012BBA
:1073000000F0D380C0F0F780022B40F01081BDF96F
:107310000C1004F5406000F075FA002800F034818C
:10732000B8F1000F00F042813B780A2B4FF0000AC1
:107330004FF00101BDD11AE14FF0000A524641461B
:107340002046FFF7A5FC3B780A2BBCD194F8803D82
:1073500023B194F83C3D002B40F02B8194F8813D03
:10736000002BB0D0B4F81ECDBDF80E30D4F8A4EC8C
:10737000D4F8B01CD4F8AC0CD4F89C2CC4F89CEC19
:107380001CFB03F301FB0EF11BB2C4F8A43C00FB91
:107390000313D4F8B81C0191D4F8B41CD4F8A80C89
:1073A00002FB013E0199D4F8A03CD4F8C82CC4F8E3
:1073B000A00C01FB10EED4F8BC1CD4F8C00CC4F82F
:1073C000C02C03FB11EED4F8D43C03FB02F1D4F83B
:1073D000D02C4FEAEE3E0EF30E0E0FFA8EF302FBA8
:1073E000031CD4F8DC1C0191D4F8D81CD4F8CC2CA4
:1073F000C4F8A83CC4F8C83C019B00FB01CC03FBCB
:1074000012C1D4F8C40CD4F8E03C00FB1313D4F838
:10741000EC1CD4F8F80CC4F8C42CDB1303F30E02F4
:1074200013B2D4F8F42CC4F8CC3C00FB01FCC4F833
:10743000EC3C02FB03C3D4F8E42CC4F8E41CD4F8FD
:10744000FC1CD4F8F00C02FB0133D4F8001DD4F876
:10745000E82CC4F8E80C01FB1031D4F8043D02FB21
:10746000131B4FEAEB3B0BF30E0B0FFA8BF3C4F835
:10747000F03C04F5496000F0E5FD014604F542608A
:1074800000F084FA94F85C3D002B00F0A180012309
:10749000B54284F85D3D7FF419AF05B0BDE8F08FCB
:1074A000009800F0D1FC80461FE74FF0000ABDF9BC
:1074B0000C1004F5406000F0A5F994F84C1D8346CB
:1074C00004F55463002957D0012184F84D1D184656
:1074D00003A9FFF701FC3B78BAF1000F1AD1BBF109
:1074E000000F17D10A2B7FF4EEAE524659462046C4
:1074F000FFF7CEFBE4E6B8F1000F7FF41DAF3B7859
:107500000A2B7FF4E0AEC246524641462046FFF7C2
:10751000BFFB18E70A2BE8D0524659462046FFF732
:10752000B7FB94F84C3C002B3FF4CDAEC8E6BDF958
:107530000C1004F5406000F065F960B3B8F1000F7D
:10754000E1D03B780A2B4FF0000A3FF4F7AE01215F
:10755000AFE6BDF90C1004F5406000F053F93B783C
:107560000A2B7FF4A2AE002814BF414600215246E8
:107570002046FFF78DFBA3E61846BDF90C100193DA
:10758000FEF7F4F8019BA2E73B780A2B7FF49BAE51
:1075900082460146EBE73B780A2B7FF494AE8246A5
:1075A000524641462046FFF773FBCCE6C2464146B1
:1075B000DDE7BDF90C1004F6085000F0B1F8014603
:1075C00004F5526000F00CFAC8E600BFAC78FF1F6B
:1075D0000BEB000109B204F55560FEF7C7F872E63F
:1075E00010B490F8194D1CB95DF8044BFFF7A0BB1F
:1075F0005DF8044BFFF724BE2DE9F0478046C0B08C
:107600003C4801F0C3F8B8F85A2DB8F8583D92B28A
:107610009BB29A4266D0B8F85A2DB8F8583D92B24B
:107620009BB29A423DD3B8F85A1DB8F8503DB8F80D
:10763000582D13FA82F35B1A9BB20A282BD9632BBD
:1076400029D902381FFA80F9B9F1640F28BF4FF029
:10765000640909F1FF35ADB20DF1100A0AEB4505D9
:107660000DF10E0408F5556700260DF10E013846A0
:10767000ADF80E60FFF730FBBDF80E3024F8023F86
:10768000A5424FF00003F0D1009352464B460A2129
:10769000184800F0BBFF98F83C3D4BB940B0BDE83E
:1076A000F087B8F8583DB8F85A2D9B1A9BB2C4E73A
:1076B00008F55268404600F001FA4F28EED90DF166
:1076C000100A544640AD21464046033400F0CCF940
:1076D000AC42F8D15146F022074806F03FFF40B0D7
:1076E000BDE8F08798F85C3D002BD4D0B8F8503D49
:1076F000A3E700BF58A5FF1FF04CFF1F00224FF467
:107700008041818002804280827182600273704772
:10771000C9014B42D201018043808280704700BF83
:10772000B0F9003010B47BB182798AB18368B3F5C7
:10773000166F03F1010212D9002142F6DF639A426B
:10774000826001D90023837108465DF8044B7047BD
:107750008B421ADC00230122827183600373047B55
:107760000C4BB0F9041053F824300134E4B20B2C64
:1077700003FB01F188BF002304734FEAE13188BFA6
:10778000037301F30F0109B2D7E7B0F902308B425E
:10779000E0DAD9E7AC84010030B4002200240025EF
:1077A000C0E900458260C260028242618261027764
:1077B00030BC704770B400250024C0E90045432662
:1077C0000E4D04E00134322C10D015F8106CB1428B
:1077D00005F11005F6D10A49E4B201EB0414D4E92D
:1077E000024554EA0501C0E9004502D1042070BCFD
:1077F00070478260C36070BC002070471085010034
:10780000008501002DE9F0434669456807688469F1
:1078100086614FEAE67906FB05F307FB0933A6FB11
:1078200007899944038A4FEAD87201EB610142EA61
:107830004902013302F31E02C4EB420211449BB21F
:1078400041F27072934283B04161038203D0007FA2
:1078500003B0BDE8F08386FB0123D40F44EA430460
:1078600004F31E0404FB05F5E31707FB035381FB38
:107870000189A4FB074586FB06671D444FEAD872C1
:10788000F30F067FE40F42EA490243EA470302F39B
:107890001E0203F31E03D11844EA4504836804F36F
:1078A0001E02A1EB420206B1C3689A420446B4BF6D
:1078B000002001208642207707D000901BB20648A6
:1078C000064912B207F03EF9207F0023238263614C
:1078D000A36103B0BDE8F083F04CFF1FDC8401001E
:1078E00000234361836103770382704700220260B3
:1078F0008280C280704700BF2DE9F0410023224DF5
:10790000432404E00133322B3AD015F83340A1422E
:10791000F8D11D4FDBB217EBC30731D080460068AA
:107920007B88A8F80430164618B10AF07BFBB8F83B
:10793000043058000AF074FBB8F80430C8F80000AE
:10794000DBB106EB4603002406EB830625462846FA
:107950000CF08EF880FB0601C30F43EA4103D8F810
:1079600000107A6803F30F0321F814300134B8F8DB
:107970000430A4B2A3421544E9D80020BDE8F08148
:107980000420BDE8F08100BF20880100C38830B426
:107990005A1C8488056892B29442C28098BF002223
:1079A00035F9133098BFC28019B1584200B230BCCB
:1079B0007047184630BC704738B504460025018032
:1079C000258101EB41006581657325730AF028FB71
:1079D00004F110032576606025616361204638BD9F
:1079E000037E01F50061002B36D0032B70B42BD140
:1079F0000469027B2143016102F0FF01002A30D1BA
:107A00004468038942699BB203EB430316785578B7
:107A10009278E65423445D709A70038901339BB2D7
:107A200003810289038892B29BB29A4228BF0181E6
:107A30000289438992B29BB29A4209BF0122037E16
:107A4000037E0273002202610133DBB2052B88BF83
:107A50000023037670BC704709030123016103769C
:107A6000704701224273EDE70289438992B29BB2CB
:107A70009A4210B504461AD00846616863899BB2E1
:107A800003EB43031944032207F0A2FF00212173F3
:107A9000638901339BB263816289238892B29BB26E
:107AA0009A4202D36181012010BD012010BD037BE9
:107AB00003F0FF00002BDFD110BD00BF4289038916
:107AC00092B29BB29A4212D04289038992B29BB27F
:107AD0009A4207D342890188038911FA83F3981ADD
:107AE00080B2704703894089181A80B27047027BC0
:107AF00002F0FF030AB1008870471846704700BFC4
:107B000000230376704700BF0346002110B403F83A
:107B1000011B00F2E93403F8011BA3424FF00002FD
:107B2000F9D1A0F8EA23A0F8EC23A0F8EE23A0F8FE
:107B3000F023C0F8F423A0F8F823A0F8FA23A0F863
:107B4000FC23A0F8FE235DF8044B70472DE9F04FAD
:107B50004FF0000A85B0A0F8EAA39DF838400D78F0
:107B600002949DF83C4003940192EDB1DFF8289116
:107B7000484F40F2E238412D00F08880012642242F
:107B800004E0A54246D017F82E401646721CD2B229
:107B900002EB420E002CF4D10AF1010A5FFA8AFAD4
:107BA00011F80A50002DE6D10446D0F8F453BDF880
:107BB0000810A0F8FC13BDF80C10A0F8FE13019AF1
:107BC00045F6C051B1FBF2F2B1FBF3F0A4F8EE239D
:107BD000A4F8F80325B128460AF024FAB4F8F8030B
:107BE0000AF01EFAB4F8F813C4F8F40371B10023D4
:107BF0001A461E464C0801250133A2429AB234BFF0
:107C0000057006708A4200F10100F5D3002005B02E
:107C1000BDE8F08F06EB460207EB82021D4D147A99
:107C2000002CB9D0B0F8EA2306EB460605EB860631
:107C3000013C02F1010E5EFA84FED6F804C01FFA80
:107C40008EFE4FF0004603E07245A0F8EA23A3D071
:107C500000EBD20502F0070436EA0C0B19F804B069
:107C60006C780CBF4BEA040424EA0B0402F1010B0C
:107C700042456C701FFA8BF24FEA5606E4D9002396
:107C8000A0F8EA33042005B0BDE8F08F014D0824C8
:107C90000026C7E7B0890100C08B01000378002BE4
:107CA00040D010B4B0F8EC13224C00EBD10301F03B
:107CB00007025B78A25C1340B0F8FA2305D0D0F835
:107CC000F4339B5C83B3B0F9FC33B0F8F843013272
:107CD00092B29442A0F8FA239CBF0022A0F8FA23A3
:107CE000B0F8F023B0F8EE43013292B29442A0F81B
:107CF000F02313D84A1CB0F8EA4392B20021944210
:107D0000A0F8EC23A0F8F01308D80170A0F8EC1349
:107D1000A0F8FA135DF8044B1846704718465DF852
:107D2000044B704718467047B0F8FC335B421BB2F7
:107D3000CBE700BFC08B01000378002B40D010B40C
:107D4000B0F8EC13224C00EBD10301F007025B7892
:107D5000A25C1340B0F8FA2305D0D0F8F4339B5C52
:107D600083B3B0F9FE33B0F8F843013292B29442D3
:107D7000A0F8FA239CBF0022A0F8FA23B0F8F02361
:107D8000B0F8EE43013292B29442A0F8F02313D837
:107D90004A1CB0F8EA4392B200219442A0F8EC23C6
:107DA000A0F8F01308D80170A0F8EC13A0F8FA13AB
:107DB0005DF8044B1846704718465DF8044B704751
:107DC00018467047B0F8FE335B421BB2CBE700BFEA
:107DD000C08B0100B0F8EC336BB9B0F8F03353B995
:107DE000B0F8FA333BB90122A0F8EC33A0F8F03335
:107DF000A0F8FA330270704700230370A0F8EC3348
:107E0000A0F8F033A0F8FA33704700BF007870474D
:107E1000B0F8EC3343B9B0F8F0332BB9B0F8FA034B
:107E2000003018BF01207047012070470022026017
:107E300042600281C260026102754275704700BFF4
:107E400080E80600704700BF2DE9F043C568414C4B
:107E500002690689056104FB05F3DF17DB0F43EABE
:107E60004703013603F31E03C2EB430303EB811107
:107E7000B3B23C2B83B0C160038103D0007D03B05B
:107E8000BDE8F08381FB05894FEAD873064643EAD3
:107E9000490303F31E0304FB03F481FB0101E31711
:107EA00085FB0589E40F44EA4304C20F4FEAD87307
:107EB000307D04F31E0442EA410243EA490302F31F
:107EC0001E0203F31E031344A3EB4404A0B933685A
:107ED0009C4220DA727D0132D2B2092A727518D919
:107EE000B27D092A32D90020307500233381F36036
:107EF000336103B0BDE8F08373689C420DDBB27D53
:107F0000717D0132D2B20929B2751DD9092A1BD857
:107F100001203075E9E77075E5E7717D00220929D8
:107F2000B275F5D832750022B27500921BB222B23A
:107F300009490A4806F006FE0848B37D727D0849E3
:107F400006F0ACFD307DD0E70022EBE70122327570
:107F5000EBE700BF4DC5FB30C88B0100F04CFF1FA5
:107F6000F08B01000023C360036103750381704738
:107F700000224FF48041018082704260027270479B
:107F800001EB810101807047837823B3426842F698
:107F9000DF639A4210B40BD80023013245F6BF517B
:107FA0008A4288BF002242605DF8044B1846704741
:107FB000017A0A4BB0F9004033F911300131C9B2EE
:107FC0003B2903FB04F388BF0021DB13017203F399
:107FD0000F031BB2E1E71846704700BF0C8C01008D
:107FE0000023012282704360037270470023837074
:107FF000704700BF002202604260704702EB4202FD
:10800000D20045F6C05303FB01210160704700BF59
:1080100003680248A0FB033000097047ABAAAAAA74
:1080200003680BB101234360704700BF0023436026
:10803000704700BF43681BB102680AB10B4443603C
:10804000704700BF4068003018BF0120704700BF74
:10805000036833B1406828B183422CBF002001205F
:1080600070471846704700BF38B500254FF461636C
:10807000044685828381C5820570456085600576EA
:10808000457642F6302009F0CBFF231D206125778D
:10809000A360204638BD00BF002383820370C382E3
:1080A0004360037643760377704700BF3B4BA3FBE7
:1080B0000232520802EB42020A4491422DE9F04199
:1080C00034D003310332012503E003319142457678
:1080D0002CD0037E03F0FF04002BF6D10769838ABE
:1080E00011F8038C11F802CC11F801EC9BB203EBF0
:1080F0004303FE1807F8038086F801C086F802E003
:10810000838A01339BB28382868A8389B6B29BB20B
:108110009E4228BF8482848AC38AA4B29BB29C42B6
:1081200001F1030108BF05769142D2D1037FBBB9AB
:10813000C28A838A92B29BB29A4222D0C28A838A2E
:1081400092B29BB29A420DD2838AC28A9B1A9BB288
:10815000B3F5967F94BF002301230377BDE8F08138
:10816000BDE8F081C18A8389828A13FA82F35B1A9F
:108170009BB2B3F5967F94BF002301230377BDE83C
:10818000F081027E02F0FF03002AE6D08389B3F576
:10819000967F94BF00230123DFE700BFABAAAAAA02
:1081A000027F002A3FD0F0B5037883B1032B3CD186
:1081B0004368C3F30B03A3F500630B80037801331B
:1081C000DBB2052B88BF002303701046F0BD848A04
:1081D000C38AA4B29BB29C422AD00569C38A9BB2CF
:1081E00003EB4303EC180026EF5C94F802E065789B
:1081F0000676C38A01339BB2C382C48A8389A4B240
:108200009BB29C4200D3C6820446002344F8043F3C
:108210000771457180F806E0436884601B0BA3F585
:1082200000630B80CAE71046704700230B80C5E748
:10823000047E04F0FF03002CCFD103771A46C4E775
:10824000C28A838A92B29BB29A421BD0C28A838A24
:1082500092B29BB29A4208D3C38A818A8289581A01
:1082600080B290420AD9002070478289818AC38AED
:1082700012FA83F3581A80B29042F4D800EB40000F
:1082800080B27047037E002BEDD1808900EB400067
:1082900080B2704770B504460626002585F00105BA
:1082A0002946204601F076F82946204601F07AF862
:1082B0002946204601F07AF82946204601F07AF84E
:1082C0002946204601F07AF82946204601F07AF83E
:1082D0002946204601F07AF8013EFA21204601F0B5
:1082E000BBF816F0FF06D9D13146204601F05EF802
:1082F0003146204601F05EF83146204601F05EF836
:108300003146204601F05EF83146204601F05EF825
:108310002046012101F04AF82046FA2101F09CF89C
:108320002046012101F046F82046FA2101F094F898
:108330002046012101F042F82046FA2101F08CF894
:108340002046012101F03EF82046FA2101F084F890
:108350002046012101F03AF82046FA2101F07CF88C
:108360003146204601F032F82046FA2101F074F837
:108370003146204601F026F82046FA2101F06CF83B
:108380003146204601F01AF82046FA2101F064F83F
:108390003146204601F00EF82046FA2101F05CF843
:1083A00031462046BDE8704001F000B82DE9F04F9D
:1083B00000244FF41676054685B084810470C4818C
:1083C0004474047486804FF4166009F029FE4FF45B
:1083D000FA73AC83AB82A860EC8385F8214085F802
:1083E00020404FF4FA6009F01BFEAC85A861EC85D3
:1083F000AE8485F8304085F831404FF4966009F03E
:108400000FFE05F1600B05F144020192A8626C6356
:108410002146AC63EC632C645B466C64AC64EC6436
:108420002C65A5F85440AC65EC6505F1B00223F865
:10843000021B9A424FF00000F9D105F1BC030293F0
:10844000A5F8B000C5F8B400C5F8B8001A4605F59F
:10845000A47422F8020BA2424FF00001F9D105F5F5
:10846000AA7AA5F84811C5F84C11C5F85011524622
:1084700005F5F07422F8021BA2424FF00000F9D17A
:1084800005F5F679A5F8E001C5F8E401C5F8E801BD
:108490004A4605F50A7122F8020B8A42FBD105F51E
:1084A0000D78424605F52170002122F8021B824218
:1084B000FBD105F52476324605F54770002122F8F8
:1084C000021B90424FF00004F9D14FF48042012387
:1084D0004FF40061A5F81E23A5F82023A5F8222358
:1084E000A5F82423A5F82623A5F82823A5F82A23F0
:1084F000A5F82C23A5F82E23A5F83023A5F83223C0
:10850000A5F83413A5F8361385F84033214685F8CD
:108510001C4385F83843C5F83C4385F84143A5F82A
:108520004243A5F84443C5F8484385F84C4310221C
:10853000019803930BF0EAFD039B6B632D4A019BAB
:10854000AB63EA63214685F84040502258460BF061
:10855000DDFD0C21284AC5F858B0A5F85410EA658D
:1085600021468C220298DFF8A0B00BF0CFFD2A271D
:10857000029BC5F8B4302146A5F8B070C5F8B8B074
:108580008C2250460BF0C2FD2146A5F84871C5F873
:1085900050B1C5F84CA13C2248460BF0B7FD174B33
:1085A000C5F8E8310622A5F8E0212146C5F8E49196
:1085B000502240460BF0AAFD114BC5F830320A227A
:1085C0002146A5F82822C5F82C828C2230460BF0D3
:1085D0009DFD0C4BC5F88C322846A5F88472C5F871
:1085E000886200F013FD2846FFF754FE284605B0C8
:1085F000BDE8F08F800DFF1F140DFF1F980DFF1FAA
:10860000000DFF1F2C0DFF1FA40DFF1F2DE9F04FC4
:10861000067885B0DDF83880002E70D090F84C5385
:108620000446002D6BD11F46554B15461A780E4651
:1086300052B990F81C13012251401A7000F0AEFE9E
:108640005049514806F01EFA711E0A2907D8DFE882
:1086500001F05C5F6E7162656806066B5900B4F9E3
:1086600020A3002F4BD0013FBFB205EB4707464682
:10867000023D4FF0010935F9023FB4F8362303FB00
:108680000AF3DB1303F30F0313449BB2B3F5805FCC
:1086900004D3B4F844230132A4F84423B8F1000F02
:1086A0004ED03278ADF804308DF8062094F82030A2
:1086B000019A039203F0FF0B002B3ED1A069A38B1C
:1086C0009BB200EB8300042203A907F081F9A38B7E
:1086D00001339BB2A383A28BA38A92B29BB29A422C
:1086E00028BFA4F81CB0A28BE38B92B29BB29A4233
:1086F00008BF84F82090AF4206F10106BBD105B057
:10870000BDE8F08FB4F932A3ABE7B4F922A3A8E730
:10871000B4F924A3A5E7B4F92AA3A2E7B4F92EA3D8
:108720009FE7B4F92CA39CE7B4F930A399E7B4F917
:1087300026A396E7B4F928A393E784F82190DAE713
:10874000ADF800308DF8028094F82030009A029243
:10875000002BF2D1A069A38B9BB200EB8300042213
:1087600002A907F035F9A38B01339BB2A383A28B37
:10877000A38A92B29BB29A42B5D3A4F81C80B2E706
:1087800050A5FF1F848C0100F04CFF1FC28B838B10
:1087900092B29BB29A4219D0C28B838B92B29BB297
:1087A0009A4208D3C38B818B828A581A80B2904236
:1087B00088BF00207047828A818BC38B12FA83F3B3
:1087C000581A80B2904288BF0020704790F820303D
:1087D0000BB100207047808A704700BF38B5044C49
:1087E00023788B420D4601D000F0DCFD257038BDAA
:1087F000AD78FF1F80F84113704700BF70B5314E50
:1088000033788B421DD0013B05460C46092B09D815
:10881000DFE803F01D2125292D3105080835002149
:1088200000F0D8FD631E092B0AD8DFE803F02C31D5
:10883000363B40450509090B2846012100F0CAFDD9
:10884000347070BD2846012100F0F0FDF8E70021EA
:1088500000F0ACFDE6E7002100F0ACFDE2E700210E
:1088600000F0ACFDDEE7002100F0ACFDDAE700210E
:1088700000F0ACFDD6E7002100F0C2FDD2E70021F8
:1088800000F0D4FDCEE72846012100F08FFDD7E7A8
:108890002846012100F08EFDD2E72846012100F094
:1088A0008DFDCDE72846012100F08CFDC8E7284664
:1088B000012100F08BFDC3E72846012100F0A0FD57
:1088C000BEE700BFAC78FF1F38B5057805B138BDED
:1088D000044600F0C3FB0123294623702046BDE86F
:1088E0003840FFF78BBF00BF2DE9F04FD0F83C3385
:1088F000027801338DB00446C0F83C33002A00F002
:10890000B980D0F848134BF67F32914211D9944A7E
:108910001278511E042900F2F580022A00F0158118
:1089200000212046FFF76AFFD4F83C330022C4F848
:10893000482345F6BF52934200F2C78094F838337B
:10894000002B40F0D380E28BA38B92B29BB29A4271
:1089500000F0D280E28BA38B92B29BB29A4280F05D
:108960009980A38BE28B9B1A9BB2002B00F09C801A
:10897000E289A38992B29BB29A4200F0E180E28937
:10898000A38992B29BB29A4280F0D280A389E289F5
:108990009B1A9BB2012B6AD9002594F841A3B4F825
:1089A0003493B4F91E83AB4603AF04AEA289E389C6
:1089B00092B29BB29A4200F0B680A168E3899BB262
:1089C00001EB830104220AA807F002F884F810B032
:1089D000E38901339BB2E381E289A38892B29BB21F
:1089E0009A4201D3A4F80EB09DF82A10A28DE38D0F
:1089F000795592B29BB29A4200F08F80A16AE38DC2
:108A00009BB205AA31F8131084F830B0E38D22F838
:108A1000151001339BB2E385E28DA38C92B29BB219
:108A20009A4201D3A4F82EB0BAF1000F0BD0BDF8D2
:108A300028309BB2002B6AD0BDF8283040F6FF7278
:108A40009BB2934263D0BDF82830C9EB03031BB23D
:108A500003FB08F3DB1303F30F0326F8153001358E
:108A6000022DA3D194F84C33002B00F085800DB07B
:108A7000BDE8F08F3B498B42F9D990F84013C0F81C
:108A80003C2381F0010180F8401300F083FC0DB01D
:108A9000BDE8F08FE18BA38AA28B13FA82F35B1AF5
:108AA0009BB2002B7FF464AF2F4B1A78002A3FF45F
:108AB0005FAF002294F81C131A70204600F06EFC81
:108AC0002A492B4805F0DEFF52E794F840130023B3
:108AD00081F00101C4F83C3384F84013204600F0D3
:108AE00059FC94F83833002B3FF42DAF204600F0AA
:108AF00047FC84F84C0326E794F82030002BD3D0B1
:108B0000A38A32E7063A012A3FF610AF08E7B4F825
:108B100042330133A4F8423395E794F83030002B08
:108B20007FF46CAF80E7237C002B7FF446AF5BE7DC
:108B3000E189A388A28913FA82F35B1A9BB229E721
:108B4000237C002B93D0A38824E7074B1B78002BB2
:108B50003FF4E6AE00210748FBF70EF8E0E600BF61
:108B6000AC78FF1F7FA9030050A5FF1F8C8C01006C
:108B7000F04CFF1FB078FF1F08A92A46304609F0C5
:108B8000CBFB2B4608A90AAA04F134000AF008FE20
:108B90000A9B0B9AA649BDF810E00878BDF81210A0
:108BA0001A4402EBD2735B1403F30F039BB2C3EBC3
:108BB0000E02CB1AADF81820ADF81A30002828D1D3
:108BC0009C4B1B78002B44D19B4B1B78002B5CD11A
:108BD0009A4B1B78002B4AD1994B1B78002B40F005
:108BE0008880984B1B78002B75D1974B1B78002BF6
:108BF00063D1964B1B78002B55D1954B1B78002BDE
:108C00003FF435AF06AC214602229248F7F788FFC1
:108C10002DE701287ED0022800F08F80032800F085
:108C2000AE80042800F0BE80052800F0CE80072822
:108C300000F0DE800A2800F02781632800F03481EC
:108C400060287FF414AF022205A98348F9F7AEF833
:108C50000DE707AA2B4606A904F154000AF0D8F83C
:108C60002B4607A905AA7D48FCF74EF9ACE707AAF1
:108C700006A904F50A7002230AF0CAF807A902231C
:108C800005AA774801F032FFA6E707AA06A904F56E
:108C9000F07002230AF0BCF807A9022305AA714864
:108CA00002F0D4FE94E7204600F06AFB022301465E
:108CB00006AA6D48FEF794FC9FE707AA06A904F5EB
:108CC000217002230AF0A4F807A9022305AA674825
:108CD00000F0F8FF8DE707AA06A904F5A4700223A7
:108CE0000AF096F807A9022305AA614806F020FCBD
:108CF0007BE73146022307AA04F1B0000AF088F8A6
:108D00005C4B1B7807A9002B33D002225A48FAF794
:108D10004DF866E7474B1B78002B3FF4A8AE04F1F3
:108D2000540007AA2B4606A90AF072F82B4607A999
:108D300005AA4A48FCF7E8F899E6414B1B78002B56
:108D40003FF495AE2B46314604F1B00007AA0AF075
:108D50005FF8484B1B78002B63D0484B1B78002BE7
:108D600059D000953B4607A905AA4548FAF740F8AF
:108D70007DE6022305AA4348F9F780FC31E7314B31
:108D80001B78002B3FF473AE04F5A47007AA2B46A2
:108D900006A90AF03DF82B4607A905AA344806F0B3
:108DA000C7FB64E6244B1B78002B3FF460AE04F550
:108DB000F07007AA2B4606A90AF02AF82B4607A945
:108DC00005AA284802F042FE51E61C4B1B78002BF6
:108DD0003FF44DAE04F50A7007AA2B4606A90AF027
:108DE00017F82B4607A905AA1D4801F07FFE3EE6AD
:108DF000154B1B78002B3FF43AAE04F5217007AAFF
:108E000006A902230AF004F807A9022305AA1748B5
:108E100000F058FF2BE62A4607A91748F9F7C6FFC6
:108E200025E62B4607A905AA1648F9F727FC1EE6F2
:108E3000AC78FF1F580EFF1F5A0EFF1F550EFF1F65
:108E4000570EFF1F560EFF1F520EFF1F530EFF1F20
:108E5000590EFF1F18F5FF1FA473FF1F8084FF1F0B
:108E600070E5FF1F204FFF1FE8D2FF1FC822FF1F22
:108E7000A8A8FF1F540EFF1F1C7FFF1F50A5FF1F38
:108E80004830FF1F28BCFF1F204600F079FA06ACCF
:108E90000146022322460B48FEF7A2FB0A4B1B7831
:108EA000002B3FF4E4ADAEE6314604F1540007AACE
:108EB000022309F0ADFF07A902220448F8F70AFCD3
:108EC000D5E500BFE8D2FF1F590EFF1FE8BBFF1F0B
:108ED0002DE9F04F9DF828B09DF848A0BDF95480C9
:108EE000BDF950C09DF84C909DF824E09DF82C7081
:108EF0009DF830609DF834509DF8384080F81C3360
:108F00004FEACB1B4FEACA1AA0F820B3A0F830A34F
:108F10009DF83CB09DF840A09DF8443008F50068ED
:108F20000CF5006C4FEAC9194FEACE1EFF01F6019D
:108F3000ED01E401A0F834834FEACB1B4FEACA18D5
:108F4000DB01A0F836C39DF858C0A0F8329380F832
:108F500038C3A0F81EE3A0F82273A0F82463A0F899
:108F60002653A0F82843A0F82AB3A0F82C83A0F831
:108F70002E3319B1CEF1000EA0F81EE3B2B17F423C
:108F800076426D426442CBF1000BC8F100085B42AF
:108F9000A0F82273A0F82463A0F82653A0F8284371
:108FA000A0F82AB3A0F82C83A0F82E33BDE8F08FE8
:108FB00030B4B0F84243B0F844330025641B18BF06
:108FC00001245B1B18BF01230C701370A0F84253DF
:108FD000A0F8445330BC70470346002290F82100AB
:108FE00083F82120704700BF03460022407C5A745A
:108FF000704700BF0023C0F848337047D0F84803DB
:10900000704700BF90F84C03704700BF08B50121BE
:10901000052006F09FFE0121062006F09BFE01219F
:10902000032006F097FE0021042006F093FE0121A4
:10903000092006F08FFE01210A2006F08BFE012197
:109040000B2006F087FE01210C2006F083FE012193
:109050001820BDE8084006F07DBE00BF4F4A5049C9
:10906000F8B513684F4E504F504D514C43F4805358
:109070001360C02333700B68A2F55042083A43F0E6
:1090800000630B604FF0350E042312264021C7F811
:1090900000E02E6021601360136843F080031360CA
:1090A000136813F08003FBD14249434A434D0F68D4
:1090B0001268434C2E68CD6824683A441431324417
:1090C0000968404E404F2A4422440A44C2F34E02EB
:1090D0003E4D3F493F4C42F40042326045268022DB
:1090E0002E600A6021683C4A3C4E05F5002541F09F
:1090F000006121602035352139601224042134605B
:109100002B601160136843F08003136013461968E5
:1091100011F08004FBD1324A324B334DD2F800E0DB
:109120001B6832492F68D6680D6890F81C133048C8
:10913000734414323B4412682E4F33442B4413447F
:10914000C3F34E032C4E2D4D2D4A43F400433B6098
:109150008E274FF4407337602B600368294EA5F5C6
:1091600030450C3D43F001030360042740F2F31047
:1091700022231460376028601360136843F00103F2
:109180001360052006F0D2FD2146062006F0CEFD34
:1091900001210320BDE8F84006F0C8BD2C80044042
:1091A0003C80044021C00C4008B003400CB0034098
:1091B00020B0034038B003403CB0034040B003400F
:1091C00048B003402CB0034008B00B4000B003404F
:1091D00004E100E03080044024B00B400CB00B40B0
:1091E00038B00B403CB00B4040B00B4048B00B4097
:1091F000388004402CB00B401880044014B0044068
:10920000000004400400044030B583B04FF4006215
:109210000023ADF800208DF80230828BC38B92B210
:109220009BB29A42044600F08480A169E38B9BB212
:1092300001EB83010422684606F0CAFB002184F892
:109240002010E38B01339BB2E383E28BA38A92B2BB
:109250009BB29A4200D3E183414BBDF80010414AD2
:109260001B6811801A060DD53F4B1B689BB2ADF8E9
:109270000030237C009A019203F0FF05002B3AD0C6
:1092800001236374394B1B681B0614D5384B1A68CD
:1092900094F8303003F0FF01002B50D0012384F804
:1092A0003130324B04221A60D4F848330133C4F809
:1092B000483303B030BD94F8303003F0FF02002B88
:1092C000ECD1A16AA38D9BB221F81320A38D0133A9
:1092D0009BB2A385A18DA38C89B29BB2994228BF72
:1092E000A285A28DE38D92B29BB29A4204BF012364
:1092F00084F83030D5E7A068A38904229BB200EB44
:1093000083000DEB020106F063FBA38901339BB2DE
:10931000A381A289A38892B29BB29A4228BFA58159
:10932000A289E38992B29BB29A4204BF01232374BB
:10933000A8E790F82030002B7FF477AF8CE7A06A85
:10934000A38D9BB220F81320A38D01339BB2A3857C
:10935000A28DA38C92B29BB29A42C2D3A185C0E7E0
:1093600000B0034000C00C4010B0034000B00B4000
:1093700010B00B400148FFF747BF00BF58A5FF1FC3
:1093800008B5042006F0D8FCA0F10100B0FA80F086
:10939000400908BD032006F0C9BC00BF052006F047
:1093A000C5BC00BF062006F0C1BC00BF092006F006
:1093B000BDBC00BF0A2006F0B9BC00BF0B2006F000
:1093C000B5BC00BF0C2006F0B1BC00BF182006F0F1
:1093D000ADBC00BF10B549B10121092006F0A6FCC3
:1093E00001210C20BDE8104006F0A0BC0C4609206D
:1093F00006F09CFC21460C20BDE8104006F096BC0F
:1094000010B549B10121092006F090FC01210A2084
:10941000BDE8104006F08ABC0C46092006F086FC28
:1094200021460A20BDE8104006F080BC10B549B1C5
:109430000121092006F07AFC01210B20BDE8104033
:1094400006F074BC0C46092006F070FC21460B2087
:10945000BDE8104006F06ABC084606F081BC00BFBB
:10946000012070470846102244F2580106F0B0BAB5
:109470000346002203F8012B811D03F8012B8B42C8
:10948000FBD130B400F28675002423F8024BAB42C6
:109490004FF00002F9D142F20F73A0F88A37A0F81A
:1094A0008C37A0F88E37A0F89037A0F89237A0F844
:1094B0008627A0F88827C0F89427A0F8982780F876
:1094C0009A2780F89B2700F29C7300F2BC7423F863
:1094D000022BA3424FF00001F9D1A0F8BC1700F213
:1094E000BE7300F2DE7423F8021B9C424FF00002B0
:1094F000F9D16323A0F8DE27C0F8E427A0F8E82715
:1095000080F8E03730BC7047002342F20F726321CD
:1095100080F8E0170370A0F88837A0F88637C0F805
:109520009437A0F8BC37A0F8DE37A0F8983780F859
:109530009A3780F89B37C0F8E437A0F8E837A0F8EE
:109540008A27A0F88C27A0F88E27A0F89027A0F8EB
:1095500092277047F0B5044683B0002A7AD03F4F77
:109560004FF47A5E3E467546002014E09E42B8BF36
:109570001E469D42A8BF1D464B1D9BB2B3F5707F92
:1095800000F10100A1F2BB3138BF194683B228BFF8
:1095900089B29A420CD904EB4103B3F90630002B8F
:1095A000E4DC9E45A8BF9E469F42B8BF1F46E3E746
:1095B00072190EEB070352105B10D6187610951B2C
:1095C0001BB22DB236B212B201950096244925483D
:1095D00005F024FB94F8E037632B29D004EB430219
:1095E0000133DBB20F2BA2F89C67A2F8BE5704F23E
:1095F0009A7184F8E03704F2BC7004F2BA7725D887
:1096000000221346A4F8BC27A4F8DE2731F8026F25
:1096100030F8025F32442B44B94212B21BB2F5D18A
:1096200012111B11A4F8BC27A4F8DE3703B0F0BD5B
:1096300004F29A7104F2BC700B46024604F2BA7747
:1096400023F8026FBB4222F8025FF9D1002384F8AD
:10965000E037D5E7154616461346B5E780C1FFFF4C
:10966000B48C0100F04CFF1F2DE9F04FBDF82450E1
:10967000BDF928C0BDF92C80002A79D0AE1C013577
:10968000DFF8F0E01FFA8CFCB6B2ADB2C8F1000909
:10969000002729E04FEAE40A04F0070413F80AB0AF
:1096A0001EF804402BEA040403F80A4005F0070BF7
:1096B000EC101EF80BB013F804A04BEA0A0A03F8EA
:1096C00004A04C1DA4B2B4F5707F07F1010728BFB8
:1096D000A1F2BB31BFB22CBF89B22146023602359E
:1096E000BA42B6B2ADB243D000EB410AB41EBAF8EA
:1096F00006A0CCEB0A0A0FFA8AFACA45A4B2C9DB63
:10970000BAF1000F1CDBC2454FEAE40A04F007047B
:1097100013F80AB01EF8044044EA0B0403F80A40A8
:1097200005F0070B4FEAE5041EF80BB013F804A090
:10973000B4BF2AEA0B0A4BEA0A0A03F804A0C0E7FE
:109740004FEAE40A04F0070413F80AB01EF80440D4
:109750002BEA040403F80A4005F0070BEC101EF88E
:109760000BB013F804A02AEA0B0A03F804A0A8E738
:10977000BDE8F08F888D01002DE9F0471546B0F85F
:10978000862702440446507886B048409DF83860E9
:109790009DF83C801F4605F0C7FAB04200F2858074
:1097A000B4F88897DFF840C109F29D36B6B2B6F535
:1097B000707F28BFA9F1230105F1FF3005F10702F1
:1097C0002CBF89B2314600254FF47A5E04EB410389
:1097D00010F901AFB3F906309C45B8BF9C469E45D1
:1097E000A8BF9E46BAF1010F63D0BAF1030F62D051
:1097F000BAF1FF3F01D003EB43031D444B1D9BB265
:10980000B3F5707F26BFA1F2BB3189B219468242FF
:10981000DCD1D4F89437AB4247DA94F8E037632BC5
:1098200051D0B4F9BC37B4F9DE270292B6F5707F97
:1098300024BFA9F12306B6B24FF000090822314631
:109840000193204605ABCDF80090FFF70DFF9DF882
:1098500014303878584005F067FA7B7882469DF8D6
:109860001500584005F060FA5044C0B2804526D338
:10987000B4F88837A4F88E3703F2973292B2B2F573
:10988000707F4FF0040128BF293B4FF00100C4F85E
:109890009457A4F88A67A4F8981734BFA4F88C27C3
:1098A000A4F88C3706B0BDE8F087002006B0BDE80C
:1098B000F087ED1AA2E703EB4303ED1A9EE7484653
:1098C00006B0BDE8F0870EEB0C035B10C3EB0C0C8D
:1098D00044F63E1202FB0CFC1BB24CF3CF32A4F850
:1098E000BC37A4F8DE27A0E780C1FFFF70B582B0C7
:1098F000002501950095404B404AF2210446FFF7B0
:109900003BFF019500953E4B3E4A06460D21204601
:10991000FFF732FF94F89A37054666BB002849D016
:10992000002B4BD0013BDBB2012B84F89A3720D1BE
:10993000B4F88E3703F2BF3292B2B2F5707F28BF0F
:1099400003F1FF32A4F890275A1C92B2B2F5707F4F
:1099500024BFA3F2BF33A4F8923794F89B37237047
:109960004FF0000338BFA4F8922784F89A3784F8A0
:109970009B3702B070BD002BD4D1C4F8E437A4F8F3
:10998000E83701212048FEF729FF01211E48FEF794
:1099900031FF63210523012284F8E01784F89A3708
:1099A00084F89B27E5B9013BDBB2012B84F89A3799
:1099B000BED0DEE7002BB5D102B070BDC4F8E437ED
:1099C000A4F8E83701211048FEF708FF01210E48EE
:1099D000FEF710FF6322052384F8E02784F89A3706
:1099E000022384F89B3794F89A37013BDBB2012BB2
:1099F00084F89A379CD0BCE7908D0100AC8C0100B4
:109A0000948C0100988C010058A5FF1FB0F8E8372E
:109A100010B504464BB931220E4804F0F3FC002384
:109A2000C4F8E437A4F8E83710BDD4F8E427B2FB53
:109A3000F3F3C3F3072281F8323081F8312005486F
:109A4000332204F0DFFC0023C4F8E437A4F8E8373D
:109A500010BD00BFF04CFF1FB0F8E83710B504464A
:109A60004BB931220E4804F001FD0023C4F8E4375D
:109A7000A4F8E83710BDD4F8E427B2FBF3F3C3F33E
:109A8000072281F8323081F831200548332204F072
:109A9000EDFC0023C4F8E437A4F8E83710BD00BF9C
:109AA000F04CFF1FF0B5B0F89027B0F89217B0F85F
:109AB00088378A4293B0044608D29A4240F288809E
:109AC000B4F88C27934245D013B0F0BD9A4201D927
:109AD0009942F5D302250126704B714A01950096F3
:109AE0000D212046FFF748FE0195074600966D4B75
:109AF0006D4AFD212046FFF73FFE002F73D100285D
:109B000074D0B4F9DE17B4F9BC37B4F98E276748BE
:109B10000091674905F016F800216648FEF75EFEE1
:109B200000216448FEF766FE604804F0D3FCB4F8F8
:109B3000883742F20F72002163209342217084F82B
:109B40009A1784F89B17C4F89417A4F88C2784F804
:109B5000E007B9D1B4F89837042B00F08680C02212
:109B6000B4F88A172046FFF7F5FC2378012B51D073
:109B7000022B3ED0B4F9DE37B4F9BC07B4F88A172B
:109B8000029308220190009205ABC0222046FFF705
:109B90006BFDB4F89857013DADB2A4F89857002D6D
:109BA00044D02378A5F10305B5FA85F56D09012B9D
:109BB0008DF8145029D0022B03D105A92046FFF7B8
:109BC0004BFF0023C4F8943784F89B3713B0F0BDE3
:109BD0009942FFF475AF02250126019500962F4B9F
:109BE0002F4A0D217EE7257000288AD1B4F88837E6
:109BF00066E7B4F9DE17B4F9BC37B4F98E272B4801
:109C000000912D4904F09EFFB4E705A92046FFF717
:109C1000FDFED6E7B4F9DE17B4F9BC37B4F98E27E8
:109C200022480091254904F08DFFA3E724491F48ED
:109C300004F028FF29461F48FEF7D0FD29461D489D
:109C4000FEF7D8FD194804F067FC42F20F72632357
:109C5000257084F89A5784F89B57C4F89457A4F851
:109C60008C2784F8E03713B0F0BDB4F88E3703F2D8
:109C7000BF3292B2B2F5707F28BF03F1FF32A4F871
:109C800090275A1C92B2B2F5707F2ABFA3F2BF335D
:109C9000A4F89227A4F8923761E700BF948C0100E2
:109CA000988C0100A08C0100A48C0100F04CFF1FD7
:109CB000D48C010058A5FF1F348D0100008D0100D8
:109CC000648D0100002B4DD02DE9F0415D1EEDB2F9
:109CD000044601EB45058F1EA2F10208002619E09B
:109CE000FFF7E0FEB4F8883701339BB2B3F5707F1D
:109CF00038BFA4F88837B4F8863728BFA4F8886737
:109D000001339BB2042B94BFA4F88637A4F886676E
:109D1000BD4225D038F802EFD4F8E407B4F8E837AC
:109D2000B4F8862737F9021F224470440133C4F87F
:109D3000E407A4F8E83753785B00DBB20029B8BF2A
:109D400043F001035370B4F88827237804EB4202F0
:109D5000013B012BD1802046C2D9FFF7C7FDC1E7E7
:109D6000BDE8F081704700BF70B5044600264FF48F
:109D70007A602681667366812080267308F050F928
:109D800004F11C056060266131466661A6612B46C0
:109D900004F13C0223F8021B9342FBD104F2EC4095
:109DA000002203F8012B98424FF00001F9D14FF443
:109DB0009653F022A4F8EC14A4F8EE14C4F8F814A6
:109DC000A4F8F024C4F8F434202228460AF09EF9BE
:109DD00005210922034B2174A5616282636120463B
:109DE00070BD00BFF80DFF1F312AF0B402D004206F
:109DF000F0BC70474289038992B29BB29A4217D055
:109E00004289038992B29BB29A420BD2048902889A
:109E1000438912FA83F31B1B9BB29A420CD2052092
:109E2000F0BC70474389048902881B1B9BB2F4E78E
:109E3000037B002BF3D103882F2BF0D94B1C01257A
:109E4000313103E04573013399421CD0027B02F0AB
:109E5000FF06002AF6D1446802891F7892B2A754FF
:109E60000289013292B2028104890288A4B292B2BC
:109E7000944228BF068104894289A4B292B29442D6
:109E800008BF0573DFE70020B2E700BFF0B58FB071
:109E900002AC04AA4FF4F77E40F2C9574FF63726BA
:109EA0004FF6126501F0C003802B1CD0C02B18D0D8
:109EB000ABB12680023489009442C9B2F2D102A922
:109EC00022461030042308F0B9FA002300932246FA
:109ED000142307210548FEF799FB0FB0F0BD25803C
:109EE000E8E72780E6E7A4F800E0E3E758A5FF1FCE
:109EF00010B58EB0002402A904AA103004230394E4
:109F0000029408F09BFA009404AA14230721024843
:109F1000FEF77CFB0EB010BD58A5FF1FB0F8EC3467
:109F200070B504464BB35348FEF730FC1428054681
:109F300040F29A80B4F8EE344F4E01E0142D43D92C
:109F40005A1C2344A4F8EE2493F83C102046FFF753
:109F50009DFF3378143DADB21BB1D4F8F434C4F88E
:109F6000F834B4F8EE34B4F8EC249A42E6D800237E
:109F7000A4F8EE34A4F8EC3470BD4189028989B2AA
:109F800092B2914244D04189028989B292B29142FF
:109F90001BD202894189521A92B2FAB1374A127819
:109FA000002A3AD1B4F8F01400295ED07720E218E4
:109FB00001339BB2994282F83C00F8D1A4F8EC142A
:109FC0000023A4F8EE34AEE770BD408922882189D1
:109FD00012FA81F2121A92B2002ADFD1D4F8F834C0
:109FE000002BF1D02348FEF7D1FB1428054602D8F8
:109FF0003EE0142DE8D92046FFF77AFFD4F8F83474
:10A00000143D013BADB2C4F8F834002BF1D170BD62
:10A01000027B002AE2D00288BFE7002018E06168D6
:10A02000628992B28D5C20736289013292B2628140
:10A030006189228889B292B2914200D360815A1C10
:10A04000E11893B2302BA4F8EC3481F83C50B7D02F
:10A050002189628989B292B29142E0D1227B02F0D9
:10A06000FF05002ADBD1EAE770BDA4F8EE14B5E7DE
:10A0700070BD00BF58A5FF1F540EFF1F50A5FF1F46
:10A0800001EB4101890001F5167189B2B1F5966FB6
:10A090008ABF4FF49663A0F8F014A0F8F03470472C
:10A0A0004289038992B29BB29A421DD042890389A8
:10A0B00092B29BB29A4208D34389018902885B1A03
:10A0C0009BB293420AD900207047018902884389D4
:10A0D00012FA83F35B1A9BB29342F4D80748A0FBB1
:10A0E0000330C0F347107047037B002BEBD103888C
:10A0F0000248A0FB0330C0F347107047ABAAAAAADE
:10A100004FF4966303FB01F1C0F8F414704700BFED
:10A11000014803F06FB800BFF04CFF1F10B55C485A
:10A120005C4C04F023FB5C48FEF7DEFB5B4B1B78CA
:10A13000002B61D02378012B5BD0594A12780AB1E9
:10A14000022B7DD0574A127812B1032B00F08C807D
:10A15000554A12780AB1042B7CD0544A12780AB1BD
:10A16000052B7CD0524A127812B1072B00F0818067
:10A17000504A127852B1062B04D04F4801F02EFFFE
:10A18000002865D04C4801F0DBFF23784B4A127859
:10A1900022B3FBB10A2B1DD0632B6FD0A3F15C025D
:10A1A000D2B2062A08D84D2121FA02F2D20703D5ED
:10A1B0004348F7F7B1F92378A3F16602052A22D9BB
:10A1C0005D2B26D05B2B2AD06C2B2ED0652B32D06A
:10A1D000A3B110BD3B48F6F70BFF23783A4A12783B
:10A1E000002AD9D00A2BD7D13848FDF705FA2378B1
:10A1F000D2E73748FBF7B2F923789EE73548BDE848
:10A200001040F6F787BF3448F7F760FC23785D2BE2
:10A21000D8D13248F7F75EFD23785B2BD4D1304894
:10A22000F7F718FD23786C2BD0D12E48F7F7E6FC12
:10A230002378652BCCD12C48F7F78EFD2378C7E720
:10A240002A4B1B78FBB12A48F9F750FF237879E7AE
:10A2500023789BE7274801F0D7FD23787DE7264840
:10A2600000F096FD23787DE7244805F0B5FA2378C1
:10A270006EE72348FFF752FE237879E72148F7F786
:10A280005DFA23788AE72048F8F7D4FA237859E76B
:10A29000F04CFF1FAC78FF1F58A5FF1F580EFF1F83
:10A2A000570EFF1F560EFF1F5A0EFF1F550EFF1FA2
:10A2B000520EFF1F5B0EFF1F6471FF1F590EFF1F21
:10A2C000ECF4FF1F6420FF1F530EFF1FE8D2FF1F97
:10A2D000C01DFF1FD019FF1F7084FF1F6CE5FF1FFB
:10A2E00054A5FF1FCC19FF1F6C84FF1F540EFF1FC6
:10A2F000B078FF1F9C79FF1FB42AFF1F70E0FF1F7B
:10A30000B073FF1FA4FEFF1FA8FEFF1F08B52F4854
:10A31000F9F76AFF2E48FAF781FE2E48F7F742F95F
:10A320002D48F7F707FA2D48F8F768FB2C48F8F79F
:10A3300053FD2C48F9F77CFA2B48F7F785FD2B489D
:10A34000F8F7BAF92A48F6F7CDFF2A4804F03AFDA3
:10A35000294805F043F9294800F024FE284801F077
:10A36000E3FB2848F7F7B2FC274800F06DF82748D0
:10A3700000F00EFC2648F7F767FC2648FFF778F850
:10A380002548FFF7F1FC2548F7F734FC244801F095
:10A39000EFFD2448F7F7DCFC2348FBF703FA2348DA
:10A3A000F7F788FB2248F6F771FB2248F6F7CEFC58
:10A3B0002148F7F7F3FC2148F6F798FE204802F011
:10A3C00053F92048BDE80840FDF7F0BF8084FF1F27
:10A3D000C01DFF1FE8BBFF1FA4FEFF1F1C7FFF1F48
:10A3E0004830FF1FB078FF1F28BCFF1FA8FEFF1FCB
:10A3F000ECF4FF1FA8A8FF1F70E0FF1F204FFF1FF6
:10A400009C79FF1F6CE5FF1F70E5FF1FB42AFF1F3B
:10A4100054A5FF1FC822FF1FB073FF1FCC19FF1FD9
:10A420006471FF1F6C84FF1FE8D2FF1F7084FF1F41
:10A4300018F5FF1F6420FF1FA473FF1FD019FF1F13
:10A44000F04CFF1F58A5FF1F0346002203F8022B04
:10A4500000F1160123F8022B8B42FBD130B400F639
:10A460001675002423F8024BAB424FF00002F9D1DD
:10A4700042F20F73A0F81A3FA0F81C3FA0F81E3F4D
:10A48000A0F8203FA0F8223FA0F8162FA0F8182F20
:10A49000C0F8242FA0F8282F80F82A2F00F62C735C
:10A4A00000F64C7423F8022BA3424FF00001F9D1BF
:10A4B000A0F84C1F00F64E7300F66E7423F8021BD2
:10A4C0009C424FF00002F9D16323A0F86E2FC0F830
:10A4D000742FA0F8782F80F8703F30BC704700BF11
:10A4E000002342F20F72632180F8701F0370A0F8FE
:10A4F000183FA0F8163FC0F8243FA0F84C3FA0F842
:10A500006E3FA0F8283F80F82A3FC0F8743FA0F8BB
:10A51000783FA0F81A2FA0F81C2FA0F81E2FA0F843
:10A52000202FA0F8222F7047F0B5044683B0002AF0
:10A530007BD0404F4FF47A5E3E467546002015E0D2
:10A540009E42B8BF1E469D42A8BF1D4601F10A03A8
:10A550009BB2B3F5F06F00F10100A1F2767138BF44
:10A56000194683B228BF89B29A420CD904EB410341
:10A57000B3F91630002BE3DC9E45A8BF9E469F42F0
:10A58000B8BF1F46E2E772190EEB070352105B10CB
:10A59000D6187610951B1BB22DB236B212B20195A9
:10A5A00000962549254804F039FB94F8703F632B49
:10A5B00029D004EB43020133DBB20F2BA2F82C6F3E
:10A5C000A2F84E5F04F62A7184F8703F04F64C70CE
:10A5D00004F64A7725D800221346A4F84C2FA4F895
:10A5E0006E2F31F8026F30F8025F32442B44B942CB
:10A5F00012B21BB2F5D112111B11A4F84C2FA4F802
:10A600006E3F03B0F0BD04F62A7104F64C700B46A1
:10A61000024604F64A7723F8026FBB4222F8025F33
:10A62000F9D1002384F8703FD5E715461646134646
:10A63000B5E700BF80C1FFFFA88D0100F04CFF1FF0
:10A640002DE9F04FBDF82450BDF928C0BDF92C808C
:10A65000002A7AD0AE1C0135DFF8F4E01FFA8CFC3A
:10A66000B6B2ADB2C8F1000900272AE04FEAE40A09
:10A6700004F0070413F80AB01EF804402BEA04049F
:10A6800003F80A4005F0070BEC101EF80BB013F8A6
:10A6900004A04BEA0A0A03F804A001F10A04A4B2D8
:10A6A000B4F5F06F07F1010728BFA1F27671BFB2D0
:10A6B0002CBF89B2214602360235BA42B6B2ADB2DB
:10A6C00043D000EB410AB41EBAF816A0CCEB0A0A3C
:10A6D0000FFA8AFACA45A4B2C8DBBAF1000F1CDB34
:10A6E000C2454FEAE40A04F0070413F80AB01EF862
:10A6F000044044EA0B0403F80A4005F0070B4FEA54
:10A70000E5041EF80BB013F804A0B4BF2AEA0B0A44
:10A710004BEA0A0A03F804A0BFE74FEAE40A04F090
:10A72000070413F80AB01EF804402BEA040403F8E7
:10A730000A4005F0070BEC101EF80BB013F804A04C
:10A740002AEA0B0A03F804A0A7E7BDE8F08F00BFD0
:10A75000188E0100B0F8163F00EB43032DE9F04FCF
:10A7600005465888C0F3090080F4A67089B080F0CF
:10A77000010004F0DFFA022840D8B5F818CF554997
:10A78000554F0CF22676B6B2B6F5F06F26BFACF197
:10A790005A031FFA83F8B04601F1090E6FF0020365
:10A7A00000244FF47A5005EB4802B2F91620974284
:10A7B000B8BF17469042A8BF1046012B19D0032BF3
:10A7C00013D0013301D002EB4202144408F10A0312
:10A7D0009BB2B3F5F06F24BFA8F276739BB28E459F
:10A7E00010D0984611F9013FDDE702EB4202A41AAE
:10A7F000ECE7A41AEAE7059B9B453FD9002009B086
:10A80000BDE8F08FD5F8243FA342F7DA95F8703F02
:10A81000632B50D0B5F94C3FB5F96E2F0292B6F5C7
:10A82000F06F24BFACF15A06B6B200270DF11C0A36
:10A83000019331465346284600970A22FFF700FF4E
:10A840002B78DFF89890DFF89880BB4214BF032381
:10A850000123BB460593CD20FF211AF807200A40AB
:10A86000504004F061FA01375844032F5FFA80FB2F
:10A87000C1D019F8011F18F8010FEEE7B5F8183F1D
:10A88000A5F81E3F03F21B7292B2B2F5F06F4FF0C3
:10A89000060128BF653B4FF00100C5F8244FA5F81D
:10A8A0001A6FA5F8281F34BFA5F81C2FA5F81C3F68
:10A8B00009B0BDE8F08FC3195B10FF1A44F63E12D1
:10A8C00002FB07F71BB247F3CF32A5F84C3FA5F8C0
:10A8D0006E2FA3E7948D010080C1FFFFA08D0100C2
:10A8E000A48D010010B50446FFF734FF94F82A3F09
:10A8F00028B33BB3013BDBB2012B84F82A3F20D1C4
:10A90000B4F81E3F03F27F7292B2B2F5F06F28BF27
:10A9100003F1FF32A4F8202F5A1C92B2B2F5F06F67
:10A9200024BFA3F27F73A4F8223F4FF0000338BF87
:10A93000A4F8222F84F82A3F0122227010BD002B98
:10A94000D8D110BDC4F8743FA4F8783F012107485E
:10A95000FDF744FF01210548FDF74CFF6322042366
:10A9600084F8702F84F82A3F10BD00BF58A5FF1F40
:10A97000B0F8783F10B504464BB931220E4803F0C9
:10A98000EBFC0023C4F8743FA4F8783F10BDD4F862
:10A99000742FB2FBF3F3C3F3072281F8323081F84E
:10A9A00031200548332203F0D7FC0023C4F8743F5C
:10A9B000A4F8783F10BD00BFF04CFF1F30B5B0F8D1
:10A9C000202FB0F8221FB0F8183F8A4293B00446F7
:10A9D00007D29A4207D9B4F81C2F9A420ED013B06E
:10A9E00030BD9A4201D99942F5D32046FFF7B2FE15
:10A9F000B4F8183FB4F81C2F9A42F0D1B4F8283FAD
:10AA0000062B53D0C022B4F81A1F2046FFF78CFD46
:10AA1000B4F96E1FB4F94C3FB4F91E2F2F480091C2
:10AA20002F4904F08FF8B4F96E3FB4F94C0FB4F825
:10AA30001A1F029308220190009205ABC022204603
:10AA4000FFF7FEFDB4F8285F013DADB2A4F8285F22
:10AA50007DB1A5F10505B5FA85F56D0905A9204675
:10AA60008DF81450FFF784FF0023C4F8243F13B07F
:10AA700030BD1C49194804F005F829461A48FDF76D
:10AA8000ADFE29461848FDF7B5FE144803F098FCC2
:10AA900042F20F726323257084F82A5FC4F8245FA2
:10AAA000A4F81C2F84F8703F13B030BDB4F81E3FDB
:10AAB00003F27F7292B2B2F5F06F28BF03F1FF325A
:10AAC000A4F8202F5A1C92B2B2F5F06F2ABFA3F25D
:10AAD0007F73A4F8222FA4F8223F93E7F04CFF1FC6
:10AAE000CC8D0100F48D010058A5FF1F002B4DD027
:10AAF0002DE9F0415D1EEDB2044601EB45058F1EC8
:10AB0000A2F10208002619E0FFF758FFB4F8183F39
:10AB100001339BB2B3F5F06F38BFA4F8183FB4F817
:10AB2000163F28BFA4F8186F01339BB2092B94BFBE
:10AB3000A4F8163FA4F8166FBD4225D038F802EFEE
:10AB4000D4F8740FB4F8783FB4F8162F37F9021F11
:10AB500004EB420270440133C4F8740FA4F8783F48
:10AB600053885B009BB20029B8BF43F001035380B8
:10AB7000B4F8183F227804EB4303012AD982204617
:10AB8000C2D0FFF7AFFEC1E7BDE8F081704700BF5C
:10AB9000F8B5054600244FF47A602C816C736C8103
:10ABA00028802C7307F03CFA05F1280768602C61B7
:10ABB00022466C61AC613B4605F1480623F8022B46
:10ABC000B342FBD105F1D4013346002223F8022B16
:10ABD0008B42FBD105F28451002203F8012B8B42FA
:10ABE0004FF00004F9D140F6B833F022C5F88C35A7
:10ABF000A5F88445A5F88645C5F89045A5F88825AB
:10AC000021462022384609F081FA21468C2230461E
:10AC10000A2409F07BFA09200549064B2C741622F8
:10AC20006882AF612E626961AA836B622846F8BDB3
:10AC3000880EFF1F5C0EFF1F312AF0B402D00420E3
:10AC4000F0BC70474289038992B29BB29A4217D0F6
:10AC50004289038992B29BB29A420BD2048902883C
:10AC6000438912FA83F31B1B9BB29A420CD2052034
:10AC7000F0BC70474389048902881B1B9BB2F4E730
:10AC8000037B002BF3D103882F2BF0D94B1C01251C
:10AC9000313103E04573013399421CD0027B02F04D
:10ACA000FF06002AF6D1446802891F7892B2A754A1
:10ACB0000289013292B2028104890288A4B292B25E
:10ACC000944228BF068104894289A4B292B2944278
:10ACD00008BF0573DFE70020B2E700BFF0B5ADB0F5
:10ACE000054602AC04AA4FF0F50E40F2DF274FF6FE
:10ACF00021564FF60B7001F0C003802B24D0C02BDF
:10AD000020D0EBB12680023489009442C9B2F2D13E
:10AD100002A9224605F11000042307F08FFB21460B
:10AD200005F11C0018AA282308F072F800230093EC
:10AD300018AA282305210648FDF768FC2DB0F0BDB0
:10AD40002080E0E72780DEE7A4F800E0DBE700BF33
:10AD500058A5FF1F30B5ADB00024054602A904AACE
:10AD6000103004230394029407F068FB04A905F152
:10AD70001C0018AA282308F04BF8009418AA2823CE
:10AD800005210248FDF742FC2DB030BD58A5FF1F3C
:10AD9000F8B5B0F8843504464BB35B48FDF7F6FCD4
:10ADA0002828054640F2AE80B4F88635574E01E0BB
:10ADB000282D6ED95A1C2344A4F8862593F8D41064
:10ADC0002046FFF78BFF3378283DADB21BB1D4F896
:10ADD0008C35C4F89035B4F88635B4F884259A4299
:10ADE000E6D80023A4F88635A4F88435F8BD418957
:10ADF000028989B292B2914254D04189028989B2C2
:10AE000092B2914246D202894189521A92B23AB321
:10AE10003F4A1278002A4AD1B4F888253AB15F2017
:10AE2000E11801339BB29A4281F8D400F8D1A018FE
:10AE3000511C931C14FA81F1033214FA83F357273F
:10AE400080F8D470752692B2FD25002081F8D46078
:10AE5000A4F8842583F8D450A4F88605002A9CD150
:10AE6000D4F89035ABB12848FDF790FC282805466A
:10AE700002D848E0282D0CD92046FFF76BFFD4F804
:10AE80009035283D013BADB2C4F89035002BF1D18F
:10AE9000F8BDF8BD40892288218912FA81F2121A80
:10AEA00092B2B4E7027B002ADAD00288AFE7002032
:10AEB00018E06168628992B28D5C20736289013208
:10AEC00092B262816189228889B292B2914200D3A2
:10AED00060815A1CE11893B2302BA4F8843581F8B4
:10AEE000D4500BD02189628989B292B29142E0D1CB
:10AEF000227B02F0FF05002ADBD1EAE70023A4F859
:10AF000086354AE7F8BDF8BD58A5FF1F540EFF1F50
:10AF100050A5FF1F01EB4101490001F5967189B26F
:10AF2000B1F5966F8ABF4FF49663A0F88815A0F824
:10AF3000883570474289038992B29BB29A421DD0EC
:10AF40004289038992B29BB29A4208D3438901890C
:10AF500002885B1A9BB293420AD90020704701898C
:10AF60000288438912FA83F35B1A9BB29342F4D8A6
:10AF70000748A0FB0330C0F347107047037B002B4A
:10AF8000EBD103880248A0FB0330C0F347107047A1
:10AF9000ABAAAAAA4FF4167303FB01F1C0F88C15F3
:10AFA000704700BF03460022F0B403F8042B0546A7
:10AFB00000F1180143F8042B8B42FBD105F5075132
:10AFC0001831002423F8024B8B424FF00002F9D1D4
:10AFD00042F2D81642F2DA1342F2DC1442F2DE11E7
:10AFE000AA53EA5242F20F732B5342F2E0176B520C
:10AFF00042F2E21642F2E41442F2E611EB53AB5392
:10B0000042F2E8172B5342F2EC166B5242F2F01464
:10B0100042F2F211EB5305F50850AA5105F507531A
:10B020002A536A543433143023F8022B83424FF0EE
:10B030000001F9D142F2142205F508531846A9522D
:10B040001633363023F8021B98424FF00002F9D134
:10B0500042F2362742F2382642F23C2005F50951E9
:10B0600042F24223EA536327AF552A500A80EA543A
:10B070002846F0BC704700BFF0B542F2DA1742F242
:10B08000D81642F2EC15002342F23822C35342F2A2
:10B09000DC14037042F2DE1183534351632585545F
:10B0A00042F20F72025342F2E017425242F2E616A7
:10B0B00042F2E81542F2E21442F2E411C25342F2C3
:10B0C000142E825342F23627425342F2F0160253B4
:10B0D00042F2F215425242F23C2400F5095142F28A
:10B0E000422220F80E30C3538353435503510B8043
:10B0F0008354F0BDF0B5044683B0002A00F08C8084
:10B10000474F4FF47A5E3E467546002016E09E4259
:10B11000B8BF1E469D42A8BF1D464B1D9BB2B3F54E
:10B12000875FA1F5865100F10100A1F11B0138BF35
:10B13000194683B228BF89B29A420CD901F10C0397
:10B1400034F91330002BE2DC9E45A8BF9E469F4297
:10B15000B8BF1F46E1E772190EEB070352105B10F0
:10B16000D6187610951B1BB22DB236B212B20195CD
:10B1700000962C492C4803F051FD42F23822A35C82
:10B18000632B33D004EB430142F2F41742F2162052
:10B190000133CE53DBB20D5204F50850074604F5D7
:10B1A00007510F2BA35401F1320100F1140007F1F4
:10B1B00012072CD842F2362242F2142500236353A0
:10B1C000A3521A4631F8026F30F8025F32442B4422
:10B1D000B94212B21BB2F5D142F2142042F236212A
:10B1E00012111B112252635203B0F0BD04F5075136
:10B1F00004F508503231143004F508570B46024666
:10B20000123723F8026FBB4222F8025FF9D142F2F3
:10B2100038230022E254CDE7154616461346A6E72A
:10B2200080C1FFFF408E0100F04CFF1F2DE9F04F61
:10B23000BDF82450BDF928C0BDF92C80002A7BD070
:10B24000AE1C0135DFF8F4E01FFA8CFCB6B2ADB2EB
:10B25000C8F1000900272BE04FEAE40A04F00704D4
:10B2600013F80AB01EF804402BEA040403F80A405D
:10B2700005F0070BEC101EF80BB013F804A04BEA16
:10B280000A0A03F804A04C1DA4B2B4F5875F28BFD6
:10B29000A1F5865107F1010728BF1B39BFB22CBFAA
:10B2A00089B2214602360235BA42B6B2ADB243D0B7
:10B2B00001F10C0AB41E30F81AA0CCEB0A0A0FFAFE
:10B2C0008AFACA45A4B2C7DBBAF1000F1CDBC2453B
:10B2D0004FEAE40A04F0070413F80AB01EF8044029
:10B2E00044EA0B0403F80A4005F0070B4FEAE504B3
:10B2F0001EF80BB013F804A0B4BF2AEA0B0A4BEAFD
:10B300000A0A03F804A0BEE74FEAE40A04F00704BF
:10B3100013F80AB01EF804402BEA040403F80A40AC
:10B3200005F0070BEC101EF80BB013F804A02AEA86
:10B330000B0A03F804A0A6E7BDE8F08FA48F010074
:10B340002DE9F04F42F2D81305467548EB5A05EB4C
:10B35000830387B05B6823F07F43584003F0EAFC27
:10B3600002287CD842F2DA136E4935F803C06E4FDA
:10B370000CF583560D36B6B2B6F5875F26BFACF135
:10B3800073031FFA83F8B04601F1170E032300245C
:10B390004FF47A5008F10C0235F912209742B8BFE9
:10B3A00017469042A8BF1046012B1AD0032B14D089
:10B3B000013301D002EB4202144408F1050293B2BA
:10B3C000B3F5875F03D3A8F586531B3B9BB28E452D
:10B3D00009D0984611F9013FDCE702EB4202A41ABA
:10B3E000EBE7A41AE9E742F2EC13EB58A34236DA92
:10B3F00042F23823EB5C632B70D042F2142342F20A
:10B400003622EB5EAA5E0292B6F5875F24BFACF1EE
:10B410007306B6B200270193284604AB00971822A2
:10B420003146FFF703FF2B78DFF80081BB420DF1B7
:10B43000100B14BF4FF0040A4FF0020A08F105097F
:10B44000552001E018F8010F1BF8013B584003F0AC
:10B450006BFCC8453844C7B2F4D1574503D9002026
:10B4600007B0BDE8F08F42F2DA1342F2E812EB5A6D
:10B47000AB5203F58352073242F2EC1742F2F0105E
:10B4800042F2DE1192B2EC51B2F5875F4FF0050443
:10B490002C526E5233D242F2E0116A522A78CAB963
:10B4A00003F2BB7242F2E61042F2DC1192B2B2F544
:10B4B000875F2B526E5228D242F2E2116A5203F297
:10B4C000BD7292B2B2F5875F25D342F2E412A3F6C1
:10B4D0002313AB52012007B0BDE8F08FC3195B10F6
:10B4E000FF1A44F63E1202FB07F742F2362042F200
:10B4F00014211BB247F3CF322A526B5283E742F238
:10B50000E012A3F17901A952C8E742F2E212A3F6D0
:10B510002511A952D3E742F2E413EA52DAE700BF59
:10B52000A030FB00208E010080C1FFFF388E01009B
:10B5300038B50446FFF704FF38B342F2F215635DF5
:10B54000002B39D0013BDBB242F2F212012BA354A3
:10B5500020D142F2E613E35A03F2BB7292B2B2F583
:10B56000875F18D242F2E211625203F2BD7292B2C8
:10B57000B2F5875F1AD242F2E413E25242F2F212BB
:10B580000021A1540123237038BD42F2F213E35C81
:10B59000002BD7D138BD42F2E212A3F62511A152F9
:10B5A00003F2BD7292B2B2F5875FE4D342F2E412C5
:10B5B000A3F62313A352E1E704F5095242F23C211A
:10B5C0000848635013800121FDF708F9012105485F
:10B5D000FDF710F942F2382263210923A154635583
:10B5E00038BD00BF58A5FF1F42F2DC13F0B5C35AA7
:10B5F00003F1780189B2B1F5875F9FB0044603D3A8
:10B60000A3F58351083989B242F2362342F214225B
:10B61000E35EA25E0293002301920093082204AB32
:10B620002046FFF703FE9DF8113042F2422203F05C
:10B630000F03A3540F2B3AD8DFE813F09000390022
:10B640003900BC00390039003900100039003900D8
:10B6500039003900E60039003900660042F2DC1793
:10B66000B422E15B204642F23626FFF743FD42F268
:10B67000142542F2E612A15F635FA25E6E4800915C
:10B680006E4903F05FFAE15BA25F635F02920822FA
:10B690000193009205ABB4222046FFF7C7FD0123BA
:10B6A00005A92E2264488DF8143002F0D1FD42F233
:10B6B000E813E25A02F586531F339BB2B3F5875F56
:10B6C00012D242F2E2116352531C9BB2B3F5875F70
:10B6D00013D242F2E412A35242F2EC130022E250DF
:10B6E000022323701FB0F0BD42F2E213511EE1525B
:10B6F000531C9BB2B3F5875FEBD3A2F5865242F29F
:10B70000E4131F3AE252E7E742F2DC172046E15B1E
:10B7100042F23626D822FFF7EDFC42F2142542F21F
:10B72000E612A15F635FA25E43480091444903F0C3
:10B7300009FAA25FE15B635F029208220193009223
:10B7400005AB2046D822FFF771FD012305A937225A
:10B7500039488DF8143002F07BFDA8E742F2DC177F
:10B760002046E15B42F236264FF4C672FFF7C2FC78
:10B7700042F2142542F2E612A15F635FA25E2E48F8
:10B780000091304903F0DEF9A25FE15B635F029252
:10B7900008220193009205AB20464FF4C672FFF7D2
:10B7A00045FD012305A9642223488DF8143002F0D9
:10B7B0004FFD7CE742F2DC172046E15B42F2362681
:10B7C0004822FFF797FC42F2142542F2E612A15FED
:10B7D000635FA25E184800911B4903F0B3F9A25FB2
:10B7E000E15B635F029208220193009205AB204661
:10B7F0004822FFF71BFD012305A913220E488DF8EF
:10B80000143002F025FD52E742F2E61542F23627E7
:10B8100042F21426615BB4222046FFF76BFCE15F25
:10B82000625FA35F04480091084903F08BF9615BF4
:10B83000E25FA35F2AE700BFF04CFF1FC08E01004C
:10B84000208F0100608E0100F08E0100908E0100BB
:10B8500042F2E21242F2E413815AC25A42F2DA137D
:10B86000914210B5C35A044604D299420FD89A4265
:10B8700004D210BD994201D99A420FD32046FFF756
:10B880005FFD42F2DA1342F2E412E35AA25A9A42FC
:10B89000EFD12046BDE81040FFF7A6BE10BD00BFA7
:10B8A00070B500F5095504462B884BB9D9220C48D0
:10B8B00002F000FD42F23C220023A3502B8070BD19
:10B8C00042F23C20DB222058B0FBF3F3C3F3072005
:10B8D00081F8D90081F8DA30014802F0EBFCE9E7A1
:10B8E000F04CFF1FF0B542F2E41342F2E212C15AEB
:10B8F000825A42F2DA138A42BDB00446C35A08D2D1
:10B900009A4208D942F2E012A25A9A4210D03DB0AF
:10B91000F0BD9A4201D99942F4D32046FFF710FDB9
:10B9200042F2DA1342F2E012E35AA25A9A42EED1FC
:10B9300042F2F013E35A052B5ED042F2DE174FF4C9
:10B940005872E15B204642F23626FFF7D3FB42F203
:10B95000142542F2E812A15F635FA25E37480091AE
:10B96000374903F0EFF8A25F635FE15B02920822C0
:10B970000193009205AB4FF458722046FFF756FC36
:10B9800042F2F013E55A013DADB2E55285B1A5F1A1
:10B990000405B5FA85F56D0905A920468DF8145002
:10B9A000FFF77EFF42F2EC130022E2503DB0F0BD03
:10B9B0002449224803F066F829462348FCF70EFF85
:10B9C00029462148FCF716FF1C4802F0A5FC42F26C
:10B9D000E01642F2382042F2F21142F2EC1242F248
:10B9E000422342F20F772570A753632626546554ED
:10B9F000A550E5543DB0F0BD42F2E813E25A02F51D
:10BA000086531F339BB2B3F5875F0BD242F2E2112C
:10BA10006352531C9BB2B3F5875F08D242F2E41223
:10BA2000A3528AE742F2E213511EE152F1E7A2F576
:10BA3000865242F2E4131F3AE2527EE7F04CFF1FB7
:10BA4000508F0100808F010058A5FF1F002B6AD086
:10BA50002DE9F04F03F1FF3983B05FFA89F300F568
:10BA6000075700F5085901EB4303044600F5095058
:10BA70003E460093831C8D1EA2F1020809F13C0989
:10BA800018371A36019383464FF0000A19E0204612
:10BA9000FFF728FF3188013189B2B1F5875F23BFF5
:10BAA000019BA6F800A083F800A031803988009B94
:10BAB000013189B2042994BF3980A7F800A0AB42B4
:10BAC0002ED0D9F8001038F802CFBBF800E0388843
:10BAD00001EB0C0304EB80000EF1010E35F9021F9F
:10BAE000C9F80030ABF800E0436800294FEA43038F
:10BAF000B8BF43F001034360308894F800E00C3095
:10BB0000BEF1010F24F8101006D0BEF1020FBED016
:10BB10002046FFF70DFDBDE72046FFF799FEB9E788
:10BB200003B0BDE8F08F70472DE9F04105460024D1
:10BB30004FF47A602C816C736C8128802C7306F032
:10BB40006FFA05F1280768602C6122466C61AC61D0
:10BB50003B4605F1480623F8022BB342FBD105F121
:10BB6000C0013346002223F8022B8B42FBD105F59E
:10BB7000AE61002203F8012B8B424FF00004F9D193
:10BB800041F270734FF02008F022C5F87835A5F81F
:10BB9000742521464246A5F87045A5F87245C5F8BA
:10BBA0007C45384608F0B2FA21467822304608F043
:10BBB000ADFA05200821064A064B2874A5F81C801A
:10BBC000AF612E6269826A616B622846BDE8F081CE
:10BBD0007C0FFF1F3C0FFF1F122A01D80420704763
:10BBE000F0B544890389A4B29BB29C4216D0448923
:10BBF0000389A4B29BB29C4208D343890589048877
:10BC00005B1B9BB2A3420DD90520F0BD05890488BA
:10BC1000438914FA83F35B1B9BB2F3E7037B002B8E
:10BC2000F2D103889A42EFD8037B03F0FF05002B83
:10BC30002FD00123013A43734AB300252B46012636
:10BC400005E046730133DBB293421D461FD2047BED
:10BC500004F0FF07002CF4D1D0F804E004890D446F
:10BC6000A4B26D780EF8045004890134A4B20481A2
:10BC700005890488ADB2A4B2A54228BF0781058911
:10BC80004489ADB2A4B2A54208BF0673DAE700202A
:10BC9000F0BD446803899BB2013AE2540389013341
:10BCA0009BB2038104890388A4B29BB29C4228BF43
:10BCB000058104894389A4B29BB29C42BCD1012373
:10BCC0000373B9E7F0B599B0054602AC04AA4FF486
:10BCD000D27E40F2EC474FF614364FF65C6001F02E
:10BCE000C003802B24D0C02B20D0EBB1268002349F
:10BCF00089009442C9B2F2D102A9224605F110008E
:10BD0000042306F09BFB214605F11C000EAA142318
:10BD100007F07EF8002300930EAA1423042106489E
:10BD2000FCF774FC19B0F0BD2080E0E72780DEE767
:10BD3000A4F800E0DBE700BF58A5FF1F30B599B0BD
:10BD40000024054602A904AA103004230394029497
:10BD500006F074FB04A905F11C000EAA142307F0D9
:10BD600057F800940EAA142304210248FCF74EFC55
:10BD700019B030BD58A5FF1F01EB4101890001F545
:10BD8000167189B2B1F5966F8ABF4FF49663A0F829
:10BD90007415A0F8743570474289038992B29BB23A
:10BDA0009A421DD04289038992B29BB29A4208D32B
:10BDB0004389018902885B1A9BB293420AD9002009
:10BDC000704701890288438912FA83F35B1A9BB298
:10BDD0009342F4D80748DB08A0FB0330C0B2704799
:10BDE000037B002BEBD103880248DB08A0FB033068
:10BDF000C0B270475F427B094FF4966303FB01F1C9
:10BE0000C0F87815704700BF70B5B0F8703582B0D3
:10BE100004464BB35348FCF7B9FC1428054621D916
:10BE2000B4F87235504E01E0142D1BD95A1C23442E
:10BE3000A4F8722593F8C0102046FFF743FF33782B
:10BE4000143DADB21BB1D4F87835C4F87C35B4F8E4
:10BE50007235B4F870259A42E6D80023A4F87235FA
:10BE6000A4F8703502B070BD4189028989B292B2DE
:10BE7000914244D04189028989B292B291421AD248
:10BE800002894189521A92B2F2B1384A1278002AD4
:10BE90003AD1B4F8741500295ED07720E218013346
:10BEA0009BB28B4282F8C000F8D10022A4F8703512
:10BEB000A4F87225AEE740892288218912FA81F21E
:10BEC000121A92B2002AE0D1D4F87C35002BC9D0E6
:10BED0002448FCF75BFC1428054602D8C2E7142D61
:10BEE000C0D92046FFF72AFFD4F87C35143D013B2A
:10BEF000ADB2C4F87C35002BF1D102B070BD027B2D
:10BF0000002AE1D00288BFE70DF106012046F9F7CB
:10BF1000FBFA9DF8063013B300252E460DF10701FC
:10BF200020468DF80760F9F7EFFAB4F870359DF800
:10BF300006109DF8070001355A1CEDB2234492B259
:10BF4000A942A4F8702583F8C000E7D80023A4F81C
:10BF50007235002AB8D05DE7A4F87215B4E7B4F8DA
:10BF60007025F3E758A5FF1F540EFF1F50A5FF1FB4
:10BF700070B5054600244FF47A602C816C736C8197
:10BF800028802C7306F04CF805F11C0668602246E8
:10BF9000334605F5B87123F8022B8B42FBD105F52A
:10BFA0000E70002203F8012B98424FF00001F9D1E6
:10BFB0004823A5F83C32A5F83812A5F83A124FF4F8
:10BFC000AA72304608F0A2F80622034B6E612A825C
:10BFD000AB61284670BD00BFCC0FFF1FB0F8382200
:10BFE0000346B2B94189028989B292B291421AD00C
:10BFF0004189028989B292B291420CD340891A8850
:10C000001B8912FA83F3181A80B2003018BF01207E
:10C0100070470120704702894089101A80B20030B1
:10C0200018BF01207047027B02F0FF00002AF1D008
:10C030001888EAE7442AF0B402D00420F0BC704724
:10C040004289038992B29BB29A4217D042890389EE
:10C0500092B29BB29A420BD204890288438912FAA7
:10C0600083F31B1B9BB293420CD90520F0BC704795
:10C070004389048902881B1B9BB2F4E7037B002BD6
:10C08000F3D10388432BF0D901F14404012503E0E7
:10C09000457301318C421CD0037B03F0FF06002B5B
:10C0A000F6D1426803890F789BB2D75403890133D4
:10C0B0009BB203810289038892B29BB29A4228BF45
:10C0C00006810289438992B29BB29A4208BF0573E6
:10C0D000DFE70020B2E700BF70B50646ADF5227D70
:10C0E0000C46002502AB14F0800F4FF028021149D6
:10C0F00003EB050003D102AB0F492822581928355C
:10C1000003F066FC6400B5F5A07FE4B2EAD102A9B1
:10C1100006F1100052AAA02306F07AFE0023009335
:10C1200052AAA02306210548FCF770FA0DF5227DDE
:10C1300070BD00BFD48F0100AC8F010058A5FF1F58
:10C14000428938B5038992B29BB29A426CD0428937
:10C15000038992B29BB29A4234D2038942899B1AD4
:10C160009BB2002B37D0B0F83832002B36D13A4A88
:10C170001278002A5DD01C4618E04168428992B2CC
:10C180008D5C04734289013292B2428141890288F6
:10C1900089B292B2914200D344815A1CC11893B221
:10C1A000442BA0F8383281F8705150D0018942896F
:10C1B00089B292B29142E0D1027B02F0FF05002ADF
:10C1C000DBD1EAE741890388028913FA82F35B1A1B
:10C1D0009BB2002BC7D1B0F8383223B304461F48B6
:10C1E000FCF7D4FAA028054635D9B4F83A3201E074
:10C1F000A02D18D95A1C2344A4F83A2293F87011A0
:10C200002046FFF769FFB4F83A32B4F83822A03D6F
:10C210009A42ADB2ECD80023A4F83A32A4F83832EE
:10C2200038BDA0F83A1238BD037B002BD3D0038869
:10C2300097E7B0F83C120029F3D0AA24C2180133C2
:10C240009BB28B4282F87041F8D1A0F838320023BB
:10C25000A0F83A32C2E738BD50A5FF1F58A5FF1F0E
:10C2600001EB41014908483189B296298ABF9623DA
:10C27000A0F83C12A0F83C32704700BF4289038905
:10C2800092B29BB29A421DD04289038992B29BB26C
:10C290009A4208D34389018902885B1A9BB2934270
:10C2A0000AD90020704701890288438912FA83F372
:10C2B0005B1A9BB29342F4D80748A0FB0330C0F34B
:10C2C00087107047037B002BEBD103880248A0FB4B
:10C2D0000330C0F387107047F1F0F0F0022909D065
:10C2E000032905D0012901D00020704705F0EEBBDD
:10C2F00004F0E2BC04F03AB9022909D0032905D0C0
:10C30000012901D00020704705F072BC04F0BCBCCC
:10C3100004F014B9022908B50DD0032907D001296A
:10C3200001D0002008BD05F0ADFBC0B208BD04F08F
:10C33000D7FCC0B208BD04F02DF9C0B208BD00BFE3
:10C3400010B502299DF8084018D003290CD0012906
:10C3500000D010BD1946104605F0C6FB002CF8D0E1
:10C36000BDE8104005F068BC1946104604F06AFCB0
:10C37000002CEED0BDE8104004F07ABC19461046FF
:10C3800004F040F8002CE4D0BDE8104004F0CAB836
:10C39000022926D0032920D0012900D07047134854
:10C3A000134AF0B40468134D134F40F2EE2613788D
:10C3B0003BB12B78DB0704D5036839685B1A0E2B79
:10C3C00006D8036811781B1B21B1B3F5FA6FEED9BB
:10C3D000F0BC7047B342EAD9FAE71146074805F0C6
:10C3E0005FBD1146064805F0A3BC00BF9C030020BA
:10C3F00088050020A0050020180600207C10FF1FE3
:10C400006810FF1F2DE9F04F437890F806E084781C
:10C41000027890F803C090F8048090F8059099B0E5
:10C4200003EB8303072909940EF0010ACEF3400BB6
:10C430004FEA4303CEF3800E4FF000040BD90725DB
:10C4400018AE37196E1C455D07F8345CF5B201343F
:10C450008D42E4B2F4D318A90C4400250999009147
:10C46000CDF818E0CDF814B0CDF810A0CDF80C90B0
:10C47000CDF80880CDF804C00BA904F8345C03485B
:10C48000F9F7EAFA19B0BDE8F08F00BFE8D2FF1F54
:10C490002DE9F041437890F803E0027890F802C06B
:10C4A00090F8048003EB83030EEB8E0E052992B007
:10C4B0004FEA43034FEA4E0E4FF000040BD9052517
:10C4C00012AE37196E1C455D07F8345CF5B20134C5
:10C4D0008D42E4B2F4D312A90C440025CDF80880B3
:10C4E0008DE8005005A904F8345C0348F9F7F6FA22
:10C4F00012B0BDE8F08100BFE8D2FF1FF0B50446DE
:10C500008FB0A679257AA378627821780396667928
:10C51000029626790196E6780096C5F38017EE0913
:10C5200008970796C5F34017E67A069705F00F05BA
:10C5300094F80AE00595677A0D96667BCDF830E0B1
:10C54000257B0648E479049401EB81010B970A9658
:10C550000995F9F7E7FA0FB0F0BD00BFE8D2FF1F69
:10C56000F0B584780278437890F803E004EB840413
:10C5700004294FEA440C91B04FF000040BD9042574
:10C5800010AE37196E1C455D07F8345CF5B2013406
:10C590008D42E4B2F4D310A90C4400258DE800507C
:10C5A00003A904F8345C0248F9F724FB11B0F0BD8C
:10C5B000E8D2FF1F30B5A5B0E0230A788DF80C3023
:10C5C000F1238DF80E30AAB10324A31E24AD254417
:10C5D000DBB205F8842CCA5C0134E4B2002AF4D141
:10C5E000A3B20121009103AA8DF80D40FFF7A8FE28
:10C5F00025B030BD03231C46F3E700BFF0B5A5B05E
:10C60000E0230F788DF80C30F22315468DF80E30AC
:10C6100027B3032200E01A46941E24AEE4B2164467
:10C62000531C06F8847C0F5DDBB2002FF3D1D61CBF
:10C63000941CF6B21A46E4B2B3B224A90A440C44DC
:10C640002F120121009102F8847C04F8845C03AA73
:10C650008DF80D60FFF774FE25B0F0BD05231E4672
:10C6600004240322E9E700BF70B50346054600F540
:10C670000071002203F8012B8B424FF00004F9D126
:10C680004FF4B976A5F81042A5F80042A5F8124279
:10C69000A5F8024285F8044285F8144285F815424F
:10C6A000A5F80862304605F0BBFCA5F82842C5F89D
:10C6B0000C02A5F82A42A5F820623046C5F81842B7
:10C6C000A5F81C4285F82C4285F82D4205F0A8FCFF
:10C6D000C5F82402284670BDF0B505468DB07848EF
:10C6E000FCF788FC774B784A1B7817788DF8133065
:10C6F00073488DF814700123E02614240DF10F0205
:10C700000DF10E018DF812308DF810608DF811408A
:10C71000FCF74EFC9DF80E302BB19DF8143043F021
:10C7200002038DF814306648FCF75EFC28B19DF8D2
:10C73000143043F004038DF814306148FCF74CFCCE
:10C7400028B19DF8143043F008038DF814305C488C
:10C75000FCF758FC9DF8143008B143F010039DF825
:10C760000F200AB143F020035849594A097812783A
:10C7700000290CBF002140210B4300218DF814300B
:10C780008DF81510002A40F085808DF81620514B49
:10C790001B78002B36D0504B1B78002B71D04F48A4
:10C7A000F7F73CFA8DF817004C48F7F76DFA4C4B49
:10C7B0008DF818001B786BB34A4803F0CFF84A4B4A
:10C7C0008DF819001B785BB34848FFF7E5FA484B32
:10C7D0008DF81A001B784BB34648FEF7ABFB464B6F
:10C7E0008DF81B001B783BB34448FDF759FC444BC4
:10C7F0008DF81C001B782BB34248FAF757FA8DF8D6
:10C800001D0021E08DF817308DF81830344B1B785F
:10C81000002BD1D18DF81930334B1B78002BD3D19D
:10C820008DF81A30324B1B78002BD5D18DF81B3088
:10C83000314B1B78002BD7D18DF81C30304B1B7837
:10C84000002BD9D18DF81D302F4B1A7800238DF88D
:10C850001E308DF81F301ABB2C4B8DF820201B7812
:10C860003BBB8DF82130002428460094142304AAF1
:10C8700001218DF822408DF82340FFF761FD0DB0B6
:10C88000F0BD0A2322488DF81730F6F771F88DF8BD
:10C890001800BBE71F48F8F707FE8DF8160076E78B
:10C8A0001D48FFF7EBFC194B8DF820001B78002B7F
:10C8B000D7D01A48F4F7E6FB8DF82100D3E700BF84
:10C8C00058A5FF1FAC78FF1F50A5FF1FAD78FF1FB5
:10C8D000580EFF1F570EFF1F540EFF1FB078FF1F8B
:10C8E000560EFF1F70E0FF1F5A0EFF1F9C79FF1F9F
:10C8F000550EFF1FB42AFF1F520EFF1FB073FF1FFC
:10C90000530EFF1FE8D2FF1F5B0EFF1F590EFF1FC4
:10C91000A8FEFF1FC01DFF1F6471FF1F6420FF1FC3
:10C9200070B5B4B00323002402217F22E02605461F
:10C930001C488DF80D308DF808608DF80B108DF8BF
:10C940000C208DF809408DF80A40FCF789FD21463E
:10C950008DF80E0010220DF10F0007F0D7FB0DF13E
:10C960000F011048104EFCF77DFD4D21084617239E
:10C9700002E00846B15C234634AC1C44A3F1150226
:10C98000013304F8C80CD2B2DCB20029F1D1009115
:10C990002846234602AA01218DF80940FFF7D0FC62
:10C9A00034B070BD58A5FF1F2C9501004B1E10B56B
:10C9B0000C466B2B00F28181DFE813F03D01220170
:10C9C00018010E010401FA00F0007F017F01E70069
:10C9D0007F017F017F017F017F017F017F017F0157
:10C9E0007F017F017F017F017F017F017F017F0147
:10C9F0007F017F017F017F017F017F017F017F0137
:10CA00007F017F017F017F017F017F017F017F0126
:10CA10007F017F017F017F017F017F017F017F0116
:10CA20007F017F017F017F017F017F017F017F0106
:10CA30007F017F017F017F017F017F017F017F01F6
:10CA40007F017F017F017F017F017F017F017F01E6
:10CA50007F017F017F017F017F017F017F017F01D6
:10CA60007F017F017F017F017F017F017F017F01C6
:10CA7000DE00D500CC007F01C300BA007F01B10009
:10CA8000A8007F019F006C0096006B0161016C00A3
:10CA9000570175019C4B93F80432002B40F019812B
:10CAA0009A48F7F727FC9A48F5F7CCFF9948F5F72D
:10CAB00015FA9948F6F7EEF9032C40F0CA8097482A
:10CAC000FEF7DAFA9648FDF70BFD9648FCF71CFDD9
:10CAD0009548F8F76DFF9548F4F7FCFB214694481C
:10CAE000BDE81040FBF78ABE874890F80432002B5F
:10CAF000D6D09049FFF75EFDD2E7834890F8043224
:10CB0000002BCDD08C49FFF755FDC9E77E4890F842
:10CB10000432002BC4D08949FFF74CFDC0E77A48A6
:10CB200090F80432002BBBD08549FFF743FDB7E7EF
:10CB3000754890F80432002BB2D08249FFF73AFDD5
:10CB4000AEE7714890F80432002BA9D07E49FFF778
:10CB500031FDA5E76C4890F80432002BA0D07B494A
:10CB6000FFF728FD9CE7684890F80432002B97D027
:10CB70007749FFF71FFD93E7634890F80432002BD5
:10CB80008ED07449FFF716FD8AE75F4890F80432AB
:10CB9000002B85D07049FFF70DFD81E75A4890F8CA
:10CBA0000432002B3FF47CAF6C49FFF703FD77E7BD
:10CBB000554890F80432002B3FF472AF6849FFF7F4
:10CBC000F9FC6DE7504890F80432002B3FF468AF51
:10CBD0006449FFF7EFFC63E74B4890F80432002B01
:10CBE0003FF45EAF6049FFF7E5FC59E7464890F82F
:10CBF0000432002B3FF454AF5C49FFF7DBFC4FE7F6
:10CC0000414890F80432002B6CD14048F7F772FB92
:10CC1000574802F037F94148FEF72EFA4048FDF731
:10CC20005FFC072C3FF454AF3E48FCF76DFC0A2C28
:10CC30003FF451AF4CE7344890F80432002B4DD10B
:10CC40003348F5F7FFFE3348F5F748F93248F6F771
:10CC500021F9474802F016F9042C4BD13048FDF772
:10CC60003FFC3048FCF750FC32E7274890F804328C
:10CC7000002B3FF415AF3F49FFF79CFC10E722481B
:10CC800090F80432002B3FF40BAF3B49FFF792FCC6
:10CC900006E71D4890F80432002B3FF401AF3749F6
:10CCA000FFF788FCFCE6184890F80432002B3FF4AC
:10CCB000F7AE3349FFF77EFCF2E6134890F80432F2
:10CCC000A3B9012CBCD01148F7F714FB022C9FD05C
:10CCD000E9E62C490C48FFF76DFCE1E62A49FFF72D
:10CCE00069FCADE72949FFF765FC8EE72849FFF7A6
:10CCF00061FCE6E70948FEF7BFF9052C8ED109482B
:10CD0000FCF702FCE4E600BFF04CFF1F8084FF1F2D
:10CD10001C7FFF1F28BCFF1F4830FF1F204FFF1F35
:10CD200070E5FF1FC822FF1FE8D2FF1FD019FF1FA9
:10CD300058A5FF1F289101001C920100949001004A
:10CD4000B4900100D0900100EC900100AC91010082
:10CD5000D0910100F89101008490010060900100E1
:10CD6000709001004C9001003C9001002090010067
:10CD7000A8A8FF1F8C9101006C9101004C9101004B
:10CD80003C92010008910100FC8F0100109001000D
:10CD9000589201002DE9F04F0E78C6F3001380F889
:10CDA0000432CD78322DA9B003D9042029B0BDE8D2
:10CDB000F08F4C7891F804E091F802A004F0080399
:10CDC00004F0020704F0040204F0100804F0200C40
:10CDD00004F04009DBB2BEF1050FFFB2D2B20F93EF
:10CDE0005FFA88F85FFA8CFB5FFA89F940F23481C8
:10CDF000BEF1070F00F04E81BEF1060F00F04F812B
:10CE0000BEF10A0F00F05081AEF15B0C5FFA8CFCB2
:10CE1000BCF1110FC9D8AB4B23FA0CFC1CF0010F6D
:10CE2000C3D08B7E10930F2BBFD80B7F1193A3F130
:10CE30007C0CBCF10E0FB8D88C4671469CF807E00C
:10CE4000CDF850E09CF808E0CDF854E09CF809E0FB
:10CE5000CDF858E09CF80AE0CDF85CE09CF80BE0D7
:10CE6000CDF860E09CF80CE0CDF864E09CF80DE0B3
:10CE7000CDF868E09CF80EE0CDF86CE09CF80FE08F
:10CE8000CDF870E09CF810E0CDF874E09CF811E06B
:10CE9000CDF878E09CF814E0CDF87CE09CF815E043
:10CEA0009CF805302792CDF880E09CF806209CF88D
:10CEB00016E012931392CDF884E09CF817E0CDF8B9
:10CEC00088E09CF81BE0CDF88CE09CF81DE0CDF8E4
:10CED00090E09CF81EE0CDF894E09CF81FE0CDF8BF
:10CEE00098E0FFF763FD7849DFF838E2774804F00F
:10CEF00001040C70F4432946C4F3C0148EF80040BA
:10CF0000F8F7C2FA724C7348003718BF0127294658
:10CF10002770F5F763FD109C6F482146F7F742F93B
:10CF200021466E48F5F79EFF23996C48F5F7A6FF5A
:10CF300021466B48F5F7B8F921466A486A4CF5F77F
:10CF400047FF279A6948003218BF012229462270FC
:10CF500002F0F4FC1F9A6548C6F3C00102F02EFDF2
:10CF60000F9C634A6348231C18BF01232946137092
:10CF7000FEF702FF20995F48FEF73EFF18F1000818
:10CF80005D4B5E4818BF4FF00108294683F80080CA
:10CF9000FDF7C0FF21995948FDF7FCFF19F1000981
:10CFA000574B584818BF4FF00109294683F80090A5
:10CFB000FDF766F822995348FDF7A2F8524B534803
:10CFC0000AF0010229461A70FFF74AF9504B5148FE
:10CFD0002499CAF3400A83F800A0F4F74DF8119D94
:10CFE000269B259A4C48A5F1800149B2F3F78CFEA7
:10CFF0001B9C139A129B1E981D990794179C0A90CC
:10D0000009911C9F1A9819990394803A1BF1000406
:10D01000A3F18003414D0C920B9308970690059164
:10D0200016981599149B189F029018BF0124C6F3F7
:10D030004012019100930D920497C6F38003C6F34A
:10D04000400206F0010136482C70FBF741FF3448DE
:10D05000FBF73AFC0020A9E6BEF1010F03D1E3077C
:10D060007FF5A3AEDDE6BEF1020F0BD0BEF1030FDC
:10D070000CD0BEF1040F1CD10F9B002B7FF4D1AE5E
:10D08000704693E6002F3FF490AECAE6002A3FF4C4
:10D090008CAEC6E6B9F1000F3FF487AEC1E61AF0D8
:10D0A000010F3FF482AEBCE6BBF1000F3FF47DAE52
:10D0B000B7E6BEF1050F7FF4B4AEB8F1000F3FF450
:10D0C00074AEAEE6BFFD0300580EFF1FC01DFF1F6C
:10D0D000570EFF1FA8FEFF1FB078FF1F4830FF1F2D
:10D0E00028BCFF1F1C7FFF1F560EFF1F70E0FF1F95
:10D0F0005A0EFF1F9C79FF1F550EFF1FB42AFF1FFA
:10D10000520EFF1FB073FF1F5B0EFF1F6471FF1FE6
:10D11000590EFF1F6420FF1F18F5FF1F530EFF1F3E
:10D1200058A5FF1F540EFF1F08B5284B09781B7820
:10D130008B4222D0052913D9072936D0062939D0A8
:10D140000A2915D0A1F15B03DBB2112B0ED8204ABE
:10D1500022FA03F3DB0709D5FFF728FC002008BDFE
:10D1600001290CD11B4B1B78002BF5D1042008BDE5
:10D17000194B1B78002BF9D0EEE7002008BD0229DF
:10D1800008D003290CD0042919D1144B1B78002B8B
:10D19000ECD0E1E7124B1B78002BDDD1042008BD59
:10D1A000104B1B78002BE1D0D6E70F4B1B78002BE0
:10D1B000DCD0D1E70D4B1B78002BD7D0CCE705296D
:10D1C000CAD10B4B1B78002BD0D0C5E7AC78FF1F22
:10D1D000BFFD0300580EFF1F530EFF1F5A0EFF1F07
:10D1E000570EFF1F560EFF1F520EFF1F5B0EFF1F35
:10D1F000550EFF1F10B54FF4E12204460121FFF741
:10D20000C7F820464FF416520321BDE81040FFF73F
:10D21000BFB800BFF0B5044687B01646912900F2AA
:10D220007884DFE811F07304700461044604330469
:10D23000760476047604E7037604CA03760476045B
:10D24000760476047604A903890376044103760400
:10D250007604760476041C037604FA027604DD0272
:10D26000BD02A00276048302760476047604760476
:10D2700076047604760476047604760476047604DE
:10D28000760476047604620241027604760476041B
:10D2900076047604760476047604760476047604BE
:10D2A0007604760476042402760476047604760402
:10D2B0000702CB0176047604AE0176047604760488
:10D2C0007604760476049101760476047604760476
:10D2D0006E01760476047604760476047604760489
:10D2E000760476047604530138011D01F9007604B2
:10D2F0009200760476047604760476047604760446
:10D30000760476047604760476047604760476044D
:10D31000760476047604760476047604760476043D
:10D32000760476047604C4007604760476047604E3
:10D33000760476047604760476047604760476041D
:10D34000760476047604BD00BD00AB4A12783AB18B
:10D35000AA4D2A78002A00F0E1840A2A00F0DE842F
:10D3600002221646A64890F8043213B1A549FFF7E9
:10D3700045F905200022034600924FF0E00E7F277A
:10D3800065258DF8110004AA012120468DF814604E
:10D390008DF810E08DF812708DF81350FEF7D0FF65
:10D3A0000023A4F80032A4F8023207B0F0BD002B2D
:10D3B000F6D0013B9BB201333344012004E084F8F2
:10D3C00015020136B342EBD094F8142202F0FF05A7
:10D3D000002AF4D1D4F80C12B4F81022377892B2A3
:10D3E0008F54B4F81022013292B2A4F81022B4F88B
:10D3F0001012B4F8082289B292B2914228BFA4F860
:10D400001052B4F81012B4F8122289B292B29142BA
:10D4100008BF84F81402D4E7032B00F20584042229
:10D420001546774890F8043213B17749FFF7E6F8CC
:10D4300005200022009203464FF0E00E7F2763266E
:10D4400004AA8DF8145001218DF8110020468DF8A2
:10D4500010E08DF812708DF81360FEF771FF9FE7F2
:10D460000D2B00F2AA8304221546654890F8043279
:10D4700013B16649FFF7C2F8052000220092034667
:10D480004FF0E00E7F27622604AA8DF81450012188
:10D490008DF81100DAE7052B00F28083042215468F
:10D4A000574890F8043213B15949FFF7A7F80520FF
:10D4B0000022009203464FF0E00E7F27612604AA67
:10D4C0008DF8145001218DF81100BFE7072B00F2F1
:10D4D0005583042215464A4890F8043213B14D4949
:10D4E000FFF78CF805200022009203464FF0E00E73
:10D4F0007F27602604AA8DF8145001218DF81100B1
:10D50000A4E7454A12783AB13C4A1278002A00F062
:10D5100018840A2A00F0158402221546384890F82B
:10D52000043213B13D49FFF769F80520002200924B
:10D5300003464FF0E00E7F27552604AA8DF81450BD
:10D5400001218DF8110081E7354A12783AB12B4D4F
:10D550002A78002A00F03184062A00F02E84022264
:10D560001646274890F8043213B12E49FFF746F8C3
:10D5700005200022034600924FF0E00E7F27502541
:10D58000FFE6294A12783AB11C4D2A78002A00F0A9
:10D59000BB83072A00F0B88302221646184890F889
:10D5A000043213B12149FFF729F805200022034670
:10D5B00000924FF0E00E7F274925E2E61A4A1278E2
:10D5C0003AB10E4D2A78002A00F0C783072A00F0EE
:10D5D000C483022216460A4890F8043213B1144953
:10D5E000FFF70CF805200022034600924FF0E00EF2
:10D5F0007F274625C5E600BF530EFF1FAC78FF1FEF
:10D60000F04CFF1FF4940100CC920100AC92010099
:10D610008C9201006C920100590EFF1F10950100C1
:10D620005B0EFF1FD4940100520EFF1FB89401003F
:10D6300094940100AC4A12783AB1AC4D2A78002A91
:10D6400000F03C83072A00F0398302221646A848DE
:10D6500090F8043213B1A749FEF7D0FF052000224D
:10D66000034600924FF0E00E7F27452589E6A24A47
:10D6700012783AB19D4D2A78002A00F03283052AAB
:10D6800000F02F8302221646994890F8043213B115
:10D690009A49FEF7B3FF05200022034600924FF09F
:10D6A000E00E7F2740256CE6954A12782AB18F4F0D
:10D6B0003A7812F0FB0F00F06D83022215468C4879
:10D6C00090F8043213B18F49FEF798FF052000222D
:10D6D000009203464FF0E00E7F27312604AA8DF812
:10D6E000145001218DF81100B0E6854A12782AB154
:10D6F0007E4F3A7812F0FB0F00F07283022215463B
:10D700007B4890F8043213B17F49FEF777FF05207C
:10D710000022009203464FF0E00E7F27302604AA35
:10D720008DF8145001218DF811008FE6774A127898
:10D730003AB16E4D2A78002A00F01983032A00F0CE
:10D740001683022216466A4890F8043213B17049D3
:10D75000FEF754FF05200022034600924FF0E00E32
:10D760007F2720250DE66B4A1278002A40F046827A
:10D77000022215465E4890F8043213B16649FEF75E
:10D780003DFF05200022009203464FF0E00E7F2768
:10D790001E2604AA8DF8145001218DF8110055E6BB
:10D7A0005C4A1278002A00F0E681012B00F03083F9
:10D7B000042215464E4890F8043213B15749FEF73B
:10D7C0001DFF05200022009203464FF0E00E7F2748
:10D7D0001D2604AA8DF8145001218DF8110035E69C
:10D7E0004C4A1278002A40F0148202221546404822
:10D7F00090F8043213B14A49FEF700FF05200022D9
:10D80000009203464FF0E00E7F271C2604AA8DF8F5
:10D81000145001218DF8110018E63E4A1278002AB2
:10D8200000F09781314D2A7812F0FD0F40F0918180
:10D830003C4A1278002A00F0E48231461A463A48FF
:10D84000F6F7DEF80646002E40F071832B78002BA9
:10D850007FF4A6AD02212046FFF7A8F8A0E52D4AE7
:10D8600012784AB1214F3A7812F0FD0F04D12D4AB7
:10D870001278002A40F00983022215461C4890F8CD
:10D88000043213B12949FEF7B9FE052000220092A7
:10D8900003464FF0E00E7F27182604AA8DF8145097
:10D8A00001218DF81100D1E5214B1B7823B10F4EDA
:10D8B0003378012B40F20283022215460C4890F87F
:10D8C000043213B11B49FEF799FE05200022009295
:10D8D00003464FF0E00E7F27132604AA8DF814505C
:10D8E00001218DF81100B1E5520EFF1FAC78FF1F2A
:10D8F000F04CFF1F6C940100550EFF1F5094010067
:10D900005A0EFF1F3494010018940100560EFF1F99
:10D91000F4930100570EFF1FD89301009C93010060
:10D92000B8930100540EFF1FB078FF1F80930100D1
:10D93000580EFF1F64930100C34A127822B1C34FEF
:10D940003A78012A40F2D58202221546C04890F862
:10D95000043213B1BF49FEF751FE052000220092A8
:10D9600003464FF0E00E7F27112604AA8DF81450CD
:10D9700001218DF8110069E5B34A127822B1B34F45
:10D980003A78012A40F2A98202221546B04890F85E
:10D99000043213B1B049FEF731FE052000221026F3
:10D9A000009203464FF0E00E7F270DEB06028DF844
:10D9B000145001218DF8110048E5A44A1278002A7C
:10D9C00000F0628105221546A14890F8043213B197
:10D9D000A249FEF713FE05200022009203464FF0F5
:10D9E000E00E7F270A2604AA8DF8145001218DF835
:10D9F00011002BE5954D2A78632A00F02882022732
:10DA0000A2F15C01C9B206290DD84D2020FA01F11E
:10DA1000C90708D51A46314691480393F3F7A6FD86
:10DA20002A78039B0746A2F16601052940F222816C
:10DA30005D2A00F016825B2A00F01D826C2A00F03D
:10DA4000FC81652A7ED0002F00F0D481804890F8B8
:10DA500004321BB13AB28349FEF7D0FD0520002203
:10DA6000034600924FF0E00E7F2608258DF8110046
:10DA700004AA012120468DF814708DF810E08DF86D
:10DA800012608DF81350FEF75BFC89E40425002238
:10DA90000092E02770262B4604AA01218DF8115030
:10DAA0008DF813508DF810708DF81260FEF748FC59
:10DAB00076E4002B40F08F800421002205200092A4
:10DAC0000346E0277F26032504AA8DF814108DF85D
:10DAD0001100012120468DF810708DF812608DF82C
:10DAE0001350FEF72DFC5BE4242B00F2D8800421B8
:10DAF0000022052000920346E0277F26022504AA83
:10DB00008DF81410E3E7FEF7E7FD49E4FEF708FFA0
:10DB100046E40520012600220D46034600924FF000
:10DB2000E00E7F278DF81100314604AA20468DF8BB
:10DB300013508DF814608DF810E08DF81270FEF718
:10DB4000FFFB2DE41A4631464748F4F719F907461A
:10DB500079E7022216463E4890F8043213B1434951
:10DB6000FEF74CFD05200022034600924FF0E00E28
:10DB70007F271A2505E4022215461BE61946304682
:10DB8000FEF740FC0546002840F0958104200095F2
:10DB90000346E0277026602504AA98E71946304618
:10DBA000FEF776FC0546002840F0828104200095AF
:10DBB0000346E02770266125EEE73046FEF79EFC1F
:10DBC0000546002840F07181042000950346E027B7
:10DBD00070266225E0E73146FFF7A6FA01460028E5
:10DBE0007FF46BAF042500902B464FF0E00E7027BA
:10DBF000032604AA01218DF8115027E41A46314664
:10DC00001B48F5F7A1FF054600283FF4C9AB02B257
:10DC1000B0E51A4631461648F5F75AFF0546002882
:10DC20003FF4BEAB02B2E2E519463046FEF798FC7F
:10DC30000546002840F03681042000950346E02781
:10DC400070266325A8E700BF580EFF1FAC78FF1FA2
:10DC5000F04CFF1F44930100249301001093010036
:10DC6000ECF4FF1FEC9201006C84FF1F8093010015
:10DC7000B078FF1F1A463146B8480393F3F7ACFF5C
:10DC80002A78039B0746D3E61A463146B448F3F791
:10DC900095FA054600283FF483AB02B294E631467C
:10DCA000FFF778F8014600287FF422AF04250090A2
:10DCB0002B464FF0E00E702702269AE73146DAB283
:10DCC000A848FCF791F80646002840F03A812B78E6
:10DCD000002B7FF465AB07212046FEF767FEFFF7B8
:10DCE0005FBB31461A46A048FCF7A6FF064600284F
:10DCF00040F02A812B78002B7FF452AB052120467F
:10DD0000FEF754FEFFF74CBB3146DAB29548FCF7FC
:10DD10006BF806460028DAD002B23FE43146DAB2A8
:10DD20009248F8F7D1FF0646002840F004812B788E
:10DD3000002B7FF435AB0A212046FEF737FEFFF7B4
:10DD40002FBB1A4631468A48F3F71AF805460028D1
:10DD50003FF426AB02B2FFF7E1BB3146DAB28148AD
:10DD6000FCF742F806460028B1D002B233E431464F
:10DD70001A46804801F074FC0646002840F0E7800F
:10DD80002B78002B7FF40CAB03212046FEF70EFE10
:10DD9000FFF706BB1A4631467748FDF71DFF0546DB
:10DDA000002840F0CB803B78002B7FF4F9AA0421B7
:10DDB0002046FEF7FBFDFFF7F3BA31461A466F48DF
:10DDC000FEF738F90646002840F0C4802B78002B77
:10DDD0007FF4E6AA06212046FEF7E8FDFFF7E0BA49
:10DDE0001A4631466448FDF7F7FE05460028DAD0AA
:10DDF00002B285E4042000970346E0277026082538
:10DE0000CAE631461A465E48F4F790FC06461AE523
:10DE10003178012977D000297FF4CAAC594B1B789F
:10DE2000022B7FF4C5AC584B1B78002B3FF4B8AAEB
:10DE30005648F5F7A1FEFFF7B3BA1A4631465448E3
:10DE40000393F3F7F3FE2A78039B0746F9E51A4696
:10DE5000314650480393F3F70BFE2A78039B07469D
:10DE6000CEE51A4631464C480393F3F75FFF2A7814
:10DE7000039B0746DFE51A46314648480393F3F70C
:10DE800013FF2A78039B0746D8E51A4631463F48D8
:10DE9000F5F74EFD054600284BD13B78002B7FF46B
:10DEA0007FAAD7E402B2FFF7BCBA02B2FFF7DDBA2D
:10DEB00002B2FFF7F5BA02B2FFF70DBB3848F7F729
:10DEC00089F9054678BB3378002B7FF469AA0121D4
:10DED0002046FEF76BFDFFF763BA1A46314630481D
:10DEE000F7F7D6F8054600BB3B78002B7FF458AA1D
:10DEF000EDE71A4631462A48F7F71CF9054600288F
:10DF0000F2D002B222E51F4A1278022A7FF450AC06
:10DF10001D4A1278002A7FF443AA19461B48F5F7D8
:10DF20002BFEFFF73DBA02B2C8E402B22EE532B2D0
:10DF300011E602B2A2E402B2FFF714BA02B2FFF78E
:10DF4000BEBB02B2FFF783BB02B2FFF79DBB02B2BA
:10DF5000FFF7F9BB02B2FFF704BB00BF7084FF1FDD
:10DF6000D019FF1FB073FF1FB42AFF1FE8D2FF1F95
:10DF70006420FF1F70E0FF1F9C79FF1F6471FF1F6B
:10DF8000A8FEFF1FAC78FF1F50A5FF1FB078FF1F32
:10DF9000CC19FF1FA4FEFF1F6CE5FF1F54A5FF1F38
:10DFA000C01DFF1F164B1B78012B00D97047154B66
:10DFB0001B78002BFAD030B591B0E02410238DF8F7
:10DFC0000C408DF80E30C2B10332D4B201390323B4
:10DFD00010AA1A440133DBB211F8015F02F8345C75
:10DFE000A342F5D1A3B200220092012103AA8DF829
:10DFF0000D40FEF7A5F911B030BD03231C46F2E732
:10E00000AC78FF1F580EFF1F164B1B78012B00D951
:10E010007047154B1B78002BFAD030B589B0E0243F
:10E0200011238DF80C408DF80E30C2B10332D4B2FA
:10E030000139032308AA1A440133DBB211F8015F46
:10E0400002F8145CA342F5D1A3B200220092012190
:10E0500003AA8DF80D40FEF773F909B030BD032314
:10E060001C46F2E7AC78FF1F580EFF1F0E4B1B78C3
:10E07000012B00D970470D4B1B78002BFAD070B5DF
:10E0800084B00324002200922346E026122503AA2E
:10E0900001218DF80D408DF80C608DF80E50FEF7C3
:10E0A0004FF904B070BD00BFAC78FF1F580EFF1FC2
:10E0B0000E4B1B78012B00D970470D4B1B78002BA2
:10E0C000FAD070B584B00324002200922346E026E3
:10E0D000132503AA01218DF80D408DF80C608DF8F1
:10E0E0000E50FEF72DF904B070BD00BFAC78FF1FD5
:10E0F000580EFF1F30B5174C247814F0FD0F8DB06B
:10E1000023D1154C247804B300290CBF18241A24F9
:10E11000E0218DF80A408DF80810C3B10333DDB259
:10E12000013A03230CA919440133DBB212F8014F61
:10E1300001F8284CAB42F5D1ABB20022009201218C
:10E1400002AA8DF80950FEF7FBF80DB030BD03238D
:10E150001D46F2E7AC78FF1F570EFF1F0F4B1B78D1
:10E1600013F0FD0302D10E4A127802B9704770B560
:10E1700084B000294FF00304009314BF1B26192616
:10E180002346E02503AA01218DF80E608DF80D408D
:10E190008DF80C50FEF7D4F804B070BDAC78FF1FBA
:10E1A000570EFF1F174B1B78032B01D003B170478D
:10E1B000154B1B78002BFAD030B5A5B0E0242023F6
:10E1C0008DF80C408DF80E30C2B10332D5B2013952
:10E1D000032324AA1A440133DBB211F8014F02F8D9
:10E1E000844CAB42F5D1ABB200220092012103AACC
:10E1F0008DF80D50FEF7A4F825B030BD03231D4661
:10E20000F2E700BFAC78FF1F560EFF1F0E4B1B78C6
:10E21000032B01D003B170470C4B1B78002BFAD0B5
:10E2200070B584B00324002200922346E026212505
:10E2300003AA01218DF80D408DF80C608DF80E5069
:10E24000FEF77EF804B070BDAC78FF1F560EFF1FBE
:10E25000164B1B7813F0FB0F24D1154B1B780BB317
:10E2600030B5A1B0E02430238DF808408DF80A3095
:10E27000CAB10332D5B20139032320AA1A440133AB
:10E28000DBB211F8014F02F8784CAB42F5D1ABB2DA
:10E2900000220092012102AA8DF80950FEF750F8E1
:10E2A00021B030BD704703231D46F1E7AC78FF1F56
:10E2B0005A0EFF1F164B1B7813F0FB0F24D1154B82
:10E2C0001B780BB330B5C3B0E02431238DF80C407C
:10E2D0008DF80E30CAB10332D5B20139032342AAF8
:10E2E0001A440133DBB211F8014F02F8FC4CAB4287
:10E2F000F5D1ABB200220092012103AA8DF80D5096
:10E30000FEF71EF843B030BD704703231D46F1E70A
:10E31000AC78FF1F5A0EFF1F0D4B1B7813F0FB0349
:10E3200002D10C4A127802B9704770B584B0032448
:10E330000093E0262346322503AA01218DF80D40E3
:10E340008DF80C608DF80E50FDF7FAFF04B070BD2B
:10E35000AC78FF1F5A0EFF1F174B1B78052B01D0FF
:10E3600003B17047154B1B78002BFAD030B5A5B020
:10E37000E02440238DF80C408DF80E30C2B10332FA
:10E38000D5B20139032324AA1A440133DBB211F8B0
:10E39000014F02F8844CAB42F5D1ABB2002200929F
:10E3A000012103AA8DF80D50FDF7CAFF25B030BD3D
:10E3B00003231D46F2E700BFAC78FF1F550EFF1F79
:10E3C0000E4B1B78052B01D003B170470C4B1B780B
:10E3D000002BFAD070B584B00324002200922346AB
:10E3E000E026412503AA01218DF80D408DF80C602F
:10E3F0008DF80E50FDF7A4FF04B070BDAC78FF1F80
:10E40000550EFF1F174B1B78072B01D003B1704728
:10E41000154B1B78002BFAD030B5A5B0E02445236E
:10E420008DF80C408DF80E30C2B10332D5B20139EF
:10E43000032324AA1A440133DBB211F8014F02F876
:10E44000844CAB42F5D1ABB200220092012103AA69
:10E450008DF80D50FDF774FF25B030BD03231D4628
:10E46000F2E700BFAC78FF1F520EFF1F174B1B785F
:10E47000072B01D003B17047154B1B78002BFAD046
:10E4800030B5A5B0E02446238DF80C408DF80E3051
:10E49000C2B10332D5B20139032324AA1A4401338D
:10E4A000DBB211F8014F02F8844CAB42F5D1ABB2AC
:10E4B00000220092012103AA8DF80D50FDF740FFC4
:10E4C00025B030BD03231D46F2E700BFAC78FF1F27
:10E4D000520EFF1F0E4B1B78072B01D003B1704764
:10E4E0000C4B1B78002BFAD070B584B003240022AB
:10E4F00000922346E026492503AA01218DF80D400C
:10E500008DF80C608DF80E50FDF71AFF04B070BD49
:10E51000AC78FF1F520EFF1F0E4B1B78072B01D04C
:10E5200003B170470C4B1B78002BFAD070B584B048
:10E530000324002200922346E026482503AA012155
:10E540008DF80D408DF80C608DF80E50FDF7F8FE3B
:10E5500004B070BDAC78FF1F520EFF1F254B1B7817
:10E560000A2B01D003B17047234B1B78002BFAD044
:10E5700070B5ADF5027DE023FC2A8DF808301ED879
:10E58000D31C65248DF809308DF80A406AB1551EF8
:10E59000ADB202AA0335154401390DF10A0211F892
:10E5A000014F02F8014FAA42F9D1002100919BB21C
:10E5B00002AA0121FDF7C4FE0DF5027D70BD561EB5
:10E5C000B6B2531D0436002565240DF1080E8DF8F2
:10E5D0000A30013976448DF809508DF80B400DF161
:10E5E0000B0311F8014F03F8014FB342F9D1131D8A
:10E5F000DBE700BFAC78FF1F530EFF1F104B1B78EB
:10E600000A2B01D003B170470E4B1B78002BFAD0B8
:10E61000F0B587B0042500220C4600922B46E02777
:10E62000662603AA01218DF80F408DF80D508DF854
:10E630000C708DF80E60FDF783FE07B0F0BD00BFD3
:10E64000AC78FF1F530EFF1F0E4B1B780A2B01D017
:10E6500003B170470C4B1B78002BFAD070B586B015
:10E660000324002200922346E026672503AA012105
:10E670008DF80D408DF80C608DF80E50FDF760FEA2
:10E6800006B070BDAC78FF1F530EFF1F254B1B78E3
:10E690000A2B01D003B17047234B1B78002BFAD013
:10E6A00070B5ADF5027DE023FC2A8DF808301ED848
:10E6B000D31C55248DF809308DF80A406AB1551ED7
:10E6C000ADB202AA0335154401390DF10A0211F861
:10E6D000014F02F8014FAA42F9D1002100919BB2EB
:10E6E00002AA0121FDF72CFE0DF5027D70BD561E1C
:10E6F000B6B2531D0436002555240DF1080E8DF8D1
:10E700000A30013976448DF809508DF80B400DF12F
:10E710000B0311F8014F03F8014FB342F9D1131D58
:10E72000DBE700BFAC78FF1F590EFF1F30B5C3B049
:10E7300002ADE02480232C70AB70A2B10332D4B2BE
:10E740000139032311F8012FEA540133DBB2A3424C
:10E75000F8D1A3B2002100912A4601216C70FDF787
:10E76000EFFD43B030BD03231C46F3E72DE9F04332
:10E770000446C3B0C61C071D012501212046FDF734
:10E78000ADFD8046B8B101212046FDF7C3FDB4F8C8
:10E790000032002B6ED1E02806BF2070A4F8005292
:10E7A000A4F80032A4F8023201212046FDF796FDBC
:10E7B00080460028E7D18648FAF720FC4BF67F33E5
:10E7C0009842B4F81222B4F8103288BFA4F800823C
:10E7D00092B29BB288BFA4F802829A4200F0DD8018
:10E7E000B4F81222B4F8103292B29BB29A427DD29F
:10E7F000B4F81032B4F81282C8EB03081FFA88F894
:10E80000B8F1000F40F0828003212046FDF766FD3D
:10E81000B0F1000840F3B980D4F81832984500F000
:10E82000C480B8F1F90F40F3B08003AE08F1FF37B0
:10E8300037440DF10B050DF2051901E0A9450CD087
:10E8400003212046FDF766FDD4F8182205F8010FD4
:10E85000013ABD42C4F81822F0D1C2EB0802D2B28C
:10E8600031462046FFF762FF0023A4F81C3243B074
:10E87000BDE8F083012B15D0022B1AD0E0545A1CAE
:10E88000B4F8021292B29142A4F800227FF475AF5C
:10E89000FF2923D9033B9BB23A46E1782046FEF795
:10E8A000B9FC6AE702236070A4F80202A4F80032FF
:10E8B00063E7B4F80232A0700322A4F800221BB967
:10E8C000FF30A4F8020258E7032B7FF456AF01464D
:10E8D000002332462046FEF79DFC4EE7023B9BB2EA
:10E8E0003246A1782046FEF795FC46E7B4F812823E
:10E8F000B4F80822B4F8103212FA83F3C8EB030814
:10E900001FFA88F8B8F1000F3FF47EAF03212046CC
:10E91000FDF7F2FC404555DB00273D4603AE25E000
:10E92000D4F80C22B4F812329BB2D25C84F81452A0
:10E93000B4F812328DF80C2001339BB2A4F81232D5
:10E94000B4F81222B4F8083292B29BB29A4201D3C0
:10E95000A4F8125201231F44032100953246204699
:10E96000FDF7EEFCBBB298457FF64EAFB4F810222F
:10E97000B4F812328DF80C5092B29BB29A42CFD1B9
:10E9800094F81432002BCBD1E4E70023C4F81882AA
:10E99000A4F81C3243B0BDE8F08394F81432002B85
:10E9A0003FF432AFB4F808822AE7B4F81C32632B84
:10E9B0003FF63BAFB8F1F90F3FF737AF0133A4F89B
:10E9C0001C3254E71FFA80F8B8F1000FA4D11BE7FE
:10E9D00058A5FF1F144B1B78632B00D0704730B530
:10E9E000A5B0E02408238DF80C408DF80E30C2B19C
:10E9F0000332D4B20139032324AA1A440133DBB20F
:10EA000011F8015F02F8845CA342F5D1A3B20022A1
:10EA10000092012103AA8DF80D40FDF791FC25B06D
:10EA200030BD03231C46F2E7AC78FF1F144B1B7864
:10EA3000602B00D0704730B58BB0E02409238DF8EF
:10EA400008408DF80A30C2B10332D4B20139032331
:10EA50000AAA1A440133DBB211F8015F02F8205C04
:10EA6000A342F5D1A3B200220092012102AA8DF89F
:10EA70000940FDF765FC0BB030BD03231C46F2E7EF
:10EA8000AC78FF1F90F804320BB1FDF793BD7047CF
:10EA900090F804320BB1FDF7B1BD70472DE9F0439A
:10EAA0008E4690F80412A5B000293ED09EF80010C2
:10EAB000E025F3248DF80C508DF80E40002937D056
:10EAC000032500E02546AE1E24AFF6B22F446C1C91
:10EAD00007F8841C1EF80610E4B20029F2D16E1D5E
:10EAE000AF1C05F10309F6B204351FFA86F8FFB230
:10EAF0005FFA89F9EDB29E4624AB1C4494461F444C
:10EB000099441D4412120121009104F8842C4FEA0B
:10EB10002E2407F884CC434609F8844C03AA05F850
:10EB200084EC8DF80D60FDF70BFC25B0BDE8F0839B
:10EB30004FF00708464606254FF005090427032431
:10EB4000D9E700BF2DE9F04F90F80442A5B0BDF918
:10EB5000B890002C52D091F800E0E025F4248DF814
:10EB60000C508DF80E40BEF1000F4AD0032500E096
:10EB70002546AE1E24AFF6B22F446C1C07F884EC79
:10EB800011F806E0E4B2BEF1000FF1D105F107087B
:10EB900005F1020B05F1030C05F1040E6F1D5FFA80
:10EBA00088F806351FFA88FA5FFA8BFB5FFA8CFC4F
:10EBB0005FFA8EFEFFB2EDB21E4624AB1C449B44AE
:10EBC0009C449E441F441D44012153464FEA222A7F
:10EBD000009104F884AC4FEA262A4FEA29240BF866
:10EBE000842C0CF884AC03AA0EF8846C07F8844CCF
:10EBF00005F8849C8DF80D80FDF7A2FB25B0BDE8DB
:10EC0000F08F4FF0090AD046082507274FF0060E6F
:10EC10004FF0050C4FF0040B0324CDE72DE9F04F26
:10EC200090F80442A9B0BDF9C880BDF9CCC0002C51
:10EC300067D01D460F78E0238DF81C30F5238DF842
:10EC40001E30002F60D0032400E04C46A31E28AEE7
:10EC5000DBB2264404F1010906F8847CCF5C5FFA3C
:10EC600089F9002FF1D104F1090304F1020B04F139
:10EC7000030A211D04F1050EA71DE61D0834DBB2B1
:10EC8000E4B205935FFA8BFB9BB25FFA8AFAC9B2D2
:10EC90005FFA8EFEFFB2F6B2049428AC61180391BD
:10ECA00004990295A14404EB0A05A3442144A64417
:10ECB00027442644029C04914FEA222A0121009114
:10ECC00009F884AC4FEA242A0BF8842C05F884ACAC
:10ECD000039D9DF8084005F8844C049C4FEA2829C0
:10ECE0004FEA2C2B0EF8849C07AA07F8848C06F8B0
:10ECF00084BC04F884CC9DF814408DF81D40FDF7C9
:10ED00001FFB29B0BDE8F08F0A210B230491059366
:10ED1000092608274FF0070E06214FF0050A4FF08D
:10ED2000040B4FF00309B8E7014B185C704700BFB4
:10ED3000689501000B4A10B4C0F30723C4B2C0F3B6
:10ED40000741145DD35C515C000E2344105C51FA02
:10ED500083F350FA83F0C0B283B003B05DF8044B84
:10ED6000704700BF68950100F0B583B0CDE90001A0
:10ED7000134A9DF804309DF80510D65C9DF80630C6
:10ED8000555CD45C9DF80710C7B2C0F3072312F896
:10ED900007E0D35C515CC0F30747000ED75D105C01
:10EDA000734457FA83F350FA83F056FA80F055FA19
:10EDB00080F054FA80F051FA80F0C0B203B0F0BD98
:10EDC000689501000346002203F8042B00F11801A6
:10EDD00043F8042B8B42FBD100F59651F0B5183166
:10EDE000002523F8025B8B424FF00002F9D141F27B
:10EDF000D82741F2DA2341F2DC2641F2DE2500F584
:10EE00009751C253C25242F20F73835341F2E22E22
:10EE1000435341F2E4270B8041F2E82641F2EC250E
:10EE200041F2EE2120F80E3000F59854C353825180
:10EE300000F59753425342541033103423F8022BF9
:10EE4000A3424FF00001F9D141F2103200F598537E
:10EE500000F5995481521233123423F8021B9C425C
:10EE60004FF00002F9D141F2323641F2343441F22E
:10EE7000383141F23C336325825305554250C2522A
:10EE8000F0BD00BFF0B441F2E82141F2DA2541F2D1
:10EE9000D824002341F234324353037003534350C8
:10EEA0006321815441F2DC2741F2DE2600F59755BB
:10EEB00041F2E22441F2E42142F20F72C253825342
:10EEC00041F210372A8041F23236025341F2EC25EA
:10EED000425241F2EE2441F2383141F23C32C35306
:10EEE0008353435303554350F0BC8352704700BFD4
:10EEF000F0B5044683B0002A00F08A80464F4FF4F4
:10EF00007A5E3E467546002014E09E42B8BF1E461B
:10EF10009D42A8BF1D464B1D9BB2B3F5166F00F175
:10EF20000100A1F65B1138BF194683B228BF89B230
:10EF30009A420CD901F10C0334F91330002BE4DCB4
:10EF40009E45A8BF9E469F42B8BF1F46E3E7721981
:10EF50000EEB070352105B10D6187610951B1BB2F0
:10EF60002DB236B212B2019500962C492C48FFF70B
:10EF700055FE41F23432A35C632B33D004EB4301E2
:10EF800041F2F02741F212300133CE53DBB20D5281
:10EF900004F59850074604F597510F2BA35401F13F
:10EFA0000E0100F1100007F10E072CD841F23232A9
:10EFB00041F2103500236353A3521A4631F8026F11
:10EFC00030F8025F32442B44B94212B21BB2F5D181
:10EFD00041F2103041F2323112111B1122526352B0
:10EFE00003B0F0BD04F5975104F598500E31103080
:10EFF00004F598570B4602460E3723F8026FBB42C2
:10F0000022F8025FF9D141F234330022E254CDE715
:10F01000154616461346A6E780C1FFFF7C96010001
:10F02000F04CFF1F2DE9F04FBDF82450BDF928C06A
:10F03000BDF92C80002A79D0AE1C0135DFF8F0E054
:10F040001FFA8CFCB6B2ADB2C8F10009002729E066
:10F050004FEAE40A04F0070413F80AB01EF804406B
:10F060002BEA040403F80A4005F0070BEC101EF825
:10F070000BB013F804A04BEA0A0A03F804A04C1DD5
:10F08000A4B2B4F5166F07F1010728BFA1F65B1112
:10F09000BFB22CBF89B2214602360235BA42B6B29F
:10F0A000ADB243D001F10C0AB41E30F81AA0CCEB7B
:10F0B0000A0A0FFA8AFACA45A4B2C9DBBAF1000FEC
:10F0C0001CDBC2454FEAE40A04F0070413F80AB057
:10F0D0001EF8044044EA0B0403F80A4005F0070B4D
:10F0E0004FEAE5041EF80BB013F804A0B4BF2AEAF7
:10F0F0000B0A4BEA0A0A03F804A0C0E74FEAE40A45
:10F1000004F0070413F80AB01EF804402BEA0404C4
:10F1100003F80A4005F0070BEC101EF80BB013F8CB
:10F1200004A02AEA0B0A03F804A0A8E7BDE8F08FC0
:10F13000E89601002DE9F04F41F2D82305466048DA
:10F14000EB5A05EB830387B05B68C3F313035840A6
:10F15000FFF7F0FD03287BD841F2DA23594935F84F
:10F1600003C0594F0CF60116B6B2B6F5166F26BF9E
:10F17000ACF15F031FFA83F8B04601F1130E6FF094
:10F18000020300244FF47A5008F10C0235F91220E2
:10F190009742B8BF17469042A8BF1046012B19D01E
:10F1A000032B13D0013301D002EB4202144408F1C7
:10F1B00005039BB2B3F5166F24BFA8F65B139BB291
:10F1C0008E4509D0984611F9013FDDE702EB420276
:10F1D000A41AECE7A41AEAE741F2E823EB58A342A9
:10F1E00036DA41F23433EB5C632B53D041F2103307
:10F1F00041F23232EB5EAA5E0292B6F5166F24BF80
:10F20000ACF15F06B6B200270193009704AB14225D
:10F2100031462846FFF706FF2B78DFF8B080BB4267
:10F220000DF1100B14BF4FF0040A4FF0020A08F161
:10F230000409D42301E018F8013F1BF8010B5840E2
:10F24000FFF772FDC8453844C7B2F4D1574503D91A
:10F25000002007B0BDE8F08F41F2DA2341F2E82246
:10F26000EB5AAC5003F6FB0241F2EC2405F5975142
:10F2700041F2DC2092B20227B2F5166F2F530B80B9
:10F280002E5218D341F2DE22653BAB52012007B06B
:10F29000BDE8F08FC3195B10FF1A44F63E1202FB63
:10F2A00007F741F2323041F210311BB247F3CF324F
:10F2B0002A526B52A0E741F2DE23EA52E6E700BF92
:10F2C000ADB507006896010080C1FFFFF096010010
:10F2D00038B50446FFF72EFF30B341F2EE25635DEB
:10F2E000002B36D0013BDBB241F2EE22012BA354BE
:10F2F0001FD104F597531B8803F65F1292B2B2F543
:10F30000166F17D241F2E22162525A1C92B2B2F544
:10F31000166F18D241F2E423E25241F2EE220021AC
:10F32000A1540123237038BD41F2EE23E35C002B8E
:10F33000D8D138BD41F2E222591EA1525A1C92B2D4
:10F34000B2F5166FE6D341F2E422A3F65F13A3529F
:10F35000E3E741F23C3241F2383108486350A352AE
:10F360000121F9F73BFA01210448F9F743FA41F288
:10F37000343263210423A154635538BD58A5FF1FBF
:10F3800038B541F23C330446C35A5BB979220D4883
:10F39000FEF708FF41F2383141F23C32002363505E
:10F3A000A35238BD41F238307B222058B0FBF3F332
:10F3B000C3F3072081F8790081F87A300148FEF71D
:10F3C000F1FEE7E7F04CFF1F2DE9F04141F2E423A5
:10F3D00041F2E222C15A825A41F2DA238A42A4B0AF
:10F3E0000446C35A09D29A4209D941F2DE22A25AEE
:10F3F0009A4211D024B0BDE8F0819A4201D99942D5
:10F40000F3D32046FFF796FE41F2DA2341F2DE22E3
:10F41000E35AA25A9A42EDD141F2EC2304F59758EF
:10F42000E35A022B5CD041F2DC2741F2323641F242
:10F430001035E15B4FF4F0722046FFF759FDA15FF4
:10F44000635FB8F90020364800913649FFF77AFB30
:10F45000A25F635FE15B029208220193009205AB19
:10F460004FF4F0722046FFF7DDFD41F2EC23E55A40
:10F47000013DADB2E5528DB1A5F10105B5FA85F5B5
:10F480006D0905A920468DF81450FFF779FF41F268
:10F49000E8230022E25024B0BDE8F0812249204850
:10F4A000FFF7F0FA29462148F9F798F929461F484D
:10F4B000F9F7A0F91A48FEF7A9FE41F2DE2641F25B
:10F4C000343141F2EE2241F2E82342F20F77632019
:10F4D0002570A7536054A554E55024B0BDE8F081D1
:10F4E000B8F8003003F65F1292B2B2F5166F0BD285
:10F4F00041F2E22162525A1C92B2B2F5166F08D262
:10F5000041F2E423E2528EE741F2E222591EA15277
:10F51000F1E741F2E422A3F65F13A35283E700BFB1
:10F52000F04CFF1F9C960100C496010058A5FF1FD8
:10F53000002B51D02DE9F84F00F5995A00F5965758
:10F5400003F1FF39D3463E465FFA89F9044601EBE1
:10F5500049098D1EA2F102080AF1180A0BF11C0BD1
:10F5600018371A3612E0FFF72FFF338801339BB2AA
:10F57000B3F5166F28BF002333803B8801339BB25D
:10F58000042B88BF0023A9453B8023D038F802EF25
:10F59000BBF800003B88DAF8002035F9021F04EBC5
:10F5A000830301307244CAF80020ABF800005868A9
:10F5B00000294FEA4000B8BF40F00100586033888E
:10F5C00020780C33012824F813102046CBD0FFF705
:10F5D0007FFECAE7BDE8F88F704700BF70B50446EC
:10F5E00000264FF47A602681667366812080267338
:10F5F00002F016FD04F11C0560602661314666616B
:10F60000A6612B4604F13C0223F8021B9342FBD176
:10F6100004F2EC40002203F8012B98424FF0000165
:10F62000F9D14FF49653F022A4F8EC14A4F8EE1498
:10F6300084F8F214C4F8F814A4F8F024C4F8F434EC
:10F640002022284604F062FD05210922034B217483
:10F65000A56162826361204670BD00BFD80FFF1FA5
:10F66000792AF0B402D00420F0BC704742890389A3
:10F6700092B29BB29A4217D04289038992B29BB24E
:10F680009A420BD204890288438912FA83F31B1B26
:10F690009BB29A420CD20520F0BC70474389048982
:10F6A00002881B1B9BB2F4E7037B002BF3D103887A
:10F6B000772BF0D94B1C0125793103E045730133D9
:10F6C00099421CD0027B02F0FF06002AF6D1446862
:10F6D00002891F7892B2A7540289013292B2028144
:10F6E00004890288A4B292B2944228BF0681048998
:10F6F0004289A4B292B2944208BF0573DFE70020AA
:10F70000B2E700BF2DE9F043DFF890C090F8F25463
:10F71000DFF88C90DFF88C80DFF88CE08FB002ACE3
:10F7200004AA40F2772740F2657601F0C003802BEF
:10F730002AD0C02B21D0D3B1002D14BF4B46434655
:10F740002380023489009442C9B2EED102A9224634
:10F750001030042302F072FE00230093224614238B
:10F7600003210D48F8F752FF0FB0BDE8F083002DDC
:10F7700014BF634673462380E3E7002D14BF4FF4A4
:10F780006D7333462380DCE7002D14BF4FF49E7366
:10F790003B462380D5E700BF58A5FF1FC4FEFFFFEF
:10F7A0004CFCFFFF9BF8FFFF89FDFFFF10B58EB0FB
:10F7B000002402A904AA103004230394029402F046
:10F7C0003DFE009404AA142303210248F8F71EFF0B
:10F7D0000EB010BD58A5FF1FB0F8EC3470B504464C
:10F7E0004BB35348F8F7D2FF1428054640F29A80ED
:10F7F000B4F8EE344F4E01E0142D43D95A1C234483
:10F80000A4F8EE2493F83C102046FFF77BFF3378F2
:10F81000143DADB21BB1D4F8F434C4F8F834B4F8E4
:10F82000EE34B4F8EC249A42E6D80023A4F8EE347F
:10F83000A4F8EC3470BD4189028989B292B2914238
:10F8400044D04189028989B292B291421BD2028985
:10F850004189521A92B2FAB1374A1278002A3AD143
:10F86000B4F8F01400295ED07720E21801339BB27F
:10F87000994282F83C00F8D1A4F8EC140023A4F8D3
:10F88000EE34AEE770BD40892288218912FA81F2F8
:10F89000121A92B2002ADFD1D4F8F834002BF1D03A
:10F8A0002348F8F773FF1428054602D83EE0142DCC
:10F8B000E8D92046FFF77AFFD4F8F834143D013B2D
:10F8C000ADB2C4F8F834002BF1D170BD027B002A30
:10F8D000E2D00288BFE7002018E06168628992B236
:10F8E0008D5C20736289013292B2628161892288C3
:10F8F00089B292B2914200D360815A1CE11893B24E
:10F90000782BA4F8EC3481F83C50B7D02189628977
:10F9100089B292B29142E0D1227B02F0FF05002A27
:10F92000DBD1EAE770BDA4F8EE14B5E770BD00BF07
:10F9300058A5FF1F540EFF1F50A5FF1F01EB4101EB
:10F94000890001F5167189B2B1F5966F8ABF4FF43F
:10F950009663A0F8F014A0F8F03470474289038948
:10F9600092B29BB29A421DD04289038992B29BB255
:10F970009A4208D34389018902885B1A9BB2934259
:10F980000AD90020704701890288438912FA83F35B
:10F990005B1A9BB29342F4D80748A0FB0330C0F334
:10F9A00087107047037B002BEBD103880248A0FB34
:10F9B0000330C0F387107047898888884FF49663B6
:10F9C00003FB02F280F8F214C0F8F424704700BF81
:10F9D00001B441EA000313F003036FD1403A41D36D
:10F9E00051F8043B40F8043B51F8043B40F8043B19
:10F9F00051F8043B40F8043B51F8043B40F8043B09
:10FA000051F8043B40F8043B51F8043B40F8043BF8
:10FA100051F8043B40F8043B51F8043B40F8043BE8
:10FA200051F8043B40F8043B51F8043B40F8043BD8
:10FA300051F8043B40F8043B51F8043B40F8043BC8
:10FA400051F8043B40F8043B51F8043B40F8043BB8
:10FA500051F8043B40F8043B51F8043B40F8043BA8
:10FA6000403ABDD2303211D351F8043B40F8043B48
:10FA700051F8043B40F8043B51F8043B40F8043B88
:10FA800051F8043B40F8043B103AEDD20C3205D358
:10FA900051F8043B40F8043B043AF9D204320AD04E
:10FAA000D2071CBF11F8013B00F8013B03D30B78D0
:10FAB00003704B78437001BC704700BF0C2A4AD3D7
:10FAC00010F0030311D0C3F10403D21ADB071CBFEB
:10FAD00011F8013B00F8013B07D311F8013B00F896
:10FAE000013B11F8013B00F8013B11F003033FF427
:10FAF00075AF30B4043AC91AC3F1040C51F8044B81
:10FB0000022B19D0032B0BD0240A51F8043B1D06FD
:10FB100044EA050440F8044B1C46043AF4D216E0CB
:10FB2000240E51F8043B1D0244EA050440F8044B3E
:10FB30001C46043AF4D20AE0240C51F8043B1D049C
:10FB400044EA050440F8044B1C46043AF4D204325B
:10FB5000B1EB0C0130BC043AA0D3013A11F8013BDF
:10FB600000F8013BF9D20B7803704B7843708B7827
:10FB7000837001BC704700BF08B5104C08E02368D3
:10FB800059050DD423681A050FD42368DB0411D45A
:10FB900023685803F3D501F093FA23685905F1D58A
:10FBA00000F00EF823681A05EFD500F07FFD2368FA
:10FBB000DB04EDD501F00CF9EAE700BF3480044026
:10FBC00008B5FFF7D9FF00BF014B10221A8070471C
:10FBD00000200540704700BF094908B50B6830B1E7
:10FBE0006A461844A2F50052904202D208601846B4
:10FBF00008BD03F095FF0C2303604FF0FF3008BDF4
:10FC00003410FF1FEFF3138070B9EFF310836BB95B
:10FC1000EFF305825AB94FF48070EFF311832BB1E3
:10FC2000984228BF184670474FF0FF3070470F2AA0
:10FC300001D81846F1E7014BD05CEEE7F0E300E0B5
:10FC400010B4114B53F8302092F8804234B10123A4
:10FC500079B182F880305DF8044B704703EBC00344
:10FC60005B681A6851B922F002021A605DF8044B11
:10FC7000704782F800315DF8044B704742F0030290
:10FC80001A605DF8044B7047F89601001C4A02EBBD
:10FC9000C00301295B6811D004291BD052F8300041
:10FCA000002280F8802229B1022920D0032922D005
:10FCB0001A6070474FF480721A60704752F8300033
:10FCC0004FF4A27280F880121A601A6822F02002A3
:10FCD0001A60704752F830104FF4A272012081F878
:10FCE00080021A601A6842F020021A60704740F2DF
:10FCF00003121A6070474FF481721A60704700BF98
:10FD0000F896010030B4054B054D064C0022102139
:10FD10001A602A602060196030BC704714D003401C
:10FD200004D0034000D00340704700BF3F2801D8F3
:10FD3000FFF786BF704700BF3F2806D8044B53F833
:10FD4000303093F80002C0B270470020704700BF07
:10FD5000F89601003F2801D8FFF798BF704700BF11
:10FD60002DE9F843054672B6204F214B214A1B6806
:10FD70003C68126862B6520102D5322B88BF01344A
:10FD800095B3C3F5EA331C4EDFF86490DFF8648066
:10FD9000BF334FF47A72A6FB031302FB04F404EBA7
:10FDA000931472B6D9F800103A68D8F800E062B639
:10FDB000C1F5EA33BF33A6FB03031EF0806FC4EB2B
:10FDC00093134FF47A7002D0322988BF013200FBBE
:10FDD0000233B3F57A7F04D3013D05D004F57A747C
:10FDE000DFE702F025F9DCE7BDE8F8839C0300209B
:10FDF00018E000E004ED00E089888888F8B53F4B02
:10FE00003F49DFF81CC13F4E3F4ADFF818E13F4D44
:10FE10003F4C404F4FF0006018604FF0805018602A
:10FE20004FF0005018604FF0804018604FF00040D5
:10FE300018600020086028234EF6FF71CCF80010EF
:10FE4000CEF8003033600EF5012E13602B60236076
:10FE500005F500253B6004F50024B36207F5002793
:10FE6000936206F5012602F501220EF1100E05F649
:10FE7000E87504F6E87407F57F67103220362B60CA
:10FE80002360CEF800303B6013603360224EBB61CC
:10FE9000936109223260A7F5002706F58056203FBE
:10FEA000083638603160BB60F36047F8042C06F513
:10FEB000FD2607F5FE2706F2FC7604373060396030
:10FEC000B360FB6046F8042C0836C7F8FC0F06F652
:10FED000FC76124831602B602360026002F01EF94C
:10FEE000FFF722FF1420FFF73BFF01F023FD4FF443
:10FEF0008C70BDE8F840FFF733BF00BF04E100E0BD
:10FF000004800340148003401C800340248003408D
:10FF10002C800340348003400080034000900B405D
:10FF2000088003400C8003402A4A2B491368F0B430
:10FF300043F4006313600A78284F294E294D2A4C58
:10FF40002A490023092A3B7033702B7023700B70F1
:10FF50003AD03B2A1ED0264B1B780A2B22D03A2BB4
:10FF60002DD01F2824D8002002460126214B224DE7
:10FF70001A70224C5E7004219872022288273C2657
:10FF800040209970DA7459751F74DE7028702260F1
:10FF9000F0BC70471A4B40F213321A60144B1B78B6
:10FFA0000A2BDCD1174B4FF451721F281A60DAD993
:10FFB000C0F34432C0F3471600F01F00D6E7124BDF
:10FFC0004FF451721A60CCE7104B40F213321A60B2
:10FFD000C1E700BF348004403C10FF1F1404002020
:10FFE000A50300202004002015040020A403002005
:10FFF0004810FF1F00B0064021E400E004E100E0EB
:020000021000EC
:1000000004D0044010B0044000D004400CB00440C0
:10001000284B28499B7803F0EC0200F003031343BC
:10002000420700F00F0248BF43F01003042A8B7010
:1000300038D0204B1F4A5B79C10603F0EF0348BF5D
:1000400043F0100353719379820603F0EF03194ACA
:1000500048BF43F010039371C30506D55378117858
:10006000DBB241F020011170537010F4007005D123
:10007000114B124A1968914219D0704730B40D499A
:100080000F4D8A780F4B0C480C4C42F0A0028A703E
:100090002A78046003EBC20340F247325B6830BC4D
:1000A0001A6070478B7943F040038B71C1E7186089
:1000B000704700BF00B006401C040020D400D642A8
:1000C0004810FF1FF8960100214B1B681B053ED509
:1000D00010B5204C237823B101F0AAFF2378002B20
:1000E000FAD11D481D491E4B022400220460CA702B
:1000F0001B78092B1CD03B2B01D11A4B1A601A4BD1
:100100001B7803F07F030A2B1CD03A2B02D1174B2C
:1001100000221A60164A114B1648174912681C79BA
:10012000DB79002303700B700AB10123137010BD3B
:10013000124B40F203121A600B4B1B7803F07F0343
:100140000A2BE2D10E4B40F203121A60E2E770472D
:1001500034800440A403002084E100E000B00640A5
:100160003C10FF1F04D004404810FF1F00D0044083
:10017000A003002014040020A50300200CB00440BC
:1001800010B004400A4A38B50546137803F0FF045E
:10019000002BFAD101212846FFF7DCFD2146284635
:1001A000FFF7C4FD034A044B52F835201A6038BDEE
:1001B000A4030020F89601001C04002009B140F0BF
:1001C0008000174A1378984217D010B4154C246851
:1001D00024050FD503F07F030A2B1DD03A2B12D034
:1001E000002900F07F0114BF602344230A290ED0A8
:1001F0003A2903D010705DF8044B70470A4943F464
:1002000040730B60F6E7084B00241C60E8E70749E1
:1002100043F440730B60EDE7044B00241C60DFE700
:100220004810FF1F3480044000D0044010B0044048
:10023000124B1A7882420CD011490968090507D57A
:10024000092A16D03B2A0AD009280DD03B2801D014
:10025000187070470B4A40F213311160F8E7094AF1
:10026000002109281160F1D1074A40F213311160D1
:10027000EEE7054A00211160E6E700BF3C10FF1FD2
:100280003480044004D004400CB004400D4B1B6883
:1002900013F4006305D03F2805D90B4B00201860EC
:1002A000704718467047094B10B5074C53F830306B
:1002B00023600121FFF74EFD236800221A70012000
:1002C00010BD00BF34800440A0030020F896010058
:1002D0000F4B1B6813F4006308D0172808D03C2884
:1002E00011D00C4A537B03F0FE0353730020704778
:1002F000094B40F202321A60064A537B43F0010375
:10030000537301207047054B40F202321A60F3E745
:100310003480044000B0064008B0044008D00440D7
:100320002DE9F84F2E4B1B681A0546D52D4B1B683F
:100330000BB101221A70DFF8C490DFF8C48099F87D
:100340000040D8F80030284D284E01349C422ABF86
:100350004FF0000A5FFA84FA54460746AB462B7802
:100360009C4219D1FFF74EFC402828DC33791B064C
:10037000F5D59BF80030D8F80010DBB25A1C8A4241
:1003800022D300210A461A4B9B5CDBB2DBB2F3712D
:1003900029702B789C42E5D0272C8ABF154B144B33
:1003A0001B68154988BF283CFFB21F550F4B012021
:1003B000BC22087089F800A0DA70BDE8F88FFF2829
:1003C000CDDD01F035FECAE7272A06D90949273BCA
:1003D0000968CB5CD1B2DBB2D8E7D1B2D3E700BFBA
:1003E000348004401C0400201504002000B00640A6
:1003F000A8030020D0030020A40300202004002034
:100400004410FF1F3E4B1B681A0575D52DE9F04FB0
:100410003C4B1B6883B00BB101221A704318984201
:10042000019363D2DFF8F080DFF8F090364CDFF80C
:10043000F0B0364F451C18E0227892455FFA8AF6F4
:1004400029D0BAF1270F1ED9DBF8002015F8011CBE
:10045000AAF12803D1542A462D4901230B701D44CB
:10046000019B88F800609A4240D298F80030D9F891
:10047000002003F1010A9245DED3237803F0FF0642
:1004800043B10026B246234B15F8012C03F80A208D
:100490002A46E1E7B246BC22FA7005E03A79130633
:1004A0000BD422785245CCD1FFF7ACFB4028F5DDC8
:1004B000FF28F6DD01F0BCFDF3E72278D9F8001043
:1004C000D2B2501C88420BD2272816D9DBF8001074
:1004D000273A8A5CC1B2D2B2D2B2FA712170E0E797
:1004E000002108460B4B1A5CD2B2F5E7074BBC2241
:1004F000DA7003B0BDE8F08F7047C1B2F2E700BF19
:10050000348004401C0400201504002000B0064084
:10051000A4030020A8030020200400204410FF1F93
:10052000D003002010B5044C237823B101F080FDE6
:100530002378002BFAD110BDA4030020084B094AF0
:100540001B781078DBB2C0B2834202D20138C01AE5
:100550007047054A1268013A1044C01A704700BF3C
:1005600020040020150400204410FF1F064A074BFA
:1005700010781B78C0B2DBB2984202D2044A1268EB
:100580001044C01A704700BF14040020A5030020C7
:100590003810FF1F70B4184B184D1B782A78D9B249
:1005A000D2B2914222D0164B1C68531CA34214D3E2
:1005B000002213461348C05CC0B2134E2A70326842
:1005C0004AB1994238BF0919CB1A104909688B42C0
:1005D00001D80023137070BC70473F2B09D90C4819
:1005E0003F3A0068805CDAB2C0B2E6E74FF0FF3015
:1005F000F1E7DAB2DEE700BF14040020A503002013
:100600003810FF1FD4030020A00300204C10FF1F50
:10061000180400200D4A0E4B12781B78DBB29A4268
:1006200011D00C4A11685A1C8A4204D300220A4B8A
:10063000985CC0B270473F2AF9D9084A3F3B12681C
:10064000D05CC0B270474FF0FF30704714040020F8
:10065000A50300203810FF1FD40300201804002039
:100660000D4B1B681B0516D530B40C4B0C4CDA78BF
:100670000C480D4902F0CB024025DA705D74DA783F
:1006800042F03402DA7023780268DBB20B700AB1F0
:100690000023137030BC70473480044000B0064023
:1006A000A5030020A0030020140400202DE9F04140
:1006B000504A137913F0300F44D072B6937D03F093
:1006C000FF01002B57D062B6DFF858814A4B4B4DE3
:1006D00098F800004A4C1B782F68D4F800C0DFF867
:1006E00048E11546C0B2DEB20CE09642A0F13F04EC
:1006F00004D03F2A7CD90CF8043010464A1E12F070
:10070000FF010DD0EB79421CBA42DBB2EDD3002ED3
:10071000F4D000204A1E12F0FF010EF80030F1D193
:10072000384B1A68C3B288F800305AB13649B04223
:1007300038BFBB1B09682CBF831B1B188B4224BF0F
:10074000012313702B48C178C9B20D0618D44A068C
:100750000FD5284B1B795B060BD52C4B2C491B68FE
:1007600000220A7003B11A70224B3C22DA70BDE8F5
:10077000F081BDE8F0814023D179537462B6E1E79E
:1007800003791C06E3D5234BDFF8A0E01D789EF823
:100790000030EDB2DBB29D421ED01F4C1F4A2668CE
:1007A000D2F800C01E4F0DE0272C02791ED91CF88C
:1007B00003202346D2B2D2B2C271027D072A0BD8DF
:1007C0009D4209D05C1CA642A3F12703ECD8037913
:1007D0000023FA5CD2B2EEE7DBB2064A8EF80030B4
:1007E0001379180644BF7C23D370B0E72346F0E7A3
:1007F00010468FE700B00640A50300203810FF1F09
:1008000018040020A00300204010FF1F1C0400203B
:10081000A4030020200400204410FF1FD003002068
:10082000A803002014040020D40300201504002095
:10083000084B1860084B50B101F140021A60074A9A
:10084000074B01F11A0028311060196070474022EF
:100850001A60F4E7180400203810FF1F4C10FF1F27
:100860004010FF1F044B1860044B10B12831196071
:10087000704728221A607047D00300204410FF1FE1
:100880002DE9F84F2C4B1B6807460BB101221A705B
:10089000DFF8BC90DFF8BC8099F80040D8F8003051
:1008A000264D274E01349C422ABF4FF0000A5FFAC2
:1008B00084FA5446AB462B78A3421CD1FFF7A2F929
:1008C00040282BDC33791B06F5D59BF80030D8F88F
:1008D0000010DBB25A1C8A4225D2272A29D919498D
:1008E000273B0968CB5CD1B2DBB2DBB2F371297074
:1008F0002B78A342E2D0272C8ABF124B124B1B68E5
:10090000124988BF283CFFB21F550D4B0120AC2275
:10091000087089F800A0DA70BDE8F88FFF28CADDFA
:1009200001F086FBC7E700210A46074B9B5CDBB260
:10093000DBE7D1B2F9E700BFA00400209904002052
:1009400000C00640540400202C040020980400201D
:10095000A40400205C10FF1F1B4BDFF890C01A6836
:100960001A49F0B542F48052194D1A60DFF880E060
:10097000184F194E194C00238CF800304FF4517267
:100980002B701F2840F213358EF800303B70337007
:1009900025600A6011D819460124114A114D1170C1
:1009A0001148547000212C2740269372082491701E
:1009B0001174D7702E700460F0BDC0F34431C0F3E1
:1009C000471400F01F03E8E7348004400CC00440E3
:1009D00029040020990400209804002008C0044045
:1009E00000C0064023E400E004E100E02804002009
:1009F000A4040020284B28499B7803F0EC0200F067
:100A000003031343420700F00F0248BF43F01003F3
:100A1000042A8B7038D0204B1F4A5B79C10603F043
:100A2000EF0348BF43F0100353719379820603F03C
:100A3000EF03194A48BF43F010039371C30506D56D
:100A400053781178DBB241F020011170537010F42B
:100A5000007005D1114B124A1968914219D07047A4
:100A600030B40D490F4D8A780F4B0C480C4C42F0B6
:100A7000A0028A702A78046003EBC20340F2473276
:100A80005B6830BC1A6070478B7943F040038B7110
:100A9000C1E71860704700BF00C00640A0040020F6
:100AA000D400D8426010FF1FF8960100F8B5124B31
:100AB0001B68DB041ED5114C237823B101F0B8FA72
:100AC0002378002BFAD10E4B0E4A0F4D0F4F104ECC
:100AD000104C1148082119600023D37040F2031113
:100AE0003960316029681579D2792370037011B1AA
:100AF00001230B70F8BDF8BD348004409804002039
:100B000084E100E000C006402404002008C0044046
:100B10000CC0044028040020290400200A4A38B5EB
:100B20000546137803F0FF04002BFAD10121284673
:100B3000FFF710F921462846FFF7F8F8034A044B5F
:100B400052F835201A6038BD98040020F89601004C
:100B5000A004002009B140F08000104A13789842A8
:100B60001AD010B40E4C2468E40412D503F07F03AD
:100B7000082B02D10B4B00241C60002900F07F03DE
:100B800014BF60214421082B03D1064B41F440716E
:100B9000196010705DF8044B704700BF6010FF1FB4
:100BA000348004400CC00440704700BF0D4B1B68EC
:100BB00013F4805305D03F2805D90B4B0020186053
:100BC000704718467047094B10B5074C53F8303042
:100BD00023600121FFF7BEF8236800221A7001206C
:100BE00010BD00BF3480044024040020F8960100AA
:100BF0000C4B1B6813F4805306D00E2806D00A4A0B
:100C0000537B03F0FE03537300207047074B064AE3
:100C100040F202311960537B43F00103537301200A
:100C2000704700BF3480044000C0064004C0044048
:100C3000034B1B68DB0401D5FFF722BE704700BFE2
:100C40003480044070B5094E04464518AC4204F1A6
:100C500001040AD03368DB04F8D514F8010CFFF75F
:100C60000FFEAC4204F10104F4D170BD34800440A5
:100C700010B5044C237823B101F0DAF92378002B66
:100C8000FAD110BD98040020084B094A1B7810784F
:100C9000DBB2C0B2834202D20138C01A7047054AA3
:100CA0001268013A1044C01A704700BFA404002023
:100CB000990400205C10FF1F064A074B10781B7830
:100CC000C0B2DBB2984202D2044A12681044C01A81
:100CD000704700BF28040020290400205010FF1F87
:100CE00070B4184B184D1B782A78D9B2D2B2914201
:100CF00022D0164B1C68531CA34214D30022134667
:100D00001348C05CC0B2134E2A7032684AB199428F
:100D100038BF0919CB1A104909688B4201D8002342
:100D2000137070BC70473F2B09D90C483F3A0068DC
:100D3000805CDAB2C0B2E6E74FF0FF30F1E7DAB23A
:100D4000DEE700BF28040020290400205010FF1F08
:100D500058040020240400205410FF1F9C0400208D
:100D60000D4A0E4B12781B78DBB29A4211D00C4A16
:100D700011685A1C8A4204D300220A4B985CC0B204
:100D800070473F2AF9D9084A3F3B1268D05CC0B28D
:100D900070474FF0FF3070472804002029040020DE
:100DA0005010FF1F580400209C040020054B064AE9
:100DB0001B7806491268DBB20B700AB1002313706E
:100DC000704700BF290400202404002028040020CC
:100DD00030B43C4B1A79940626D53B4DDC793B4B1D
:100DE00029781A683A4BC9B2481C9042E4B232D30F
:100DF000197801F0FF03002957D000231846354920
:100E00000C542B703449096871B1344B1B78DBB238
:100E1000834284BFD21A1318314A126898BFC31A8A
:100E2000934224BF01230B70264AD378DBB2180605
:100E30001DD45A060DD5234B1B795B0609D5294BCA
:100E400029491B6800220A7003B11A701D4B2C221D
:100E5000DA7030BC70471B789842D3D03F282FD926
:100E6000224B3F391B685C54C3B22B70CAE711791F
:100E70000906DED51E49194C08782178C9B2884286
:100E80001BD01C4A1268481C904210D2272898BFD9
:100E9000C1B20ED9184A27391268525CC1B2D2B217
:100EA0000848D2B2C2712170C3E71846AAE70021F0
:100EB0000846124A125CD2B2F2E76C21D170B8E750
:100EC000C3B29CE700C00640280400205010FF1F5A
:100ED0002904002058040020240400209904002044
:100EE0005810FF1FA0040020980400209C0400203C
:100EF000A40400205C10FF1F540400202C040020D8
:100F0000084B1860084B50B101F140021A60074AC3
:100F1000074B01F11A002831106019607047402218
:100F20001A60F4E79C0400205010FF1F5410FF1FAC
:100F30005810FF1F044B1860044B10B12831196082
:100F4000704728221A607047540400205C10FF1F6D
:100F5000431E032B14D872B60A4951F8230068B116
:100F600070B4094C058834F81320466841F82360B2
:100F7000521B24F8132062B670BC704762B67047EB
:100F800000207047000500200806002001380328D3
:100F90000BD872B6074B53F8203043B100205B6882
:100FA0000130002BFBD162B6704700207047184615
:100FB000F9E700BF54050020F0B472B61A491B4E81
:100FC000012311F8014B194F9A00240742F0010543
:100FD00005D556F8324064B156F83520BAB1013320
:100FE000052BEED162B6124B00221A70F0BC00F055
:100FF00023BD0F4C0F4D217807EB43130830013907
:101000005860217047F8325062B6F0BC7047084A09
:101010000949137807EBC5040830013B6060137081
:1010200047F8351062B6F0E7C89901000000FF1FCD
:101030007D05002088004000C8004000431E032BAF
:101040001DD81B4A400140F0100030B4104472B665
:10105000184CE25C032A1BD8DFE802F002121517D5
:1010600003220D88E25410F0080F14BFC823882310
:1010700043EA054308314160036062B630BC704703
:1010800008300222EDE70522EBE708300422E8E70A
:10109000094A52F8230038B1084A52F82300416047
:1010A00042F8231062B6E9E742F82310034AF7E753
:1010B0000000FF1F8C05002054050020640500205F
:1010C0002DE9F04FDFF814B3DFF814A387B044E044
:1010D000AD4F4FEA930807EBC809013ED9F8042049
:1010E00003F00803F6B2A2F1080003F0FF04002B9E
:1010F00040F0038157F838301B0C99B222F8081CD5
:10110000002B00F0F180A14B22F8064C42F8044C71
:1011100053F82620002A00F06C819D4D55F82630AA
:1011200058609C4C45F8260034F81630194424F8D1
:10113000161000F061FC002800F05481964A974B8D
:1011400019F0080F00F1080018BF1346C9F8040091
:1011500047F8383008238BF800309BF80040E4B2A1
:1011600060071BD58E4B1B78ABB18E490A7802F015
:10117000FF032AB1013BDBB20B70002B00F0B583FB
:1011800089490A7802F0FF032AB1013BDBB20B70F8
:10119000002B00F0F68004238BF8003004F00803E5
:1011A00003F0FF02002B00F0D5809AF80030DBB28C
:1011B0001E098DD19C08744F57F8342007EBC401E9
:1011C000C2F38302013A49680C2A7ED8DFE802F0B4
:1011D00081817D7D7D7D7D7D427D7D7D07000868EF
:1011E000724B734D01936C4B4A68724E47F8343022
:1011F00081B240F281646D4B6A6028600022012058
:10120000A1423A611A60BA61307000F2F680B1F51D
:10121000D06F80F0E882B1F5817F00F0D38200F2D8
:10122000D881802900F04D81822940F09282A988DE
:10123000614B01F07F01042900F28C825F4C890030
:101240000B44227062701A78930740F13883207043
:1012500002203AE1554B01931A6862B3584B594941
:10126000544E18880C7896F800E04028054684F023
:10127000010C28BF402544F00204BEF1000F81F8A4
:1012800000C0A0EB050007EBC40C0CBF8821C821EF
:1012900080B28EF0010E41EA0541CCF8042018809E
:1012A00086F800E02A4447F8341010B9402D18BFE2
:1012B0000022019B1A603E4B1A88B2F5A06F04D140
:1012C00000219A785970404B1A70404A01231370DC
:1012D00040E7374A158842F22100854200F05281EA
:1012E0002D4A47F83420F0E72B4A2C4B19F0080F11
:1012F00018BF134647F838302CE700F09DFB344AFE
:10130000344952F82630002B00F02D8158688C5D4E
:1013100042F8260003F10802C9F80420032C05D87E
:10132000DFE804F0120F150204228A551A8819F01A
:10133000080F0CBF8823C82343EA024347F838301C
:1013400008E702228A55F1E703228A55EEE70522D3
:101350008A55EBE7E00700F17881210600F1A281D0
:10136000A20706D51C4A1D4913780220DBB2137070
:101370000870E30602D5194B10221A7007B0BDE8B9
:10138000F08F00F085FC06E70000FF1F000500203D
:10139000AC04002008060020C8004000880040007F
:1013A000880500201105002090050020A8040020D9
:1013B0007405002010050020C02007408005002093
:1013C000BC0400207C0500209820074094200740A2
:1013D000540500208C05002088200740802007400D
:1013E00090200740B74A47F838001378013313704C
:1013F000B0E643F82600B44D93E642F22104A14240
:1014000000F0AD8000F20E81B1F5086F00F054815C
:10141000B1F5106F40F09D81AC4AA9781170AC4DC8
:10142000042402E00134142C0CD057F8343019068F
:10143000F8D505EBC40301345868083800F0FCFA0D
:10144000142CF2D1A349A44BA44A0291A449A54C5F
:101450009D4D039405964FF0000988461C4616469C
:101460000495206828B1456800F0E6FA2846002D6A
:10147000F9D100232360049B30681A46002342F808
:10148000293028B1456800F0D7FA2846002DF9D157
:1014900000223260029A98F800301146002241F88A
:1014A000042B039A0291023B4FF0000122F819101D
:1014B000032B00F2B481DFE813F0E201AE01E20198
:1014C000AE01894C022022706270EA88824280F06C
:1014D0000D8286490D78402A45F0020E944607EBAE
:1014E000CE0028BF4FF0400C04EB0C034460029385
:1014F000CCEB02004FEA0C484FF001090022C8244F
:1015000044EA080385F0010447F83E3032700C705D
:10151000DFF8BCE1764BDFF8D481002840F0208171
:10152000BCF1400F1BD144F0020407EBC403029F3F
:10153000DFF89CE15F60002A40F02781020442F05E
:10154000880286F800900D7007444EF834203B4620
:10155000402804D10020674A019910800B60664A38
:1015600001231370B1E68B5D032B00F2248101A2ED
:1015700052F823F055110100551101009916010090
:101580009F160100928862B95C4ACD1D11F8013B9B
:1015900002F8013F8D42F9D1594A1268862A00F0BB
:1015A000C9805249524E0878327840F0020580F0E6
:1015B0000100087007EBC501002A4FF000004860E9
:1015C00082F001020CBF8821C82147F83510327023
:1015D00086E640F20232914240F0B080A98801F0E4
:1015E0007F01042900F2B5806A88002A40F0B180AA
:1015F000444C89000C448146217841F0020121705D
:101600000020029080468446044638490D7845F013
:10161000020E07EBCE03B9F1000F5C600CBF88240B
:10162000C8246DE742F22124A14240F08E80A988AF
:10163000002940F04281344B344A354C1B68AD7868
:10164000136081460A462570DAE72B49204B314862
:10165000264EDFF8B0C0304DDFF8D4E02F4F022423
:101660000C702F4C18605C6098602E48D8601A612E
:101670009A610D2332702C4C8CF800302B4EFF23D6
:101680002B7001209F258EF800303A703370257042
:10169000087007B0BDE8F08F00238B555AE5012391
:1016A0008B5557E51749224B80220D2008701A7080
:1016B000A2077FF55EAE55E6044A0B4C1278227005
:1016C00003E700BF7D050020AC0400208805002052
:1016D0000000FF1F640500200005002054050020C5
:1016E0008C05002008060020800500207C050020D5
:1016F00010050020BC040020942007400F060020A5
:1017000010060020C02007409C030020180600207F
:10171000A00500208800400088200740982007404E
:10172000C004002014050020842007408C200740BE
:1017300080200740754A0F21117032E7B1F5A06F84
:1017400007D100224FF001095AE742F221329142BB
:10175000F7D06F4B0F221A706E4A01231370B4E555
:1017600040287FF6E0AE44F002040EEBC401029E76
:101770004E60AAB183F80090674A88F8005033465B
:10178000403840334EF83420E5E6029B86F800905E
:10179000020442F0C8020D7003444EF83420D7E62C
:1017A00083F80090029B5D4A88F80050403840332F
:1017B0004EF83420CFE619F0080F0CBF02230323A4
:1017C0008B55C7E4A98801F07F010429C1D86A8834
:1017D000002ABED14E4C89000C448146217821F06C
:1017E000020121700CE74E4A5468002CB1D0688881
:1017F000B5F804E003E00C325468002CA9D013883B
:101800008342F8D153887345F5D1000A03280CBFF1
:101810002078108959E64FF0010388F8003009F16B
:101820000109B9F1040F04F1040406F1040608F1FA
:1018300001087FF416AE3B4B059E3B4DDFF8F08070
:10184000002018704FF0010918F8013B05F8043B1F
:101850001A0719D44FEA890444F0020244F0030441
:10186000002347F8323047F83430304B9D4209F1BD
:101870000109E9D196F8009089F00102C0E64FF025
:10188000000388F80030CAE700F0B6F818B307EB99
:1018900049134FEA890408305860204B47F8343028
:1018A00000F0AAF868B144F0010307EBC302083066
:1018B0005060194A47F83320CEE78146A0E602205F
:1018C00003E6184B44F001021B7847F83200154A32
:1018D00001331370C0E7134B124A1B784FEA890497
:1018E000013347F834001370DAE700BE402884461D
:1018F00028BF4FF0400C04EB0C03CCEB00004FEA88
:101900000C48029300224FF001097EE611050020E9
:10191000C020074094200740C800400088004000D5
:10192000CC9901007D050020C4200740D420074049
:10193000C89901002DE9F04100F060FC0023234923
:101940001A4601EBC30041F833200133142B4260E7
:101950004FF000041D48F4D11D491E4A0B68DFF802
:101960008C801D4F1D4D1E4EDFF884C0DFF884E0D3
:1019700043F480230B60136843F040731360C0F39B
:10198000072388F8003001F52831C0F307433B7086
:10199000000EFF23CC3102F5C922287002F58472B3
:1019A0008CF800300F4D8EF800300F483370012353
:1019B00008F8083C70260C704FF40014102107F84A
:1019C0002C3C2E7004601170BDE8F0810000FF1FF8
:1019D0003480044000D80040B0200740B4200740C5
:1019E0001020074035E400E004E100E09C200740BF
:1019F000802007408820074072B60D480268B2FA7E
:101A000082F30B2B10DC4FF00041D94022EA010297
:101A1000026062B6074803EBC303DB00C218002173
:101A2000C15010465160704762B60020704700BF39
:101A30006410FF1F9803FF1F0D4B0E4AC31AA2FB31
:101A400003231B090B2B0CD80B4A127852B972B620
:101A50000A484FF00041026821FA03F31A4302607A
:101A600062B67047064A1278002AF0D0FFF7A4BA8F
:101A70009803FF1F398EE3387D0500206410FF1F97
:101A80008805002038B50F4D286878B14388028852
:101A9000C118013393420C7A02D24380204638BDEC
:101AA000FFF7CAFF002320462B6038BD064B1B788A
:101AB0002BB10320FFF74CFA28600028E6D14FF045
:101AC000FF3038BD9C05002088050020044B054AE6
:101AD0001B6890881BB11A885B88D31A184470471A
:101AE0009C050020080600202DE9F04FDFF8F89053
:101AF00083B0012289F80020019169B3DFF8EC80FE
:101B0000364F019E8346D8F80000B0B3344D448868
:101B1000C4F14001B14228BF314604EB010E00225E
:101B20001FFA8EFE2A70761AA0F802E000F1080271
:101B300051B1013C224459441BF8014B02F8014FBA
:101B40008B45F9D1B0F802E0BEF13F0F0BD8254A22
:101B500005211170002ED6D10198002389F800309C
:101B600003B0BDE8F08F4022028001460420FFF759
:101B700065FA0022C8F80020E9E73A782AB3184D40
:101B80004DF2E9044FF0010A07E0013C16D02A7833
:101B9000A2B900F04DFA3A78BAB10420FFF7F6F98D
:101BA0000728F2D889F800A0FFF726FFC8F8000040
:101BB0000028ACD10C4B013C1870E8D101234FF048
:101BC000FF302B7003B0BDE8F08F00234FF0FF30E3
:101BD00089F8003003B0BDE8F08F00BF8805002011
:101BE0009805002090050020910500209405002014
:101BF00038B50E4D0E4C28680123237028B140885B
:101C000000232370C0F1400038BD0A4B1B7813B984
